:020000040000FA
:1000000000F80202D96F0000FD34000079420000C0
:1000100000000000000000000000000000000000E0
:1000200000000000E04E0100284F0100FD340000F8
:100030000000000000000000FD34000075760000A4
:10004000F1320000FD340000FD340000F96F0000C3
:10005000814A0000856B00008D340000813500006E
:100060005918000095170000FD340000013500000C
:10007000554A0000B18C0000796F0000A56F0000A8
:10008000FD340000FD340000FD340000D179000093
:10009000F1790000FD340000FD340000FD34000063
:1000A000897E0000937E0000F33200008D6E000018
:1000B000FD340000ED6B00000000000000000000B7
:1000C0000348854600F016FF0048004785CA000037
:1000D00000F8020230B50B46014600202022012420
:1000E00009E00D46D5409D4205D31D469540491B6C
:1000F0002546954040191546521E002DF1DC30BDB5
:1001000070B500242546002801DA01244042002968
:1001100001DA01254942FFF7DDFFAC4200D0404241
:10012000002C00D0494270BDF8B5002425460029B6
:1001300004DA0E46012400214042B141002B04DACA
:100140001E46002352420125B34100F0D1FC8C46EB
:1001500017461E46AC4203D0002540428D41AC46B6
:10016000002C02D0002657429E4161463A46334653
:1001700001B0F0BD03460B439B0703D009E008C95B
:10018000121F08C0042AFAD203E00B780370401C47
:10019000491C521EF9D27047D2B201E00270401CD5
:1001A000491EFBD270470022F6E710B513460A46F7
:1001B00004461946FFF7F0FF204610BDCAB2401EA4
:1001C0004178401C8A4202D00029F9D100207047B2
:1001D000421C0178401C0029FBD1801A704730B5C1
:1001E00004460020034600E05B1C934203D2E05C1F
:1001F000CD5C401BF8D030BD30B50546002003462D
:1002000000E05B1C934205D2EC5CC85C201A01D173
:10021000002CF6D130BD00000FB400B58DB00990B0
:100220000B9010A900200091C0430A9000200C9070
:1002300006480690064807906A4609A80F9900F0FC
:10024000C1FC0DB008BC04B018470000E50B00006D
:10025000050C0000FFB5002083B0009050680190AD
:1002600091691446002697680498884705460C99BA
:100270000698084305D009E0A169761C04988847D0
:100280000546216A284688470028F5D1681C03D016
:100290000198C00704D017E00020C04307B0F0BDAC
:1002A0002068011D2160006800900DE00198C007E2
:1002B00004D1009805700098401C0090A169761C3C
:1002C0007F1E049888470546002F1CDD681C1AD045
:1002D000069800280FD0E817C00E401941118A0077
:1002E00006994009511840012A1A096801209040D6
:1002F0000142DBD107E00C980028D7D1216A2846BB
:1003000088470028D2D0E169049888470C980028D3
:1003100007D1002E05DD0198C00702D10098002109
:100320000170A068B84204DD0C98002804D0002FAA
:1003300002D00120C043B1E73046AFE770B50646B2
:1003400011F034F9046805460A220021304600F015
:10035000C5FC2C6070BDF8B502464A40D40F42007F
:100360004B0052085B089A4202D2024608461146E8
:100370004A0023D0C30D4A00DDB2120EAD1A202D63
:1003800035DA49020126490AF6058A19002C00D0FF
:10039000524220214F1B1146B9402A411018C20D6C
:1003A0009A4221D0002C17D0012D08DCDA05801AE2
:1003B000D20F8019D207DBB200F0D0FCF8BDDA050D
:1003C000801A012340001B06C01880185A4280186A
:1003D000CA0F1043490007E04908C2071143DA0574
:1003E000801A80194008801800F0B0FCF8BD610048
:1003F0000122511A001BF7E70122D2075140AAE758
:100400000122D2075040A6E7024670B54A40D30FFA
:10041000DB0740002DD04A002AD0010E140E000246
:1004200012020919400A520A8418E501044654438D
:10043000000A120A2E045043A4194219200CC54385
:10044000AA18120C0125AD03521C521912047F394F
:10045000240400D0521C104301D44000491EC2B2F3
:100460000C06C0092018401C4008802A02D003E076
:10047000002070BD40084000002900DA0020184329
:1004800070BD70B502464A40D50F40004A00ED07E6
:1004900040085208002814D0002A12D0C40DD30DF1
:1004A00041020120C0055202490A520AE41A091801
:1004B00012187D34914201D3641C00E04900002CE5
:1004C00001DA002070BD0023914201D3891A034351
:1004D000400849000028F7D100290AD0914202D1F2
:1004E0000121C90705E0914201D2012101E001216A
:1004F000C943E005C018401900F028FC70BD000099
:10050000F0B507460846584087B0C00F0490480031
:100510000E46590040084908BC1A884105D23846A1
:1005200031461E4617460B46024658004008104307
:100530004CD0300D039040055900400D490D0590F9
:10054000401A0290402872DA18030121000B0905B5
:100550000843019004980092002805D00199524266
:100560000020884100920190029840210A1A0199C6
:10057000009800F0EDFA05460C466B4607CB00F0FC
:1005800008FBC0197141039A0E0D0023D71756407E
:100590001A467A40164344D0049A002A2DD0029A73
:1005A000012A039A15DC1205C01A9141012636056D
:1005B000001C7141D20F059ED20700930192029652
:1005C0002A46234600F010FC07B0F0BD38463146FD
:1005D000FAE71605224A0F46B218C01AB7410121A0
:1005E0000905001C4F4100187F4111461818794138
:1005F000E20F10436D19644113E0E2076D081543E3
:100600006408C2071443039A01261205C01A9141D7
:100610003605001C7141CE07400830434908C01818
:1006200051412A46234600F0D2FBCDE7FFE704986C
:1006300001224000C117121A00238B410498314651
:10064000C417381AA141EEE730B40124E40763402F
:1006500030BC55E730B40124E407614030BC4FE7BB
:100660000000E0FFF0B51FB488B00B990998002492
:1006700048400999C00F490049080991C0070B99E2
:100680000090490049080B9109990898A64608432B
:100690001CD00B990A98084318D0099801244000EF
:1006A000420D4800410D099824050003000B20432A
:1006B00009900B980003000B20430B9050181C4925
:1006C0004018002201901446104605E00020014623
:1006D0000DB0F0BD032801DA034600E003239C4679
:1006E000C11A0AAE0AE05F0008ADED5B4F00F75B90
:1006F0007D430027AA187C41491C5B1E6145F2DD41
:10070000410004AB5A522104120C0A43240C401C31
:100710000828DFDB01980290009970460191009053
:10072000059B049A0799069800F05EFBD0E700004D
:100730000DFCFFFFF0B50C465C4085B0E40FE4070C
:1007400003944C0000266408590094464908024668
:100750000296224321D062460A431ED06200570D02
:100760004A000E032303550D012402462C4924059B
:10077000781B1B0B360B4018234326436146009021
:100780001C46501AB44103D30098401C009002E06C
:10079000921800985B41002803DA0020014605B05A
:1007A000F0BD0020012109050746864611E0644698
:1007B0001D46141BB54106D36546521BB341744612
:1007C00007430C43A646CD07400849082843921822
:1007D0005B4105460D43EAD11046184313D06046ED
:1007E000194650407140084306D06046101AB34184
:1007F00006D20122002306E000220123DB0702E0EB
:100800000122D2435310009874460105381C6141FF
:10081000029C039D0019694100F0D9FABFE700006E
:10082000FD0300000122D207002800DB101A002976
:1008300000DB511A814201D8012070470020704727
:100840000122D207002800DB101A002900DB511A10
:10085000814201D201207047002070470122D20757
:10086000002800DB101A002900DB511A814201D355
:1008700001207047002070470122D207002800DBCA
:10088000101A002900DB511A814201D9012070475A
:10089000002070470122D207002800DB101A00292F
:1008A00000DB511A814201D10120704700207047BE
:1008B00010B5002904DB0C460121C9074042A141C3
:1008C000002B04DB1C460123DB075242A341801AA4
:1008D000994101D3012010BD002010BD10B50029A1
:1008E00004DB0C460121C9074042A141002B04DB77
:1008F0001C460123DB075242A341101A8B4101D34E
:10090000012010BD002010BDC217C10F504010B50E
:100910004018CA079623002100F020FA10BD10B538
:1009200000229623114600F019FA10BD0EB5C21729
:10093000C10F5040CA0740180021054B0293019295
:1009400000910A460B4600F04FFA03B000BD0000CC
:10095000330400000EB505490291002100910A46BA
:100960000B46019100F040FA03B000BD33040000D3
:100970003EB5CA17CB0F002450405140C01861410A
:10098000DA07054B0293019200942246234600F0B9
:100990002BFA03B030BD000033040000C20F410049
:1009A00040020123400ADB05D207090EC0187F2947
:1009B00001DA00207047962903DC9623591AC840B3
:1009C00001E096398840002AF4D040427047410047
:1009D00040020122400AD205090E80187F2901DA5F
:1009E00000207047962903DC9622511AC8407047B0
:1009F000963988407047000070B5CD0F4A00090352
:100A00000123090B1B0519430B4BED070024520D65
:100A10009A4201DA002070BD074B34339A4203DC5E
:100A20009A1A00F0A5F802E00449511888402C43B6
:100A3000F1D0404270BD0000FF030000CDFBFFFF7E
:100A400070B5CD0F4A0009030123090B1B0519439B
:100A50000D4BED070024520D9A4202DA00200146A8
:100A600070BD094B34339A4203DC9A1A00F080F8C7
:100A700003E0064BD21800F06BF82C43F0D00022B4
:100A800040428A41114670BDFF030000CDFBFFFFCD
:100A9000C20FD207400040080BD0C10D0723DB0175
:100AA000C91840020905400A1143C2084007114312
:100AB0007047002001467047CB0FDB07490010B597
:100AC000490802460A4307D00A0D07240903E40136
:100AD000090B121B002A01DC002010BDC900440FC5
:100AE0000C43C100E018D205801800F02FF910BDAA
:100AF000F0B51FB40646002082B00546402401919F
:100B000000901BE0019922460F46304600F030F875
:100B1000049A059B801A994110D310461946224623
:100B200000F016F8361A8F41019722460120002165
:100B3000009F00F00DF838184D4100902046641ECB
:100B40000028DFDC019B00982946324607B0F0BD43
:100B500010B5202A04DB0146203A9140002010BD48
:100B6000914020239C1A0346E3401943904010BD56
:100B700010B5202A04DB0846203AD040002110BDE1
:100B80000B46D340D0402024A21A91400843194676
:100B900010BD10B5202A06DBCB170846203A1041BD
:100BA000C1170B4306E00B461341D0402024A21A84
:100BB00091400843194610BD02681378511801602E
:100BC0001846704710B5D16004495161044911625B
:100BD00000211161114600F0ADF910BDB90B000004
:100BE000210F00004268002A08D001680B78491CD8
:100BF000002B03D0521E06C0184670470121C16069
:100C0000881E70474268002A0BD0C3680168002B19
:100C100007D183688B4204D0491E521C06C00020B5
:100C200070470020C04370470FB400B589B00A4632
:100C30000DA9009100230C99002ACB60234B069349
:100C4000234B079301D0042300E00023214A0292A2
:100C5000214A0892019302466B46002000F095FB62
:100C600009B008BC04B01847F0B585B007460020AD
:100C7000C04301901E46002015460C46009102918B
:100C800004903B466A46314604A8FFF7CDFF04991D
:100C900002466018002D05D0002901D0034600E06F
:100CA00023462B6000290ED0002A02DD00998142E4
:100CB00009D0001B019000943B466A4631460294DD
:100CC00004A8FFF7B1FF05B0F0BD0000E50B000080
:100CD000050C0000FFFFFF7F210F0000F7B5009C0F
:100CE0000F4600262578641C002D05D000F014F96D
:100CF0000068405DC007F5D12B2D02D02D2D18D0F6
:100D0000641E39462046029A00F06AFC002F04D087
:100D10003968A14201D10099396071050224002986
:100D20000BDA4042002803DD10F040FC0460A0070D
:100D3000FEBD012080020643E3E70028F8DA10F048
:100D400035FC04600048FEBDFFFFFF7F002904DA88
:100D5000401C490001D140084000704770B4002495
:100D6000050C05D11024000402D1002921D0112442
:100D7000050E01D100020834050F01D10001241D28
:100D8000850F01D18000A41C002801DB4000641CF9
:100D9000002908D020252E1B0D46F540A14000D08B
:100DA00001212943084301061B1B000ADB1D02D554
:100DB000002070BC7047DB05181880180029F8DA8D
:100DC000401C4900F5D170BC40084000704710B588
:100DD000002B08DA0024401C614192185B411A4341
:100DE00001D14008400010BDF0B51FB482B00546E7
:100DF0000C0003D0084610F0C1FB02E010F0BEFB6F
:100E000020300246009021462846FFF7A1FE049BB1
:100E1000059A04460F4618431143084314D0184658
:100E200010431BD0009840210A1A18460599FFF775
:100E30009FFE05460E46009A05990498FFF788FE26
:100E4000084305D0012004E02046394607B0F0BD34
:100E50000020C11705430E432C43374300990E98D9
:100E60006305401A7905E40A00220C43FD0A0A30A2
:100E700002D500200146E9E70105101969410C9CE3
:100E80000D9D00196941FFF7A2FFDFE74A00090342
:100E90000123090B1B0519430A4B10B5520D9A4249
:100EA00002DA0020014610BD064B34339A4203DCBF
:100EB0009A1AFFF75DFE10BD034BD218FFF748FEEC
:100EC00010BD0000FF030000CDFBFFFF10B500299F
:100ED00004DB0124E40740428C412146002B04DB63
:100EE0001C460123DB075242A341994200D19042A4
:100EF00010BD0000064C0125064E05E0E36807CC56
:100F00002B430C3C98471034B442F7D3FFF7DCF87E
:100F1000244901004449010000487047481F01006E
:100F200010B50446FFF7F8FF0068005DC007C00F6A
:100F300010BD0000F3B58DB000200A9001200B9089
:100F4000002608460C300C46099062690121099878
:100F50009047051E2ED0252D2DD0216A88470028C8
:100F600018D06269012109989047216A88470028B2
:100F7000F7D1411E62690998904700E0761CA1698B
:100F80000D988847216A88470028F7D1E1690D98B4
:100F90008847DAE7A1690D9888470746A84201D13A
:100FA000761CD2E7E1690D9888477F1C02D10A9828
:100FB000002877D049E1002762693D463946099803
:100FC00090472A280CD16269012109989047012590
:100FD00006E00A214F433F18303FEBD41020054371
:100FE0006269012109989047014630390A2903D2E4
:100FF0009B498F42DEDCECE7E90600D4994F6C2870
:101000000AD04C2810D0682824D06A282ED0742802
:101010000CD07A280AD00DE0626901210998904726
:101020006C2823D004211CE02020054362690121A3
:1010300009989047A760656065284FD026DC58283E
:1010400039D01ADC452849D012DC252834D0412873
:10105000B0D143E06269012109989047682802D025
:1010600008210D43E6E70120C002DEE70220DCE7AD
:10107000462833D047282CD130E05B2870D0612837
:101080002CD063286CD0642823D161E06F284FD026
:1010900009DC662822D0672820D0692826D06E284F
:1010A00017D12EE0CDE070284DD073286FD0752871
:1010B0004ED078280DD154E0A1690D988847054697
:1010C000252800D16CE7E1690D9888476D1C00D197
:1010D0006DE7BAE00A224CE00A2252E001202346E2
:1010E0006A46C0430D9900F050F9A3E0284640211C
:1010F00008436060A807234601D5002239E000229A
:101100003FE0E80700D020E72068011D216000686B
:10111000290501D5067018E7290701D5068014E7CF
:10112000A90703D5F117066041600EE706600CE7DA
:101130002846402108436060A807234601D50822BD
:1011400017E008221DE0484928460840606016E084
:101150002846402108436060A8072346BCD5B9E76C
:1011600015E02846402108436060A80707D52346BC
:1011700010220120C0430D99C046C0465AE02346C4
:1011800010220120C0430D99C046C04652E0002104
:101190000C910B460091632802D05B2807D043E0F6
:1011A000E80601D40120A060012000903CE06269C3
:1011B0000121099890475E2805D101200C90014635
:1011C0006269099890472169002906D10B4601AA56
:1011D0008F00491CD3510829FADB002835D021693A
:1011E00000290ED1C117C90E09184A11930001AA8E
:1011F0009A1849094901411A01201368884003439C
:10120000136062690121099890475D28E5D10C9827
:10121000002808D0002001AB81005A58401CD2435E
:101220005A500828F8DB01AB01202246C0430D9933
:10123000FFF710F800280ADA401C06D10B980028A6
:1012400003D00020C0430FB0F0BD0A98FBE7E907C8
:1012500002D10A99491C0A91361800200B9074E6B5
:10126000CCCCCC0CFFFFFF7FF1F7FFFFFFB5087878
:1012700089B01546FF2805D0491C2D2804D000222E
:10128000002407E000240BE00122F9E70A235C4375
:101290000419491C0878FF28F8D1002A00D06442BC
:1012A000002004902A7801462D2A01D02B2A0FD144
:1012B0006D1C2D2A02D00022049209E00122FBE7D6
:1012C00000260A2233466D1C00F0DDF93818714102
:1012D0002F78FF2FF4D10C9AA218069202460A43E7
:1012E00004D0FF23069A9133DA4205DA00210998E7
:1012F0000A4606C00DB0F0BD0024B74AB54D2646DB
:10130000079200F00DFA029006980391002801DA86
:10131000474200E0074639050020AF4A001C514112
:101320000191009012E0F80707D022462B46304684
:101330000799FFF797F90646079122462B46104674
:101340001946FFF78FF904460D467F10002FEAD1AA
:101350000698019B0028009A0399029806DAFFF785
:10136000E9F93246079BFFF7E5F905E0FFF77AF95F
:101370003246079BFFF776F9049A002A02D0012231
:10138000D2075140099A03C2B4E7FFB591B00020DB
:1013900009900025ED432E209E685C681F46019051
:1013A000B9696D1C129888470090396A88470028EF
:1013B000F6D10098401C0AD00D20C0018443002EB5
:1013C00012DD00982B2809D02D280DD103E0002034
:1013D000C04315B0F0BD012080020443B9696D1C03
:1013E00012988847761E009003A9600501D52D202C
:1013F00000E02B206A461073491C0CA80F91029044
:101400000AE0B9696D1C12988847009001204002DB
:1014100004431398761E0560002E02DD00983028E4
:10142000EFD001990098884245D18020044308E01C
:101430000998401E09900120400204431399681C3A
:101440000860B9696D1C761E129888470090302894
:10145000EED030E00199884205D1200603D48020E7
:101460000443761E1DE0009810F06EF9002825D088
:10147000012149020C43009807AA0F990332303822
:10148000761E914208D208700F98401C0F902006DB
:1014900007D50998401E03E0200602D40998401C95
:1014A0000990A00502D51399681C0860B9696D1CE4
:1014B000129888470090002ECCDC59E0002E57DDB2
:1014C0000098652801D0452852D1A00550D50320A9
:1014D00000028443B9696D1C761E129888470090FB
:1014E000002E0CDD2B2804D02D2808D1FF20013040
:1014F0000443B9696D1C12988847761E0090E00578
:1015000001D52D2100E02B21029801700298401C8A
:101510000290019025E00120400204430EA90298A8
:101520000131761E88420ED20098029930380006AA
:10153000000E087003D10299019881420AD90298DD
:10154000401C029006E0E00501D5244801E0234854
:1015500040420990B9696D1C129888470090139811
:101560000560002E04DD009810F0EEF80028D2D1BE
:10157000F969129888470F99FF200870029903AA09
:10158000087000200A900B900CA90AA8099BFFF78D
:101590006DFEA00502D40120C0431AE724200442B6
:1015A00009D0E00713D138680B9A0A99031D3B60F4
:1015B000006806C00BE00B990A98FFF77DFA014618
:1015C000E00704D13868021D3A60006801602846CF
:1015D000FFE60000000014400000F03FF1D8FFFFDC
:1015E000F7B582B0029C00272078641C154601974D
:1015F000302802D0002D15D015E020780127641C7A
:10160000782804D0582802D0002D09D00BE0002DF6
:1016100001D0102D07D1002710252078641C02E08E
:10162000082500E00A250026009610E00099012711
:1016300069430818020C294680B2714300908E1845
:101640003804864201D3012001902078641C294689
:1016500000F056F80028E9DA0398002805D0002F9A
:1016600001D0641E00E0029C04600198002806D0AE
:101670000FF09CFF02210160C81E05B0F0BD00996B
:1016800030040843F9E7F0B51FB486B0002000909D
:10169000019002900698069980B204900798090C70
:1016A00002040014114307900027089D0998069131
:1016B0003E463C4603900398A9B20204000C0390F6
:1016C00004982D0C1543484300212246FFF740FAA9
:1016D000C719714110340E46402CECDB3846029A93
:1016E000FFF736FA009A019B801800905941029842
:1016F0000191103002904028CCDB00980BB0F0BD77
:101700003A2800D23038202302469A43412A01D396
:1017100010463738884201D30020C043704700008C
:101720000EB5054A02920022009213460192FFF77D
:101730005BFB03B000BD00003304000070B58C18E3
:101740000578401C6B075B0F01D10378401C2A1100
:1017500006D10278401C03E006780E70401C491C3C
:101760005B1EF9D12B0705D40023521E0DD40B703C
:10177000491CFAE70378401CCB1A921C03E01D7841
:101780000D70491C5B1C521EF9D5A142D8D3002014
:1017900070BD000010B52148016A8A0715D44A07B8
:1017A00015D4C90732D01E498A89002A15D0531E84
:1017B0008B8182688C6904C48C610A691B040DD01A
:1017C000002A22D10121016010BD022100E0042184
:1017D000C16113488021416110BD0A69012A09D104
:1017E000026801239A430260C361FF206830993088
:1017F0000C4A106001204861CA69002A05D0886936
:1018000009898B00C01A904710BD10BDFF226832B5
:10181000054806A109A30DF049FBC04608D00140C8
:101820009895010280E200E09C2E01004144435F54
:1018300049525148616E646C65720000556E65785E
:101840007065637465642041444320696E746572F9
:10185000727570740D0A000070B582B00023019398
:10186000444801688A6A4C6813252540132D02D12B
:10187000CB689B07DB0F4361930772D453070AD4ED
:10188000D30711D1130724D5048F838E1C1B102C72
:101890000EDD102310E0042088620220032142A202
:1018A0000EF060FB02B070BD0120886202B070BD16
:1018B000048F1B1B1C0610D0DBB20024058FC66AE8
:1018C00075192D5D0D74641CA342F7D1048FE318C4
:1018D0000387D20607D400212FE04B6A0824A343D4
:1018E0004B62D206F7D5CB68C28E448F141B5B04C3
:1018F000DB0EA34201D3438FD31ADAB2002A16D0EB
:10190000097D438F046BE1540199012A10D0012312
:101910001C46890145582D7D41184E8F9B19096B36
:10192000CD54641CE3B201999A42F2D800E0002140
:101930008B01C3185C8FA2185A878A0181184B8FBC
:10194000CC8EA3420BD301230B618058002242624C
:10195000CA6B002A03D03A31098801A8904702B027
:1019600070BD02208862044804A1084A08A30DF053
:101970009DFAC04670900102B52E01004145535FAB
:1019800049525148616E646C65720000CE020000DD
:1019900041455320696E707574206F766572666C70
:1019A0006F770D0A00000000414553206F75747079
:1019B000757420756E646572666C6F770D0A000031
:1019C000F0B581B001243F2900D993E00346806837
:1019D000456B2D688E0001A7BE59B7461B1B000042
:1019E000371B0000131B0000131B0000F51A00003A
:1019F000F51A0000F51A0000F51A0000F51A0000AB
:101A0000F51A0000F51A0000F51A0000F51A00009A
:101A1000F51A0000491B0000651B0000F51A0000C4
:101A2000F51A0000F51A0000F51A0000F51A00007A
:101A3000F51A0000F51A0000F51A0000F51A00006A
:101A4000F51A0000F51A0000F51A0000F51A00005A
:101A5000F51A0000F51A0000F51A0000F51A00004A
:101A6000F51A0000F51A0000F51A0000F51A00003A
:101A7000F51A0000F51A0000F51A0000F51A00002A
:101A8000F51A0000F51A0000F51A0000F51A00001A
:101A9000F51A0000F51A0000F51A0000F51A00000A
:101AA000F51A0000F51A0000F51A0000F51A0000FA
:101AB000F51A0000DD1A0000DD1A0000DD1A000032
:101AC000DD1A0000DD1A0000DD1A0000DD1A00003A
:101AD000DD1A0000DD1A0000DD1A0000434800692D
:101AE0000024022809D001280DD0002802D103CA01
:101AF00004F0ACFF204601B0F0BD03CA04F098FF2B
:101B0000204601B0F0BD03CA04F0B6FF204601B084
:101B1000F0BD022931D0022430E0344D00242C6184
:101B20006C619849354A01F065FE6869401C68613E
:101B3000204601B0F0BD01F097FE284602F004F9FE
:101B40000024204601B0F0BD284909690C234B430D
:101B50002749CA58C918496801F04CFE002420469C
:101B600001B0F0BD0024204604F03EFF0128C1D1A1
:101B70001E483030204900241CE001241B490F6915
:101B80000C26314679431A4A51188968214208D0F7
:101B900000247D1C15490D614C61042D10D315499D
:101BA00006E012494869401C4861032812D32949BC
:101BB00000241846224602F077F8204601B0F0BD16
:101BC0006E430B498A598919496801F013FE204672
:101BD00001B0F0BD0E20009000240A2228462146C4
:101BE00002F052F8204601B0F0BDC046DC99010277
:101BF0004C1F01004C2601002C2601001A3A01005E
:101C0000B0B504290FD804468068C04679440979E4
:101C100049008F44020A0E1C1700104910A201F05F
:101C2000E9FD0020B0BD0120B0BD01F01DFE002087
:101C3000B0BD00250321284604F0E6FE06492046F3
:101C40002A4602E003490022204602F02DF8002037
:101C5000B0BDC0463C260100BC2601008813000030
:101C6000415445300D0A0000B0B582B001240A2964
:101C700010D883687944097949008F440E290505F5
:101C80000B0B0B0B0B0B1A00194909680024224699
:101C900002F00AF8204602B0B0BD5068144908604E
:101CA000144915A2184601F0A5FD0024204602B0F3
:101CB000B0BD0024019403CA09A201AB02F012F9DD
:101CC0000228E7D1019804F0F3FE204602B0B0BD2F
:101CD000184601F0C9FD0024204602B0B0BDC04640
:101CE0002B4353513A2025642C252A0D0A0000006D
:101CF000F89A01028813000041542B4353510D0AF6
:101D000000000000B0B582B00546002404F0CAFE11
:101D100001280DD108498C60E86B426853684B601C
:101D2000009401926A4601F0BFFF204602B0B0BDA8
:101D3000E443204602B0B0BDC4930102B0B50546ED
:101D4000881E02280AD3A868012913D0002915D1BA
:101D50000C490DA201F04EFD0020B0BD022001464D
:101D600004F052FE064900242846224601F09CFF5A
:101D70002046B0BD01F078FD0020B0BD0120B0BD0F
:101D80000C2601008813000041542B4346554E3D5C
:101D9000300D0A00B0B5E0B00324E1016D462846DD
:101DA0000FF0D4FB204621462A460EF0DBF8002037
:101DB00060B0B0BDF0B597B00820149064201390C7
:101DC0002548109002200E904B20C0011690234D04
:101DD00028461430129001270F97B8021190032063
:101DE0000EA906F053F90026F443002802D020463D
:101DF00017B0F0BD0C35284601F0B4FF0028F6D12D
:101E000080200C9016490B910A90164809901648AC
:101E100008901648079016480690392005901548F6
:101E20000490154803900D95144D03A9284601F020
:101E30004BFD0028DBD1009501970F4C104911A2F2
:101E4000124B204601F0E4FE1149204601F014FF38
:101E50003446204617B0F0BD78C001025497010205
:101E600078C40102F8C40102452F0000952F00003C
:101E7000152F0000CC2701000C9A010288C901022D
:101E8000AC2501004149523738304500CC260100CD
:101E9000951D000010B50348002404700EF0F2FFF9
:101EA000204610BD109F010280B501F053F90020BB
:101EB00080BD0000F0B58DB00E4600270C970B9743
:101EC0000A970997089707970697059702908068E1
:101ED0000490406B0068019004F080FD04465BA113
:101EE00005220392FEF788F95A4D00281ED05AA108
:101EF00005222046FEF780F9002817D058A10522B8
:101F00002046FEF779F900280FD059A10522204676
:101F1000FEF772F9002809D057A105222046FEF7E6
:101F20006BF9002807D156A500E04FA505A8202190
:101F30002A4602F0A9F801203F2E00D936E0C0461B
:101F40007E4436797600B7443340474A57313131C1
:101F5000313131313131653031313131313131313E
:101F60003131313131313131313131313131313161
:101F700031313131313131313131313131311F1F75
:101F80001F1F1F1F1F1F1F1FBE48416A04290CD19E
:101F9000039A426287620C2050433D490A58081850
:101FA000416805AB049801F025FC38460DB0F0BD42
:101FB000B44C00206062A062CD49364A049801F01A
:101FC00019FCA06A401CA062EFE7049801F04CFCE9
:101FD000019801F0B9FEE8E7AA48406A05E0A9497E
:101FE000486A01220243032A1CD1A649421C4A62C4
:101FF0008F62062ACFD30BE0A2494A6A012013461A
:102000000343052BD2D1501C48628F62062803D3AC
:102010001E490DE09B48406A0C2141431C48425830
:102020004018BDE7886A401C8862032805D316491A
:102030000022029801F038FEB7E70E200090002140
:102040000A220198029B01F01FFEAEE734363030C1
:1020500030000000423A01003436303032000000D7
:102060003436303031000000554E494E45540000A2
:102070003436303036000000343630303300000063
:1020800043544E4554000000AC250100FC250100DE
:102090007C1F0100C239010070B5022956D30F29F7
:1020A00007D1784C217A012905D1002222728F496B
:1020B0004AE0012070BD866801F07AFE002004F03D
:1020C0009BFC012803D10020032104F09DFC002586
:1020D000284604F089FC012804D130346A490022E2
:1020E000204631E0304600F0EBFD00282ED030468F
:1020F000FFF708FE002829D004F090FC012807D142
:102100005F498D60F06B4268E26252684A601AE093
:10211000022004F069FC012808D159498D61F06B57
:102120004268E26252684A6110310CE0022004F019
:1021300063FC01280AD152498D62F06B4268E26269
:1021400052684A6220312A4601F0AEFD002070BD7F
:1021500010B582B003460120272931D87944097986
:1021600049008F442C132D2D162D2D2D2D2D2D2D69
:102170002D2D2D2C2D2D2D2D2D2D2D2D2D2D1C2DA1
:102180002D2D2D2D2D2D2D2D2D2D2D2904F0D2FF72
:1021900015E0DF490022184601F086FD0FE000201F
:1021A000019003CA08A201AB01F09CFE012806D1F0
:1021B000019805F0DBF802E00248012101720020DD
:1021C00002B010BDDC9901022B51495552433A200F
:1021D00022636C6F736564222C25640D0A00000075
:1021E000B0B502294AD30F2914D18568002004F024
:1021F00003FC012803D10020032104F005FC002486
:10220000204604F0F1FB012806D1D94830301E49A0
:10221000002231E00120B0BD2846FFF773FD002801
:102220002CD004F0FBFB012808D115498C60E86B29
:102230004268CF4BDA6252684A601CE0022004F028
:10224000D3FB012809D10E498C61E86B4268C84B69
:10225000DA6252684A6110310DE0022004F0CCFBD2
:1022600001280BD106498C62E86B4268C04BDA62E8
:1022700052684A622031224601F016FD0020B0BDAE
:102280003C900102DC9901022C26010080B5022954
:1022900005D3042905D19E49002201F005FD002047
:1022A00080BD012080BDC046B0B50546881E02280D
:1022B0000AD3A868012913D0002915D10C490DA211
:1022C00001F098FA0020B0BD0220032104F09CFB2D
:1022D000064900242846224601F0E6FC2046B0BD0F
:1022E00001F0C2FA0020B0BD0120B0BD4C260100B3
:1022F0008813000041542B4346554E3D310D0A00D2
:1023000010B50F290BD001291DD000291DD1FFF7D1
:10231000C1FD0020022104F077FB002010BD04461F
:10232000002004F061FB012803D10020022104F009
:102330006BFB002004F060FB012804D1044900225B
:10234000204601F0B1FC002010BD012010BDC046A8
:102350003C260100F0B581B00124322928D8054679
:102360008768786B0668C0467944097949008F44CC
:102370002F3F1919191F1F1F1F1F1F1F1F1F221F4C
:102380001F1F1F1F1F1F1F1F1F1F1F1F1F1F1F1F5D
:102390001F1F1F1F1F1F1F1F1F1F1F1F1F1F1F1F4D
:1023A0001F1F26001E4900242846224601F07CFCFF
:1023B000204601B0F0BD1B48017800291FD0184904
:1023C00000242846224601F06FFC204601B0F0BDF3
:1023D0000024FC623969384688470028FAD0114841
:1023E0000470FC62FFF756FD0E20009001220EE003
:1023F000304601F0A9FC0024204601B0F0BD0121C7
:102400000170FFF751FD0E20009000240522304698
:1024100021462B4601F038FC204601B0F0BDC046F5
:10242000CC250100FC9A010210B586B003460120BC
:102430003B2900D956E0C0467944097949008F44C8
:10244000505051513351515151515151515151519C
:10245000515151515151515151515151515151516C
:10246000515151515151515151515151515151515C
:102470005151515151391D1D1D1D1D1D002005902B
:1024800003CA02AA009218A205AB01F02BFD022894
:1024900027D1039A029817A1FDF7AEFE002820D19C
:1024A000059804F063FF1CE0B5490022184601F0CE
:1024B000FBFB16E0002002900590049003CA05AAD9
:1024C000019204AA00920DA202AB01F00BFD0328B9
:1024D00007D1049A0599029805F014F8029804F0BF
:1024E000B3FF002006B010BD25642C2025700D0A16
:1024F00000000000434C4F53454400002B5245431D
:10250000454956452C25642C25643A0D0A2565005D
:102510001C260100012901D80020704701207047C6
:10252000B0B50546881E03280BD2104604F07EFA8B
:102530000F48C16A00242846224601F0B5FB204618
:10254000B0BDAC6801290BD000290ED104F048FAC7
:102550000346084908A2204601F04CF90020B0BD0E
:10256000204601F081F90020B0BD0120B0BDC04679
:10257000DC9901028813000025730D0A0000000099
:1025800070B582B001240F293DD803468568686B79
:102590000668C0467944097949008F4407141E34FF
:1025A0003434342F373434343434434E66480024C2
:1025B00004708461C461012101716649664A28463C
:1025C00001F018F91FE0284601F04EF9304601F0FD
:1025D000BBFB0024204602B070BD5B4800240471A0
:1025E0008269042111430278002A2ED0052958D18E
:1025F000016A491C016259D2624961E0524B187864
:102600000024002831D0204602B070BD4E4B18780F
:10261000012816D103CA183351A201F063FC00202F
:1026200002B070BD48480024846101210171007826
:102630004849002812D1484A11E0434E3079002819
:102640001BD00024204602B070BD052932D10024E1
:10265000012101708461C46101713E493F4A2846ED
:1026600001F0C8F8204602B070BD03CA183340A27A
:1026700001F038FC204602B070BD002004F0BCF927
:10268000012803D10020032104F0BEF900242046D4
:1026900004F0AAF9012816D130362D49002430461D
:1026A0004BE000210162C169491CC1610E2000900C
:1026B00000241CE0C169491CC161652915D330495A
:1026C0000024184639E02846FFF71CFB00289AD062
:1026D00004F0A4F9012812D11C4900248C60E86B95
:1026E0004268F26252684A6027E00E20009002229F
:1026F0003046214601F0C8FA204602B070BD0220E3
:1027000004F072F9012809D1104900248C61E86BAA
:102710004268F26252684A6110310EE0022004F011
:102720006BF9012800D06EE7084900248C62E86B41
:102730004268F26252684A622031224601F0B4FADD
:10274000204602B070BDC046DC9901023C900102F7
:102750002C26010088130000DE390100E939010050
:102760002B43475245473A20252A2C256400000078
:102770002B435245473A20252A2C256400000000AF
:102780001C260100DC250100B0B584B001243B29E2
:1027900000D937E0134605468068C0467944097978
:1027A00049008F444B5532322F2F2F2F2F2F2F2F91
:1027B0002F2F2F2F2F2F2F2F2F2F2F2F2F2F2F2F29
:1027C0002F2F2F2F2F2F2F2F2F2F2F2F2F2F2F2F19
:1027D0002F2F2F2F2F2F2F2F2F2F1D1D1D1D1D1D75
:1027E0000024039403CB01AA00921C4A03AB01F01E
:1027F00079FB022806D1029A019819A1FDF7FCFC89
:1028000000280FD0204604B0B0BD1848006804F07E
:10281000ADFD174900242846224601F045FA20461E
:1028200004B0B0BD1148006804F0A0FD10490022BA
:10283000284601F039FA204604B0B0BD0B490B60C0
:102840001E210CA200F0D6FF0024204604B0B0BD2B
:1028500001F00AF80024204604B0B0BD423B01005C
:10286000434C4F5345204F4B00000000009B01029A
:10287000EC25010041542B434950434C4F53453DF7
:1028800025640D0A00000000F0B589B0044601205F
:102890003B2900D9AAE01646A7687A6B1568C0469E
:1028A0007944097949008F44536AA071A1A1A1A17B
:1028B000A1A1A1A1A1A18AA1A1A1A1A1A1A1A1A11F
:1028C000A1A1A1A1A1A1A1A1A1A1A1A1A1A1A1A1F8
:1028D000A1A1A1A1A1A1A1A1A1A1A1A1A1A11D1DF0
:1028E0001D1D1D1D0027089703CE06AA0092414A10
:1028F00008AB01F0F7FA022877D13F48056808983D
:10290000854272D1079A069E3CA130460592FDF79A
:1029100073FC002847D03DA13046059AFDF76CFCBA
:10292000002840D03CA13046059AFDF765FC002800
:10293000314E5AD1284604F033FD7068401C706057
:1029400003283CD303207060306804F0B1FC36E00B
:1029500029480660304604F0FFFC059026480068D0
:1029600004F0CEFC04902448006804F0D5FC0499DF
:10297000019102900598012827D02EA026E0384624
:1029800000F072FF284601F0DFF92EE01A4D2868AA
:1029900004F006FD6868401C686003280FD300221D
:1029A0006A6022490DE0144E7760284604F00EFD5F
:1029B000306804F04DFE002801D01B4900E00C49AE
:1029C0000022204601F070F90FE019A000901A498A
:1029D0001AA23846334600F00DFF0E200090002169
:1029E000B4222846234601F04FF9002009B0F0BD7B
:1029F000EC250100423B0100CC970102414C5245BD
:102A000041445920434F4E4E45435400434F4E4E90
:102A1000454354204F4B0000434F4E4E45435420F6
:102A20004641494C000000008C260100AC25010005
:102A300054435000554450008813000041542B4328
:102A4000495053544152543D25642C222573222C65
:102A5000222573222C25750D0A000000B0B582B026
:102A600014468A1E022A12D38568012917D000292C
:102A70001CD1204604F036FC00901E210EA22846F0
:102A8000234600F0B7FE0024204602B0B0BD09493D
:102A90000024224601F008F9204602B0B0BD2846C5
:102AA00000F0E2FE0024204602B0B0BD0124204622
:102AB00002B0B0BD9C26010041545E4845415254CD
:102AC000434F4E4649473D312C25642C25750D0A50
:102AD00000000000F0B583B014468A1E022A1CD301
:102AE0008568012921D0002926D1164F3C60204657
:102AF00004F0EAFBFDF76CFB0646386804F0E4FBE3
:102B00007108009101901E210FA22846234600F073
:102B100071FE0024204603B0F0BD0949002422467E
:102B200001F0C2F8204603B0F0BD284600F09CFE3C
:102B30000024204603B0F0BD0124204603B0F0BDC0
:102B4000EC250100049B010241545E48454152546A
:102B5000424541544845583D25642C25752C257324
:102B60000D0A0000F0B585B0044601203B2900D9CC
:102B700085E0A5687944097949008F443F547F5B1B
:102B80008080808080808080808080806080808065
:102B90008080808080808080808080808080808035
:102BA0008080808080808080808080808080808025
:102BB00080801D1D1D1D1D1D0020049003CA02AA3A
:102BC0000092304A04AB01F08DF9022856D12E480C
:102BD00085680498854251D1039E029F2BA13846F7
:102BE0003246FDF709FB00283AD02AA13846324682
:102BF000FDF702FB002841D128461DE0224CA260CF
:102C0000104604F095FB002838D001F0D4FAE060BB
:102C1000002833D0A36840680090234923A22846A7
:102C200000F0E8FD2AE018480021C160284600F0C5
:102C30001BFE23E01448806804F098FB19E000F0C4
:102C400083FE012804D11048C16803C900F084FF45
:102C50000D48C0680CC81349284600F00BFE0DE073
:102C6000284604F065FB0028074907D0C96801F031
:102C700078FA0B490022204601F016F8002005B032
:102C8000F0BDC046423B0100CC97010253454E4483
:102C9000204F4B0053454E44204641494C00000014
:102CA000EC250100204E00008813000041542B4306
:102CB000495053454E443D25642C25750D0A0000AE
:102CC000F0B583B0074601F073F80026304604F0F3
:102CD00039FB032835460BD10421284604F0A8FC13
:102CE000F86B51492A4600F0DFFF304603B0F0BDD3
:102CF00002970024204604F025FB0428254609D12C
:102D00000298C06B49492A4600F0CEFF264630465D
:102D100003B0F0BD0027384604F014FB05283D46FB
:102D200009D10298C06B40492A4600F0BDFF3E46DB
:102D3000304603B0F0BD01970125284604F002FBA0
:102D40000328029FC8D00125284604F0FBFA042876
:102D5000D6D00125284604F0F5FA0528019FE0D0D9
:102D60000225284604F0EEFA0328029FB4D002257B
:102D7000284604F0E7FA0428C2D00225284604F0C9
:102D8000E1FA0528019FCCD0254C2068401C032186
:102D9000FDF7B6F90D46084604F0D4FA0628029F5E
:102DA00008D1284604F0C4FA002803D001F003FA41
:102DB00000282AD1681C0321FDF7A2F90D46084618
:102DC00004F0C0FA062808D1284604F0B1FA002819
:102DD00003D001F0F0F9002817D1681C0321FDF79A
:102DE0008FF90D46084604F0ADFA0021CE430628BF
:102DF00000D07AE7284604F09BFA002800D174E757
:102E000001F0D9F9002800D16FE72560F86B05497A
:102E10002A4600F049FF0026304603B0F0BDC04608
:102E2000089B0102AC2601006C2601007C260100F3
:102E300080B58AB00620042108F09CFE4B20C0011A
:102E400009900820079064200690B448143005903B
:102E50000648039002200190012002908002049015
:102E6000032001A905F012F90AB080BD78C0010263
:102E7000B0B582B001220F293ED803468068446B6A
:102E80002468C0467944097949008F44071F2527E3
:102E9000343535353535353535350A152749002270
:102EA00004E02649CA68092A20D8521CCA6016497B
:102EB000164A00F09FFC1EE0002003F095FD01285B
:102EC00019D11E4830300E49002212E000F0CCFC2F
:102ED000204600F039FF0EE00D4908E00E2000907A
:102EE00000210122204600F0CFFE04E00549002227
:102EF000184600F0D9FE0022104602B0B0BDC04610
:102F00002C2601000C26010088130000F539010071
:102F1000BC25010080B5032005F0A0F880BD0000AD
:102F20000648416B0020002905D0054A914203D094
:102F300049680029FAD1704701207047DC990102E5
:102F4000FC250100B0B514460D460846114600F0B8
:102F5000B0FF012816D1285D002813D1002C0BD01A
:102F60006019401E00780A2806D10320084A01464D
:102F70002B460CF0F7FF05E00320054A01462B46DF
:102F80000CF0F0FF03202946224605F053F9B0BDAE
:102F90008B390100F0B585B0054604A80024047003
:102FA000E743002D12D0EA68002A0FD0686A002893
:102FB0000CD0A86A002809D0401EE96A814200D3DB
:102FC0008EE004A928469047002803D03C462046BE
:102FD00005B0F0BD514EE86A411CE962696A049A85
:102FE0000A54E86A696A002202920A54E86A0928C7
:102FF00006D1696A09224848FDF7F1F800283ED059
:103000003078411E022908D800F0D2FEB168401A7B
:103010004349884264D8414E30780A2820D001289C
:1030200023D16E6A3A213046FDF7C8F8002847D010
:10303000019002980390E96A03AB304639A200F090
:1030400051FF02284CD10398002849D00A21334A65
:10305000117001990818696A401AC01C50602FE06D
:103060007068E96A81422BD13AE004A800780A2806
:103070000FD00D2814D101202863E86A1AE001203E
:10308000307000F095FEB0603078411E0229BBD947
:10309000C3E7296B012904D102202863E86A03E011
:1030A000296BE86A022905D1022817D10298E86243
:1030B000286305E0012803D1686A00783E280FD014
:1030C000A86AE96A401E81420AD2EA6804A9284631
:1030D00090470028114E00D17DE777E702982863DA
:1030E000E96A686A00F0E5FE01280FD16B6AE86AB8
:1030F000002806D0C018401E00780A2801D10DA271
:1031000000E010A2032001460CF02CFF03480470DD
:10311000204605B0F0BDC046CE32010054970102F2
:10312000DC0500002B524543454956452C252A2CE9
:1031300025643A005B415420526563765D20257317
:10314000000000005B415420526563765D202573CA
:103150000D0A000010B5064C2078002108F0C6FCCE
:10316000044806F06BFD2078012108F0BFFC10BD7B
:10317000DE96010260E31600B0B50F2001F0E2FB1D
:10318000194D6870287033282AD120243721204611
:1031900001F024FC2120032101F020FC2220402109
:1031A00001F01CFC2320082101F018FC3020AA218A
:1031B00001F014FC0D4802210187322001F00EFCC1
:1031C0003320012101F00AFC5F21204601F006FCBA
:1031D0000F2001F0B7FB28700A2006F02FFDB0BDCC
:1031E00002480021C187B0BDFC95010262A901021D
:1031F000F0B581B0364C21210091617235490988C2
:103200006170354FFB886371BA6ABA61334D2D78AE
:103210002570090AA170190AA171B978304D81424F
:103220000AD10AF087FE6421FCF754FF398148195E
:10323000B96A4018B97800E050192A4A4A438518FB
:10324000FD620AF00DFE40190BF066FA06460D46C7
:103250002548007B0BF0ECF8244909882222A15470
:1032600082B2D20B801802B2D0175210B218684145
:10327000130E009D6355130C202563553B6DA376FB
:103280001D0AE5761D0C25771B0E63772346223336
:10329000090A5970A277BA64F864BA65F865100A29
:1032A000E0770AF047FEF861FB6A282101222046F8
:1032B0000EF0D2F80AF03EFE786109F019F8002805
:1032C000FBD1042008F0D2FB002001B0F0BDC046C5
:1032D00036D40102DC98010260990102B49801021F
:1032E000A0460100C0CC0000B2900102C0980102CB
:1032F00070477047F0B587B051480068FDF716FB7E
:1033000004460D464F48406AFDF7C2FB02460B4695
:1033100020462946FDF70EFA02460B4600244A498C
:103320002046FDF791F9039002910120059040029B
:10333000019046494831464F06E0534A10517F1CE0
:10334000891C241D642C78D0387805284148F4D194
:1033500004970691404801593C4E31613F4803595A
:10336000B3603F480059B0613E4A125932620027AB
:103370005D1A35637369F1689941059B00DB3B4633
:10338000002B01D0019BC918304E7163F369716A3B
:10339000101A9941059A00DB3A46002A01D0019A99
:1033A0008918FDF7E5FA02460B4603980299FDF7E6
:1033B00059F9FDF745FB254A9062D162401BC10FC8
:1033C0004018401010601546FDF7B0FA264A274B0A
:1033D000FDF748F9A863E963254A264BFDF742F952
:1033E0003A46254BFDF73EF93A46244BFDF788F85F
:1033F00005460E4615480564416428463A46204B6A
:10340000FDF756FA00280699049F98D10022284615
:1034100031461C4BFDF762FA069900288FD10888C7
:1034200000B2FDF783FA02460B4628463146FDF707
:1034300067F8FDF7E1FA06997FE707B0F0BDC046EF
:1034400020970102A82001000000F03F1096010221
:1034500030980102FFFF0100C49F010228A0010271
:1034600024E0010288E00102699006699006903F1D
:1034700052257997532ED33F0000594000003E401B
:1034800000408FC0006AF84050D20102B0B582B04F
:10349000194C2068056801A90020087007E09047D2
:1034A0000198401C01A90870C0B2082822D201224C
:1034B00011048140294209D02268516080002018FF
:1034C000826A002AECD001A80121E8E713028340B8
:1034D0002B4201D0022104E082402A42E0D00321A5
:1034E000134622685360800020188268002AD7D0D3
:1034F00001A8D4E702B0B0BDD0920102FEE70000FF
:1035000010B509480168CA6920231343CB610269D9
:10351000032A08D1012293050C689C430C605102D8
:10352000C26E0A43C26610BD4493010281B010B559
:1035300081B00393002807D0C16A002904D003ABEF
:103540000093C46A0021A04701B010BC01BC01B0C7
:103550000047000080B5024608480068002807D0F0
:1035600091B2120C03889A4203D040690028F9D125
:1035700080BD002200F0F4FA80BDC04684C901027B
:10358000F0B581B05C4C2068856BE80707D0E16836
:10359000002904D000208847206801218163A80702
:1035A00007D52169002904D001208847206802211D
:1035B0008163680707D56169002904D00220884724
:1035C000206804218163280707D5A169002904D058
:1035D00003208847206808218163E80607D5E16950
:1035E000002904D004208847206810218163A806A0
:1035F00007D5216A002904D00520884720682021AA
:103600008163680607D5616A002904D006208847CF
:10361000206840218163280607D5A16A002904D0CB
:10362000072088472068802181630126E80507D5A7
:10363000E16A002904D037020820884720688763A0
:10364000A80507D5216B002904D0770209208847F7
:1036500020688763680507D5616B002904D0B7022D
:103660000A20884720688763280507D5A16B0029B1
:1036700004D0F7020B20884720688763E80407D549
:10368000E16B002904D037030C208847206887634A
:10369000A80407D5216C002904D077030D208847A2
:1036A00020688763680407D5616C002904D0B703DC
:1036B0000E20884720688763280407D5A16C00295D
:1036C00004D0F7030F20884720688763E80307D5F5
:1036D000E16C002904D037041020884720688763F4
:1036E000A80307D5216D002904D07504112088474F
:1036F0002068856301B0F0BDD493010202480068E0
:10370000411E88417047C046D0980102F0B58DB087
:10371000002862D00446406800285ED0A068402897
:103720005BD8E56A002D58D0074620464030002679
:10373000039003E0019E4AE0039848E04021012203
:103740000691FCF729FDAE4202963ED2002031469A
:10375000019009900398069B3E46002EEAD0606ACD
:103760000491405C07900998401C059000210427B3
:1037700008916518EA5C012A17D10A966268D31984
:103780001B1F1B68099E9E5D0798864208D1059DF8
:103790005B5D002B0A9E22D00898401C089003E035
:1037A000403500222A70A668069B0837491CB142A2
:1037B000DFD308980028BFD00499491CE06A8142F1
:1037C000059809900398C8D301E003983E46374610
:1037D000E56A029E761CAE42B0D30DB0F0BD616AC0
:1037E0000B91E16A0C91D1590BAA204600F09CF88C
:1037F0000DB0F0BD81B0B0B583B00D46044607935F
:1038000007AB02938069E1690DF0A0FE2062654874
:103810000078002803D1216AA06900F09FF963694C
:10382000A169226A204698470146A06B002905D06D
:1038300069460C600021224B0A460CE000F084FA35
:103840007D2081002846FCF745FC0246A06B6946B6
:103850000C6000211B4B00F0D3FA002003B0B0BC79
:1038600002BC01B00847C04680B5806B00F06CFA1E
:10387000002080BD70B582B00D46044646691146F1
:103880001A46B0470146A06B002907D069460C6074
:1038900000210B4B0A4600F0B3FA0EE000F054FA98
:1038A0007D2081002846FCF715FC0246A06B694686
:1038B0000C600021034B00F0A3FA002002B070BDA1
:1038C000AD390000C339000070B50D4604468021B3
:1038D00000F0C0FA2868E06368686060A868A060CB
:1038E000E868E0602869206168696061A869A06192
:1038F000E86900262662E061286A6062686A2663D9
:10390000E662A062A86A60632046383000F02AFAB6
:10391000002802D0F643304670BD2148016821607E
:103920000460304670BDC04670B514460D4606466C
:10393000881E032802D8B06B00F006FAF06B294607
:10394000224600F00DF970BD16480178012048406C
:103950007047C04670B512480468002C1FD0114E45
:1039600011A5216920468847002815D13078002804
:103970000DD1E16A606A00F09CFA0146606A012993
:1039800003D0E16A00F0E8F8284600F0E3F82046AA
:10399000FFF7BCFE0020E0622468002CE1D170BD7E
:1039A00080C9010278C901020D0A000010B5044661
:1039B000806B00F0C9F9E06B0521002200F0D0F81F
:1039C00010BD10B50446806B00F0BEF9E06B042119
:1039D000002200F0C5F810BDF0B581B00091064698
:1039E000C7680468A01C3946FCF774FB00257068A2
:1039F000814201D1ED430BE0601C3946FCF76AFBC4
:103A0000316032695143B06808180099FCF7B2FB85
:103A1000284601B0F0BDB0B5012400250560446022
:103A200008300EC0B0BD70B50E460446C1680068CF
:103A3000401CFCF74FFB00256068814202D1ED433A
:103A4000284670BD22695043A16841183046FCF7F2
:103A500091FBE1686068401CFCF73CFB6160284614
:103A600070BDB0B5002400280DD00546006888421E
:103A7000FDD3401A286068684018E968FCF72AFB03
:103A800069602046B0BDE4432046B0BDB0B5002417
:103A900000280ED00546006840182860EA68904269
:103AA000FDD8A86840181146FCF714FBA960204611
:103AB000B0BDE4432046B0BDF0B583B01646024623
:103AC0000027F843002E22D01C46002B1FD00D46A5
:103AD000D168136899421AD9CB1AAB4217D39268AE
:103AE000019252198A423A4607D9019A8A1A0292D9
:103AF000029A52199342029A09D30292019810181D
:103B0000FCF7E8FA3160029840192060384603B0AB
:103B1000F0BD406870478068704702460020002A68
:103B200004D0106050609060D1607047C04370470F
:103B3000002803D00168484248417047012070477F
:103B4000002805D00168C068411A484248417047C2
:103B50000120704700207047002070470020704708
:103B6000F0B583B014460D4606464088012818D1AA
:103B7000306900280CD0A900405801782D2910D0B8
:103B8000F368716809686A461160506010A205E028
:103B9000F36870680068694621C115A23046FFF7D6
:103BA000C5FC7768FB6830462946224698470128BD
:103BB00008D00AE0C36830462946224698477F6805
:103BC000012802D178680028F4D103B0F0BDC046C6
:103BD00046534D3A252D38732053544154453A25C8
:103BE0002D323873204556454E543A25730D0A0040
:103BF00046534D3A252D38732053544154453A25A8
:103C00002D323873204556454E543A25750D0A001D
:103C1000F0B581B0002828D01E460C460546079B0B
:103C20000698009000206862A862E862104909883E
:103C30006B8029800F4B1F686C60009BAB602B462C
:103C40000C33C4C3A861E8612862481C0849088095
:103C500008480560002C08D06C60002128460A4600
:103C6000FFF77EFFA468002CF6D101B0F0BDC0467E
:103C700008CD010284C9010202460020002A01D0B9
:103C8000D1627047C043704710B582B004AC24883D
:103C90001B881B041B196C462360024B00F0B0F814
:103CA00002B010BD55350000F0B597B01646029130
:103CB00005464268002A30D001966A60012100243E
:103CC000284616462246FFF74BFF3046029FBE426B
:103CD00032D003A85021FCF766FA32467268002FF2
:103CE0000CD003AF029811C74068083F824209D048
:103CF000394608313C4600280F46F4D1002A019E7F
:103D0000DBD10AE0019E386868600021284632460F
:103D1000FFF726FF7F68002FF5D102988468002CFA
:103D200008D06C60002128463246FFF719FFA468CE
:103D3000002CF6D117B0F0BD00212846019E324676
:103D4000FFF70EFFE9E70000014600201F2901D917
:103D5000C043704718224A43344901238B508918C5
:103D60008860704710B50021CC4300280BD00A4A68
:103D70001368002B09D01832491C2029F8D306D12A
:103D800006A0FFF7E7FE204610BD01231360016087
:103D90000024204610BDC04608CA010274696D6542
:103DA000722049442069732066756C6C0D0A00000E
:103DB000264800687047C04670B520241B4D234E2E
:103DC0002868022817D13068A968EA68401A90422A
:103DD00011D96969002907D02879002807D0022065
:103DE00028603068A86004E00120286003E001201A
:103DF0002860286988471835641EE1D170BDC04627
:103E0000F0B5044600201F2C01D9C043F0BD059D2C
:103E100018266643054C0227A751A41921710B49A6
:103E200009682646083626C66361F0BD08CA010245
:103E300006480168491C0160054841680268002382
:103E4000521C02604B4143607047C046BCAD01024A
:103E5000C0AD010280B5FCF7A6F980BDB0B502780F
:103E6000002A24D0441C0021084601E0573A08E00B
:103E700023460001D5B2302D0C4611D3392D02D87E
:103E8000303A14460CE0412D0C4609D3462D01D89A
:103E9000373AF6E71446613CE4B2062CE6D3002438
:103EA000E2B280185C1C1A78002AE1D1B0BD002073
:103EB000B0BD10B50246012000290DD00023D45C0E
:103EC000202C02D37F2C04D307E00D2C01D00A2C28
:103ED00005D15B1C8B42F2D310BD002010BD002029
:103EE00010BD000081B0F0B584B0099300230393A6
:103EF000002800D1C2E0002A00D1BFE009AB039343
:103F00001678002E00D1A8E05623DB43009300234F
:103F10001D46002900D1A2E0252E3FD1971C5278E2
:103F20001446643C0023142C43D8C0467C442479B6
:103F30006400A7440A99A3A3A3A3A3A3A3A3A3A331
:103F40004CA3A3A3A3A3A3A35F000297039A131DEB
:103F50000393126801920122002317461E4604783B
:103F6000FF0703D02D2C01D1164607E02746303F2E
:103F7000092F09D80A275F433B19303B491E401CD3
:103F800000270029EBD13946029A019C002C03D06E
:103F9000012E00D15B4223606B1C06E00378B34224
:103FA0005BD1491E521C401C2B461678002EAFD107
:103FB00064E02A2A62D13A780378934204D0491EF9
:103FC000401C0029F8D100216B1C3A46EDE7039A0A
:103FD000131D03933E7812680023C45CB44233D0AF
:103FE000491E5B1C0029F8D13C46C7180021002A55
:103FF0002ED12EE00297039A131D0393126800231B
:10400000009E0778302F18D33A2F02D23446273437
:104010000BE0612F03D3672F344606D30DE03C46F7
:10402000413C052C09D8344620341B011B19DB19EF
:10403000491E401C0029E4D10021029C002A00D026
:1040400013606B1C2246B0E73C46C718002A00D01C
:1040500009C26B1C22463846A7E700230EE0252E36
:104060000BD15178652908D103990A1D039209687B
:10407000002900D008606B1C00E02B46184604B0F5
:10408000F0BC02BC01B0084781B010B581B00C464D
:10409000039303AB00930DF059FAA04200D3601EC6
:1040A00001B010BC02BC01B0084770B50446002046
:1040B000002A1BD0002C19D0002B17D0146001202F
:1040C000022B13D32578002D10D0641C01208D42C3
:1040D00005D1651E00262E7085005451401C984263
:1040E00004D2661C2578002D3446F0D170BDB0B5E1
:1040F00004467821FCF762F8002805D158212046B3
:10410000FCF75CF8002828D04278002A23D0841CD1
:104110000021084623460001D5B2302D0C4613D3AA
:10412000392D01D8303A0EE0412D0C460CD3462DE6
:1041300001D8373A07E01446613CE4B2062C01D3BB
:10414000002401E0573A1446E2B280185C1C1A7849
:10415000002ADFD1B0BD0020B0BD2046FCF7EEF84C
:10416000B0BD70B504460026F043002C0DD00D46BE
:1041700000290AD0204610300121FFF772FCA968FF
:1041800020342046FFF76DFC304670BD70B5044604
:104190000026F043002C0DD00D4600290AD0204601
:1041A00010300121FFF772FCA96820342046FFF788
:1041B0006DFC304670BD70B50024002814D0054653
:1041C000064610363046FFF7B3FC01280CD02846CF
:1041D0002030FFF7ADFC012806D02C683046FFF7F1
:1041E00098FC0C2141436418204670BDF0B583B0A3
:1041F00000250295019500281FD00C46064607466B
:1042000010373846FFF79CFC002816D13046203086
:1042100002AA01AB2146FFF74FFC00280DD13568FB
:104220003846FFF778FC0C214143B068029A101819
:1042300068506D186C600198A860284603B0F0BD06
:1042400070B505460C2058430024904211D2121A32
:10425000461829606860AE60EA602846103019464A
:10426000FFF75BFCE96820352846FFF756FC20463F
:1042700070BDE443204670BD04217046084204D05E
:10428000EFF30983EFF3088203E0EFF30883EFF322
:1042900009829BB004A8F0C044464D4656465F468E
:1042A00008A8F0C01846F0C86846F0C018690C901D
:1042B000202018440D9058690E9098690F90D86985
:1042C0001090EFF310801190EFF3148012900949D1
:1042D0000868139008490868149008490868159000
:1042E0000749086816901793189270461990684607
:1042F0000AF0F6FF04ED00E00CED00E010ED00E048
:1043000014ED00E0F0B581B00326002430462146CC
:1043100007F030FC04252846214607F02BFC012736
:10432000304639463A4607F0B9FB30462146324618
:1043300007F048FC284639463A4607F0AFFB022111
:104340002846224607F03EFC01B0F0BDF0B589B02A
:1043500008900425284607F089FB0A27384605F00F
:104360006DFC284607F092FB0324204607F086FBED
:1043700007900526304605F061FC284607F076FBDD
:10438000384605F05BFC284607F080FB204607F026
:1043900075FB0690304605F051FC284607F066FB99
:1043A000384605F04BFC284607F070FB204607F026
:1043B00065FB0590304605F041FC284607F056FBAA
:1043C000384605F03BFC284607F060FB204607F026
:1043D00055FB0490304605F031FC284607F046FBBB
:1043E000384605F02BFC284607F050FB204607F026
:1043F00045FB0390304605F021FC284607F036FBCC
:104400003846019705F01AFC284607F03FFB204686
:1044100007F034FB0290304605F010FC284607F008
:1044200025FB384605F00AFC284607F02FFB2046FE
:1044300007F024FB0746304605F000FC284607F04D
:1044400015FB019805F0FAFB284607F01FFB2046F4
:1044500007F014FB0446304605F0F0FB284607F051
:1044600005FB0699481E81410A460799481E81416D
:10447000480080188000059A511E8A41510040185A
:10448000049A511E8A4180188000039A511E8A4165
:1044900051004018029A511E8A4180188000791EEE
:1044A0008F4179004018611E8C4106190898002838
:1044B00003D0032007F0DAFA02E0032007F0E6FA5F
:1044C0000A24204605F0BAFB0425284607F0DEFA48
:1044D000204605F0B3FB284607F0C8FAF0B209B051
:1044E000F0BD70B50446042007F0C0FA60B20028A1
:1044F00003D4032007F0BAFA02E0032007F0C6FA5B
:104500000A25284605F09AFB0426304607F0BEFA35
:10451000284605F093FB304607F0A8FA284605F038
:104520008DFB600603D4032007F0A0FA02E003200D
:1045300007F0ACFA0A25284605F080FB0426304631
:1045400007F0A4FA284605F079FB304607F08EFA0A
:10455000284605F073FBA00603D4032007F086FA73
:1045600002E0032007F092FA0A25284605F066FBD0
:104570000426304607F08AFA284605F05FFB3046ED
:1045800007F074FA284605F059FBE00603D403202F
:1045900007F06CFA02E0032007F078FA0A252846B3
:1045A00005F04CFB0426304607F070FA284605F06B
:1045B00045FB304607F05AFA284605F03FFB200736
:1045C00003D4032007F052FA02E0032007F05EFA5A
:1045D0000A25284605F032FB0426304607F056FA35
:1045E000284605F02BFB304607F040FA284605F038
:1045F00025FB600703D4032007F038FA02E003200C
:1046000007F044FA0A25284605F018FB0426304630
:1046100007F03CFA284605F011FB304607F026FA71
:10462000284605F00BFBA00703D4032007F01EFA71
:1046300002E0032007F02AFA0A25284605F0FEFAD0
:104640000426304607F022FA284605F0F7FA3046ED
:1046500007F00CFA284605F0F1FAE00703D1032031
:1046600007F004FA02E0032007F010FA0A242046BB
:1046700005F0E4FA0425284607F008FA204605F07C
:10468000DDFA284607F0F2F9204605F0D7FA70BDAA
:10469000F0B581B003260025012430462946224684
:1046A00007F0FCF9304607F0F1F90626304605F030
:1046B000C5FA042007F0EAF9304605F0BFFA0320F6
:1046C00007F0DCF900281BD0681CFA2D0546F6D34C
:1046D0000425284607F0CAF90326304607F0C6F934
:1046E0000A27384605F0AAFA284607F0CFF93046DF
:1046F00007F0CCF9384605F0A1FA204601B0F0BD2C
:10470000032001210A4607F0C9F9042007F0AEF999
:104710000024204601B0F0BDB0B50446C00703D167
:10472000032007F0A3F902E0032007F0AFF9082502
:10473000284607F0ABF9284607F098F9A00703D4FC
:10474000032007F093F902E0032007F09FF9082502
:10475000284607F09BF9284607F088F9600703D43C
:10476000032007F083F902E0032007F08FF9082502
:10477000284607F08BF9284607F078F9200703D47C
:10478000032007F073F902E0032007F07FF9082502
:10479000284607F07BF9284607F068F9E00603D4BD
:1047A000032007F063F902E0032007F06FF9082502
:1047B000284607F06BF9284607F058F9A00603D4FD
:1047C000032007F053F902E0032007F05FF9082502
:1047D000284607F05BF9284607F048F9600603D43D
:1047E000032007F043F902E0032007F04FF9082502
:1047F000284607F04BF9284607F038F960B2002840
:1048000003D4032007F032F902E0032007F03EF959
:104810000824204607F03AF9204607F027F9072434
:10482000204607F033F9204607F020F9B0BDF0B577
:1048300081B0032700243846214607F08BF938461B
:10484000214607F097F9012538462946224607F008
:1048500025F9052638462946324607F0B3F90827D8
:104860003846214607F086F938462946224607F0A1
:1048700015F938462946324607F0A4F90727384685
:10488000214607F077F938462946224607F006F90F
:1048900038462946324607F095F901B0F0BD0000D0
:1048A00080B50B2007F0EAF812490A78002804D0F6
:1048B000002A12D003F0F2FA80BD012AFAD10020BA
:1048C00008700F49C8830C4908700C480121017019
:1048D0000BF084FC03F0E2FA80BD0748012202706D
:1048E0000A700648002101700BF09CFC03F0D6FA18
:1048F00080BDC0461C90010218900102199001026F
:1049000062A9010202484069811E4842484170473D
:104910009896010280B5FDF74DFA002801D00020DD
:10492000C04380BD80B5FEF7FBFA80BD10B50448DA
:104930000F2100242246FFF713F9204610BDC04680
:104940000C9A0102F0B581B007460324204607F017
:104950009DF80425284607F099F8204607F086F8C8
:104960000A26304605F06AF9284607F07FF832201B
:10497000FFF7B7FDFFF78CFEF8B2FFF7B2FDFFF7C8
:1049800087FE204607F082F8284607F07FF8204689
:1049900007F06CF8304605F051F9284607F066F844
:1049A0003320FFF79EFDFFF773FE0020FFF7CEFCDC
:1049B0000746284607F05AF8204607F057F83046D1
:1049C00005F03CF9284607F061F8204607F05EF84C
:1049D000304605F033F9384601B0F0BDF0B581B08E
:1049E000009107460324204607F050F8042630467D
:1049F00007F04CF8204607F039F80A25284605F05C
:104A00001DF9304607F032F83220FFF76AFDFFF754
:104A10003FFEF8B2FFF765FDFFF73AFE0098FFF79B
:104A200060FDFFF735FE304607F020F8204607F01E
:104A30001DF8284605F002F9304607F027F8204611
:104A400007F024F8284605F0F9F8284605F0F6F8AE
:104A500001B0F0BD80B50748012101700648026829
:104A60000A43026005480268002A02D0002001467D
:104A7000904780BD0ECD01021C10005010CD0102E8
:104A8000F0B599B0F548017BC67A427B0E92F44CA2
:104A9000221F1368F34A1268069242780C92027938
:104AA0000592C76A04931F4001200F907A0200D537
:104AB000BCE03A0200D5BFE0FA0102D50F98020629
:104AC0002260502508968A191826BB0102D50F9836
:104AD000430623604123079569430A9635465543AB
:104AE0001426FC0210D50F98040538463746DC4ED4
:104AF0003460DA4CA469B464D84CE4697464DA4C68
:104B0000241D34603E46074690000B90D8040D905B
:104B1000681809900E9B73430F988203B902D04D19
:104B200022D50F9841052960CC480E9616460246BC
:104B300081692965C169696509990D9801430898DA
:104B4000000108180B994018C018C84909889279C3
:104B50004A4380180A301C4605F050FB2346324673
:104B60000E9EC04988672A600F98C404380300D598
:104B70002C60F80302D50F98000428600F984104B8
:104B8000B80300D52960380400D4E4E1039402910D
:104B90000E9308920D980B990C180A980C994143A2
:104BA0000C910F98C0030B90286008F055F900286D
:104BB00001D005F005FB0C98005B410B43D109982F
:104BC00000190E9940180599090140180E90E74DFB
:104BD000287B079B4343E97A0A010D9C2243D218A4
:104BE00041188B00D2180A9B4B43D1186A7B56435D
:104BF00089190E9E2A791018DF4A128842438818B4
:104C000016903068C000800D10A9C882002511954B
:104C10007079C0077ED110A80F998182069C0094FC
:104C20000020E8A2049B0BF09DF978E00F98820524
:104C300022603A0200D43FE70F98C2052260FA01D1
:104C400000D53BE73DE7072149030840032149031D
:104C50008842089A00D07EE1069707F071FD002097
:104C6000169009901590C14CE07A217B08180A999A
:104C7000414380000D9A10434118627B0E967243A7
:104C80008A186178A379079E7343D718FA683F267C
:104C9000324063789A420C976ED105960A9A4A433D
:104CA00080580F210A0702400398401EC04B1B6822
:104CB000DB090340981810900F98C0020B90B86859
:104CC000800767D42C46283C0AF0C2F805462068C5
:104CD000000609D5C3208401786A400704D40AF08D
:104CE000B7F8401BA042F7D905980002B9684908F7
:104CF0000140B34803688268B868C40C2020204093
:104D0000DB0700D095E0002310221D461C460E9EB6
:104D10000B9FB1E010A88582B0681190069C701DB1
:104D2000924B1979E20707D1491C1971D97A1A797E
:104D30008A4202D31D7100E0D970017842781202D4
:104D40005118827812048918032291430170357139
:104D50005878401C5870D87A197B081859788842BE
:104D600000D85D70D879401ED871596B002901D0E8
:104D700010A888477E4DEDE010A80B998182F86855
:104D800030406378009000207CA20F990BF0EAF885
:104D90000E9E94E0388A874A024010A8C2822022E0
:104DA000BA5C9307DB0F3C68C3720F9B1A40827298
:104DB0006205D20C0D9B1A431692FA68130E037209
:104DC000BB69FC697C4D2D682D0C05745204920F53
:104DD000427211931394654CA07B002809980E9E93
:104DE0000B9F5FD075480068007A0328099859D056
:104DF0000C98007D08400928099853D1C3208401EC
:104E00000AF026F805460C98406A41070BD4594928
:104E100009680906890F06D10AF01AF8401BA0425A
:104E2000F1D90C98406A41030898884310A98882F8
:104E300037E0D2070E9E0B9F03D1082300221546B0
:104E400019E00C9B9A68029C224211D19A68520C7C
:104E5000022494430022134615460DE014D20102A9
:104E600028A000503CA10050FC1F000010D20102FD
:104E700004250022134614460843104318432843D0
:104E8000204310A9888238420BD10C9B198A494AC9
:104E90000A4010A9CA8219684905C90C0D9A114324
:104EA0001691324C2921615C002908D03037B84274
:104EB00005D010A908461130123109F0CFFAE77A6F
:104EC0002A48047BE519294800790E902748407844
:104ED000401C2946FBF7FEF888000D9A10431890F5
:104EE000079961433801104340182049497B4E43DC
:104EF00080191C21694340180E9909191B4B1E4A41
:104F000012884A4380181790099A0C998A60987BF6
:104F1000002800D04A629879401C9871187B9979D2
:104F20008142069F00D39A715978491C5970D97AE9
:104F30000818597888420E4D00D85A70187A401EC9
:104F400018722820185C002804D0996B002901D021
:104F500010A88847089A174202D00F9800032860CB
:104F60001C480449486019B0F0BDC04614D2010283
:104F700028A000503CA1005010D201024857204503
:104F8000542069647820256420616E642045542093
:104F900069647820256420696E2052582064657306
:104FA00063206D69736D617463680D0A0000000011
:104FB00038200040FF03000094300040409401027C
:104FC000604000404D41432045565420257820251F
:104FD000780D0A00FFFFFF03F0B5A5B01E460C9246
:104FE00008910024239422A90C8016A90C8024A9DE
:104FF00009250D80598C0D91FBF76CF82A99012930
:1050000000D0DFE03189012900D0DBE0318C0129BB
:1050100000D0D7E00D99002900D1D3E022460796B1
:105020002C990B912B99069180B205900F9415A89D
:10503000058090000E900C990C582E4600252046B5
:1050400029461746FBF7EEFB0028119636D12C2097
:105050000A9778430899081817A90A4668C868C2C9
:10506000E8C8E8C2E8C8E8C2079F119880B280008B
:105070000E5822AD019523A8009020463946059A86
:10508000069B04F0E9FD0F98401C0F90288800282B
:105090002DD03B8A239913AC039416A8029014A830
:1050A000019015AE009617A824AA04F0AFFF25883A
:1050B000308811900120149E0A9A05E013A80580FB
:1050C00014952E4628463A460E9F51000B9B119C84
:1050D0005C52591808830D84D81986600F9818857A
:1050E000521C0D9882426DD024A805889FE709962E
:1050F00016A800250580149524A8068823981290E8
:105100002F46109503E06D1CA8B2B04213D8A8B288
:10511000800017A90C5820461299FBF791FB002834
:10512000F1D1002FEFD115A8058016A8012707801F
:1051300014941094E7E715A80288B01A012805D145
:1051400015A80680099F1497119628E0102007994A
:10515000095E0129119221DB551CA8B20C18109F81
:105160000E9B099403E06D1CA8B2844218DDAAB21C
:10517000B242F8D8800017AA105810903946344629
:105180001E46FBF74FFB33462646099C0028EAD112
:1051900015A80580109F14971195E4E7109F0E9BAA
:1051A0001C463E4638461299FBF76BF9FBF7F6FBB7
:1051B0000546052800D3052513A8058001200A9A75
:1051C000274682E725B0F0BDF0B58BB00243159AB3
:1051D000149C139E2BD0054601A856C0129CD8697A
:1051E000196A09900A911E469F6B0123009309A832
:1051F00007AA0146059306F00BFD716C3846FBF7D4
:1052000040F90746E06A616BFBF73BF9002D069613
:1052100013D0044611980199012924D10921081AB3
:105220000421069A515E884229D16425B1E000200C
:105230003080207010700BB0F0BDB0880022642563
:10524000002829D0059269493846FBF715FB00284C
:10525000049C039E6FD166493846FBF70DFB00287E
:105260001DD05A2567E03C25082800D191E05F4910
:105270002046FBF701FB002819D0502589E00A29B8
:105280001DDB1D293BDC59493846FBF7F5FA0022A6
:10529000002854D05A253AE03346049C39E0554959
:1052A0003846FBF7E9FA002821D0502543E0504961
:1052B0002046FBF7E1FA00282ED0462569E03C2580
:1052C000012866D049492046FBF7D6FA0028D4D1F8
:1052D00047492046FBF7D0FA0028EED14549204641
:1052E000FBF7CAFA002854D1434920466EE04249F0
:1052F0003846FBF7C1FA00281CD128251BE03B49A2
:105300003846FBF7B9FA0022002832D05025049C19
:10531000069B0299039E41E036492046FBF7ACFA12
:10532000002836D134492046FBF7A6FA00282FD1B1
:1053300014252EE037250299059A069B2EE005924A
:105340002B493846FBF798FA002896D12949384668
:10535000FBF792FA0028B0D127493846FBF78CFAC0
:105360000028049C069B0299039E059A3BD11E25AA
:1053700014E005921E493846FBF77EFA00289CD1BE
:105380001C493846FBF778FA00281DD03C2500E080
:105390002325049C069B0299039E059A2580327062
:1053A00000200870307800280CD118681349FBF7EA
:1053B00055FA002806D12088102803D30F38208002
:1053C0000BB0F0BD0BB0F0BD0B493846FBF754FAFB
:1053D0000028049C069B0299039E059A01D114257E
:1053E000DCE72325DAE72D25D8E7C046CDCCCC3D38
:1053F000CDCC4C3DCDCCCC3C0AD7233C000020404A
:1054000070B588B00C4606464088002820D0FBF7CF
:1054100086FA059005A804A901252A4606F062FE31
:105420003088B188081AFBF76FFA0390049903A833
:1054300007AA2B4606F016FE5249079D2846FBF7A1
:105440001BFA002808D0BF200006206008B070BDFD
:105450000020206008B070BD4B492846FBF7F0F9EA
:10546000002804D03F200006206008B070BD4749E6
:105470002846FBF701FA002801D0002010E00021A7
:105480002846FBF7F9F9002801D0022008E040493E
:105490002846FBF7F1F9002801D0042000E006209F
:1054A00001957F21C905029180003A49091801A898
:1054B00006AA022306F08AFD0698206008B070BD97
:1054C000F0B587B00C460546476800263846314699
:1054D000FBF7E0F9002802D0266007B0F0BD049782
:1054E00004A803A90126324606F0FCFDA868296835
:1054F000FAF782FF0290039902A806AA334606F043
:10550000B1FD2049069D2846FBF7B6F9002804D0D6
:10551000BF200606266007B0F0BD1B492846FBF7F2
:105520008FF9002804D03F200606266007B0F0BDA2
:1055300016492846FBF7A0F9002801D0002010E00A
:1055400000212846FBF798F9002801D0022008E046
:105550000F492846FBF790F9002801D0042000E00D
:10556000062000957F21C90501918000094909188D
:10557000684605AA022306F029FD059E266007B0AD
:10558000F0BDC046CDCC0C3F295C0FBFCDCC4C3E0E
:10559000CDCC4CBE48940102F0B587B00C4606460F
:1055A0007F270088002801D0FD0503E0B08800288F
:1055B0002ED0334DFBF7B3F903907088FBF7AFF9AA
:1055C000049003A802A90126324606F08BFD029939
:1055D00004A806AA334606F045FD2A49069E304631
:1055E000FBF74AF9002802D03F20010641E0264996
:1055F0003046FBF725F9002802D0BF20010638E02D
:1056000022493046FBF738F9002805D0002024E075
:105610000020206007B0F0BD1D493046FBF72CF993
:10562000002801D0022018E01A493046FBF724F97F
:10563000002801D0042010E017493046FBF71CF980
:10564000002801D0062008E014493046FBF714F981
:10565000002801D0082000E00A200096F9050191F9
:1056600080000F490918684605AA022306F0AEFC1F
:1056700005992846FAF7C8FE206007B0F0BDC0467D
:10568000000080BF000038433333733F0000C8423E
:1056900000007042000020420000A0410000C04015
:1056A00068940102F0B59DB015460B917F210391DE
:1056B000C9051C9102911B9119A900248C80199491
:1056C00018941794598C0691198C0F91DE8B998B35
:1056D0000791997805911F882B21CA4327999142F8
:1056E00001DB7F0015E04022D243914211DC4922C8
:1056F000D243914202DB7908CF190AE05322D24308
:105700009142EEDA5D22D243914201DBBF0000E01C
:10571000FF000A971396269E597E00290BD0002180
:1057200032460F46D170917051701170121D7F1C5E
:105730005C7EA742F6D30C9311952599149122997A
:105740000D91159041088C4211D2FD4A2346A000CC
:1057500084583454270A451C7755250C871CF55569
:10576000240EC01C34545B1C9CB2A142EFD8239879
:10577000109001200990009030463146149A159FF0
:105780003B4606F053FA0D9800060890400E139D14
:1057900000D186E068000490002F3FD00022104620
:1057A0001146144606E01C461146159F401C82B265
:1057B000BA420ED283B2AB42F8D09200149B9A5EEA
:1057C0000FB2BA42034600DC2346BA42EBDC0A467B
:1057D000E9E7002F25D0002210461146129206E07C
:1057E00012931146159F401C82B2BA4214D283B262
:1057F000AB42F8D0A5B2AB420CD09200149B9A5E9B
:105800000FB2BA42034600DC129BBA42139DE7DC9A
:105810000A46E5E7139DE6E7129903E000242146D6
:1058200000E00021129110980183C4828582049FB8
:10583000F057FBF769F87921C9050E91FAF7E4FDF5
:105840001099C86109980743F057FBF75DF80E9966
:10585000FAF7DAFD109F38622004C40B3057FBF7CB
:1058600053F80E99FAF7D0FD7862601C3056FBF7BA
:105870004BF80E9C2146FAF7C7FDB8621298000457
:10588000C70BF057FBF740F82146FAF7BDFD109C17
:10589000E062781C3056FBF737F80E99FAF7B4FD42
:1058A0002063119805800C98407E410000278D42AE
:1058B00028463A46149E1ED30A9880B28AB29300B4
:1058C000F45E84420BDA491C8AB2AA42F6D9002758
:1058D00028463A4681B2691A012910D01BE0F01817
:1058E000119B1980078808040FD0500040008019D0
:1058F000001F0288084681B2691A01290BD1A8004D
:10590000301811990D80078826E00020024681B2E8
:10591000691A0129F3D00A9989B2079B4B43BB420C
:105920001AD306998A4217D80599002914D0401C29
:1059300082B2891803E0401C82B291420CD983B232
:10594000AB42F8D89200B35EBCB2A342F3DDB2180A
:10595000119B18801788EEE712970B980580119815
:1059600000882B1A002B16DD02210F9A1143032900
:1059700042D10E93411C421E10B281420EDA0E98A3
:10598000032824DB0C98808C012820D019A818A9A2
:10599000FFF736FD1FE0002018902BE00026F443AF
:1059A000374608E0B8B2400019AD2B527F1C521C9C
:1059B00010B28142E3DB13B2A3423346F2DD159B02
:1059C00098423346EEDA8000149B1B5AEAE719A886
:1059D00018A9FFF7E1FD149E139D0F9A012A13D019
:1059E000032A11D0022A04D111980088281A02280B
:1059F0000ADA0020179034E0022A01D1022BB8DA2B
:105A000000201890012AEBD1681C691E0FB2B84221
:105A100008DA0C98808C01281DD119A817A9FFF766
:105A2000BBFD1CE00022D343144608E0A5B26D0084
:105A300019AF7E53641C491C0FB2B842E9DB0DB2AA
:105A40009D421646F2DD159DAF421646EEDABD00C8
:105A5000149E765BEAE719A817A9FFF7D1FC149EFC
:105A6000139D249F189C17992046FAF7C5FC0F999F
:105A7000012900D8204638600D98002800D1CBE0DD
:105A800011990888109FB8860888281AB88012983B
:105A900080B2FAF744FF7921CC052146FAF7B4FC2D
:105AA0002146FAF7B1FCB863119F3888002849D025
:105AB00081008919091F0988129C0C1915998842BF
:105AC00003D2800080198088041915984300534937
:105AD00016AA304606F088FA169810994864FAF724
:105AE00076FFA4B2A04201D14D480FE0001BFAF7A7
:105AF00016FF1C901CA81BA9012206F0F3FA2046F1
:105B0000FAF70DFF01461B98FAF77EFC1099086022
:105B10003988491B4A1C92B2032A02D20021159FE0
:105B200017E009B20229159F12DB3F210906FAF797
:105B3000A3FE002802990CD10998810709E0C0460C
:105B4000402100400020129C15998842B9D3BCE73F
:105B50003449109801610898800E5DD0002F1CD048
:105B600000221146144610464B1B1DB2ED135B1963
:105B70006B40139D1BB29200B25E53431818A418D9
:105B8000491C8AB2BA42EFD3FAF7C9FE064620464C
:105B9000FAF7C5FE002C03D100E000260398C005EB
:105BA0001C901CA81BA901252A4606F09BFA1B9CE9
:105BB00020463146FAF728FC014610988160002FF4
:105BC000119422D000242746264613951291B8B28C
:105BD000FAF7A5FE1299FAF70FFC0546A0001499F2
:105BE000085EFAF791FE01461398C00785432846E0
:105BF000FAF70AFC01463046FAF7ADFB06467F1C71
:105C0000BCB215988442E2D300E0002611983146D8
:105C1000FAF7FAFB1099C8601DB0F0BD60A7010249
:105C20000000204100004040F0B58FB00692F74AD6
:105C300009AF70CA70C770CA70C70328079320D80D
:105C40008800F3A10858F649FAF785FB0446F549A0
:105C5000FAF781FB0D90F4492046FAF77CFB0C9093
:105C6000F2492046FAF777FB0B90F1492046FAF704
:105C700072FB0A90EF492046FAF76DFB0990EE4956
:105C800069E0042822D0062820D88800EBA1085813
:105C9000EE49FAF760FB0446ED49FAF75CFB0D901C
:105CA000EC492046FAF757FB0C90EB492046FAF7EF
:105CB00052FB0B90E9492046FAF74DFB0A90E84960
:105CC0002046FAF748FB0990FD4944E008380228CD
:105CD00021D88800FBA10858D149FAF73CFB0446BB
:105CE000FC49FAF738FB0D90FB492046FAF733FBE5
:105CF0000C90FF2081052046FAF72DFB0B90F74909
:105D00002046FAF728FB0A90CA492046FAF723FBF7
:105D10000990FE491FE08800F1A10858F449FAF7FC
:105D20001AFB0446F349FAF716FB0D90F249204698
:105D3000FAF711FB0C90F1492046FAF70CFB0B9097
:105D4000EF492046FAF707FB0A90EE492046FAF79A
:105D500002FB0990EC4900942046FAF7FCFAEC4962
:105D600009680E90EB480468EB4801684808EB4F5F
:105D700005463D400022002D08922DD0CA01120E8A
:105D800007D0280CE90D12D14000E649085AE6492F
:105D90000AE0C903090E0CD0280AE90B10D1400013
:105DA000E049085A8F2189004018E4300DE0DC49B1
:105DB0000AE081B27F2905D84800DA49085A04E090
:105DC000D94901E08F218900401800B2FAF79CFD03
:105DD000D649FAF719FB02460292039507252606D3
:105DE000D34B1A68002A089840D0791C8A420BD2FB
:105DF0001102090E13D0110C1F46D00D1FD14800FF
:105E0000C849085AC84907E01F46110E002A13D492
:105E10004800C449085AC2494018E4301FE0110440
:105E20001F46090E0ED0110AD00B12D14800BD49F1
:105E3000085A8F218900EFE7BE4808180FE0B848DC
:105E400008180CE091B27F2906D84800B549085AD5
:105E500005E0B548081802E08F218900501800B20B
:105E6000FAF752FDB149FAF7CFFA3B460590159F74
:105E70002C40F50E5B69B0491940089810D0DA0241
:105E8000D20E34D0C80B3E210140A648405AA64944
:105E90004018E43000B2FAF737FDA449FAF7B4FA33
:105EA0000490149E6800A5A1085EFAF72DFD014636
:105EB000A00009AA1058FAF74EFA0146B8B2012814
:105EC000089F019102D1022C0AD9A74F052C24D199
:105ED000189808900C2D20D80B2D16D3A44918E043
:105EE0000027022C089718D08120C70515E01A0456
:105EF000120E00D1CAE0080AC90B00D0CDE0400064
:105F00008849085A8F218900C2E7092D00D2C7E0CD
:105F100096490898FAF71FFA089001200021B54227
:105F2000034600D30B46052C00D308461799169A52
:105F30001A9C199D1843069B012B12D1079B402BDD
:105F400022D1002840D03846FAF705FA01460198D8
:105F5000FAF701FA01460098FAF74EFA059A049901
:105F60008AE0079B402B1FD1002838D03846FAF72B
:105F7000F2F901460198FAF7EEF901460098FAF7AE
:105F80003BFA059A049977E0002833D03846FAF7AF
:105F9000E2F901460198FAF7DEF901460098FAF7AE
:105FA0002BFA059A049967E000285BD03846FAF787
:105FB000D2F901460198FAF7CEF901460098FAF7AE
:105FC0001BFA059A049957E002981146FAF714FA59
:105FD0000399002900D16748059A04994CE002987A
:105FE0001146FAF709FA0399002900D16148059A88
:105FF000049941E002981146FAF7FEF90399002945
:1060000000D15C48059A049936E0C046C41F0100DF
:10601000000068C1000088C166665EC1000084C1DE
:10602000000084410000B4410000484100002040CD
:106030000000F0C0000084C10000F841333323C1E8
:10604000000050C19A9929C19A9949C19A99494128
:106050003333CB4166667641CDCCAC40333393C00D
:106060009A9949C102981146FAF7C6F9039900298D
:1060700000D14048059A049928601046FAF7BCF907
:106080000899FAF7B9F920600FB0F0BD99B27F29ED
:1060900011D848002349085AFCE623494018F9E67C
:1060A000C12001060898FAF756F90890062D00D984
:1060B00033E7002030E78F2189005818EAE6C04610
:1060C0003333F341000058C19A9961C19A9969C16B
:1060D000000084C10000AC4100003841000008C14C
:1060E000CDCC80C1CDCC88C133338FC1333397C180
:1060F00033339741CDCC8C413333F3409A9919C057
:10610000666646C1333397C1CDCCB4410000D4415B
:106110000C0000405030004068400040FFFFFF008E
:106120007C080000D02301005C050000919AF63C39
:10613000642000409C0B0000FFFF1F00FAFFFCFFE3
:10614000FEFF000002000400060008000A000C0028
:106150000E00100012001400160018001A001C0097
:106160001E00200022002400000080BF0000A0C00C
:10617000000040C00000DCC2F0B5FFB0ECB0174634
:106180000E460D900021E991E891DC91999198914A
:10619000979196911491139112919AA8F49DF39C62
:1061A000F29A002E00D1E6E10B938030F09B118033
:1061B000099529602546DBAC218095AC21800C95A2
:1061C0002980DA917F24E405B994B894B794B69401
:1061D000B594B494B394B294B194B094AF94AE9493
:1061E000AD94AC94AB94AA94A994A894A794A694C3
:1061F000A594A494A394A294A194A0949F949E94F3
:106200009D949C949B949A94046644668466C466A8
:10621000046744678467C467046444648464C46432
:10622000046544658465C465046244628462C46232
:10623000046344638463C463046044608460C46032
:10624000046144618461C461B0090B250B2800D34B
:10625000AE011095012B0B9D00D070E12B89012B15
:1062600000D06CE1298C00290E9200D18BE16B8C5F
:10627000002B00D1FAE1AA8C3021695C002900D101
:1062800088E10892109F5F431196304639460F937C
:10629000F9F720FF0590FAF737FB01462046FAF799
:1062A000F0F88321C905FAF7AFF8064696A8021D53
:1062B000119887420A9200D879E155A811909AA9BD
:1062C000069196AF15463A46059C234605F07EFE9C
:1062D00015A80F9006992A46234605F077FE02235B
:1062E0000D93384631463A4605F0BCFE012308932B
:1062F0000093E8AA10923846394605F089FCE898E0
:10630000DD901198069D29463A46234605F05EFE2B
:106310000F9829460A9A234605F058FE384631461A
:106320003A460D9B05F09EFE089B00933846394681
:10633000109A05F06DFCE898DE9011982C462946DD
:106340003A46059D2B4605F041FE0F9821460A9AD4
:106350002C462B4605F03AFE384631463A460D9B10
:1063600005F080FE089B009338463946109A05F0E8
:106370004FFCE898DF901198069D29463A4623463F
:1063800005F024FE0F9829460A9A2346254605F073
:106390001DFE384631463A460D9B05F063FE089BCC
:1063A000009338463946109A05F032FCE898E090A0
:1063B0001198069C21463A462B4605F007FE0F9899
:1063C00021460A9A2C462B4605F000FE38463146F7
:1063D0003A460D9B05F046FE089B00933846394629
:1063E000109A05F015FCE898E1901198069D294651
:1063F0003A46234605F0EAFD0F9829460A9A2346B5
:10640000254605F0E3FD384631463A460D9B05F03A
:1064100029FE089B009338463946109A05F0F8FB90
:10642000E898E2901198069C21463A462B4605F0E2
:10643000CDFD0F9821460A9A2B4605F0C7FD384638
:1064400031463A460D9B05F00DFE089B00933846F9
:106450003946109A05F0DCFBE898E3901198214644
:106460003A462B4605F0B2FD0F9821460A9A2B4674
:106470002C4605F0ABFD384631463A460D9B05F0FB
:10648000F1FD089B009338463946109A05F0C0FB91
:10649000E898E4901198069D29463A46234605F06F
:1064A00095FD0F9829460A9A2546234605F08EFD4C
:1064B000384631463A460D9B05F0D4FD089B0093C3
:1064C00038463946109A05F0A3FBE898E5901198F4
:1064D000069C21463A462B4605F078FD0F9821464A
:1064E0000A9A2B4605F072FD384631463A460D9B16
:1064F00005F0B8FD089B009338463946109A05F020
:1065000087FBE898E690119821463A462B4605F01D
:106510005DFD0F9821460A9A2B4605F057FD384637
:1065200031463A460D9B05F09DFD089B0093384689
:106530003946109A05F06CFBE898E7907AE01088ED
:106540000C9A108099919891DA9E08460F46099D01
:10655000F59CF9F751FF2860DC9827606060A66021
:106560000C34DDA80EC80EC42EC82EC42EC82EC4EE
:106570007FB06CB0F0BDFF2010800021296020802A
:106580007FB06CB0F0BD002201233021695C00298E
:1065900000D076E6DDAA1ACF1AC23ACF3AC23ACF75
:1065A0003AC20B213046F9F795FD054642E000203E
:1065B0000690059D0796089F1190069801460D9C30
:1065C0000F9A4A43D219109B5A43119BD218D200FA
:1065D000A35889002E4655AD6B503546121DA25862
:1065E00015AB5A50401C01B28E42E9DC55A89AAE58
:1065F00096AC314622462B4605F0E8FC15A83146FC
:106600000A9A2B4605F0E2FC02232046079922460F
:1066100005F028FD01230093E8AA2046214605F055
:10662000F7FA119B9800DDA9E89A0A505B1C0B2B26
:106630001846C1D1F19EDDA89AA9DCAA0B2305F06A
:10664000C5FC09210E980F9101800B98C168DC9C54
:106650002046F9F7D9FE0146A8B2E69F0F281BD8BD
:1066600008280DD30846F9F776FE14E0FF201080C5
:106670000021099A11600C9908807FB06CB0F0BDC0
:10668000042803D381220846D10502E041220846AE
:106690001106F9F7B9FE01462B20C04386420D973B
:1066A00004DB0846F9F757FE014603E04020C043EB
:1066B000864244DD0E9A0C9C0B98408A002811D02B
:1066C0000B98038A95A80390DBA80290DAA80190A2
:1066D0000094DDA80D4603F099FC29462488DA9E33
:1066E000099D68E011910F98208000273D46109782
:1066F00005E00E9804887F1CB8B2A04211D8B8B249
:106700008000DDA90C5820461199FAF799F8002865
:10671000EFD1002DEDD10C98078001250F97109433
:10672000E7E7DBA805800F9A90B2201A012811D163
:106730000C9804800D9FDA973E46099D3AE0492067
:10674000C043864200DA8BE0FF2208469105F9F744
:106750005BFEA9E710200B990E5E012E00DA90E097
:10676000551CABB21846A1B2AAB28A4217D805E0AE
:106770000E990C88A1B2AAB28A4210D88000DDA975
:106780000C58204610991F46FAF74CF83B46002853
:1067900005D10C9805800B98068A0F95109430B29D
:1067A000C1186D1CA8B28142E2DC109EDA960F9CE3
:1067B000099D0D9F11993046F9F763FEFAF7EEF83F
:1067C000052800D3052095A90880A0B20E99098854
:1067D000814218D9401C611E0CB2A04218DA12A8DE
:1067E00098A9FEF76DFE0E980188481C491E0CB250
:1067F000A04221DA12A899A9FEF762FE9999989809
:10680000099D0D9FA4E600219891999108469FE665
:106810000022134608E09CB2A40012AF3D515B1C5D
:10682000491C0CB2A042DADB8DB20A2D1546F2D813
:10683000A400DDAD2D59EEE70022134608E09CB21E
:10684000A40012AF3D515B1C491C0CB2A042D1DB2D
:106850008DB20A2D1546F2D8A400DDAD2D59EEE714
:106860005320C043864200DB1BE70E460B9881692C
:106870002046F9F7D7FF00280C9C08D10B98808B95
:1068800007E01446099D0D9F1199109E93E70B9800
:10689000C08BFAF744F801463046F9F7B5FD119080
:1068A00021E70000F0B58BB01C4609930E46034665
:1068B00000200A9040480088224F05970AA90491B9
:1068C00003940292109C0194012500950B214143F1
:1068D00089B230331C4A3046FFF74EFC38680790C7
:1068E00078680890B868069033480088334F009560
:1068F00001940297324E30363249334A3346FEF71E
:106900006BFB0698F86207983863089878630998D3
:1069100000882E4905912E4904912E490391029732
:10692000019000962C4B284629462A46FEF74CFC3F
:10693000432001060A98F9F767FDFAF72FF80BB024
:10694000F0BDC04628A70102E0DF0102F0B589B022
:106950000F9F0E9C002815D01098079016480088AD
:10696000164E01250095019102960893144B303381
:106970001449154AFEF730FB089BF762079830630D
:10698000746303E00D484763C462002518880F490B
:1069900005910F4904910F49039108490291019013
:1069A00007483030009001210B4B28460A46FEF77D
:1069B0000BFC09B0F0BDC046CCAD0102A4D401026D
:1069C0008CA00102149F0102B4D2010258A401025A
:1069D000C8AD010268AD010270AD010230487047D8
:1069E000004870470CAE0102800037490918C86B97
:1069F0000022CA637047C046800033490918886C7A
:106A000000228A647047C04680B52F4AD369002BA4
:106A100001D0126A9847002080BDC046024908781C
:106A200000220A707047C0467CC9010200207047EE
:106A300080B5182905D803468A1E03481946F9F778
:106A400099FB002080BDC046D0AD0102B0B5024622
:106A50000020022901D2C043B0BD8C1E0F2C07D8E4
:106A6000044D284611462246F9F784FB002028559C
:106A7000B0BDC046ECAD0102B0B50246002002290F
:106A800001D2C043B0BD8C1E0F2C07D8044D284640
:106A900011462246F9F76EFB00202855B0BDC046CE
:106AA000FCAD01020849087800220A707047C04610
:106AB000B0B50446044DAA68002A02D0E968204611
:106AC00090472C610020B0BDDC970102B0B5D54DD8
:106AD000286A002819D02848007800281BD00128EF
:106AE00029D127480068CE498A8A904224DA28783A
:106AF000002804D000202870022002F045F9002070
:106B0000687068621D490870B0BD002068626870D6
:106B10001A490870B0BD2878002803D101202870D8
:106B200002F032F915480121017000206862697095
:106B3000C04313490860B0BD01246C706A6A531CDD
:106B40006B62C98A884209DD132AF4DB28780028A1
:106B50000DD12C70204602F017F908E0132AEADB69
:106B60002878002803D12C70204602F00DF900206F
:106B7000686202480470B0BD60990102DD960102AE
:106B80008499010280B5124801681F220A40026000
:106B900003200840022812D10E480268D30D02D00B
:106BA000FF231B06D2180C4B1A600C4A12680C4BC0
:106BB0001A6080680B4A1080000C0B4A10801A483B
:106BC0008268002A02D082680020904780BDC046BB
:106BD0007420004064400040C8D201027830004078
:106BE000CCD20102F0A001029AD4010280B50D4876
:106BF000016889070FD5052101600B48C17800297C
:106C000008D00021C170C168002903D0C268416862
:106C10000020904780BD054805A10B4A0BA308F052
:106C200045F9C0462C04004030940102343D010077
:106C30005048595F54494D45525F49525148616E21
:106C4000646C6572000000008D0A0000556E657866
:106C500070656374656420696E74657272757074B2
:106C60000000000070B50446401E012814D803201F
:106C7000084011D13F2040030818050B281980282F
:106C80000AD8164E317801204840294604F018F9F8
:106C9000641E6D1C002CF5D170BDC04680B500206F
:106CA000014603F055FE002800D080BD0B480121AD
:106CB000017080BD70B516460C460546FF22F9F7F7
:106CC0006BFA0548311805480278012050402A46E1
:106CD000234603F09DFF70BD00E0070460A9010298
:106CE000012000037047012040037047F0B585B0D4
:106CF00049484A49016006F003F8494EF08A4A21A2
:106D0000484F7852B18A4822B952B388FB62B27AAE
:106D10003A71B2893A827982B882B48D3C87049301
:106D2000BB867D20C500F1882846F9F7D3F9F881A4
:106D3000601E844160003862B08B3B2801D83C2043
:106D4000B0830020F083308B3749088043208000D7
:106D50007080728C0F2011460140130B6B435B183F
:106D600011050C0F64214C431B191206140F0A2243
:106D700054431B192D4C2380B38C1C4604401F0B1D
:106D80006F433C191F053F0F4F43E4191B061B0FB0
:106D90005343E318264C2380F38C1C4604401F0BFE
:106DA0006F433C191F053F0F4F43E4191B061B0F90
:106DB0005343E3181F4F3B80338D18401C0B6C432B
:106DC00020181C05240F4C4300191906090F5143C4
:106DD0004018194C2080032518A228462946049BF8
:106DE00009F0C0F87088C1B20091030A17A22846C2
:106DF000294609F0B7F80D4803880D4800883988FE
:106E00002288094C248800AE17C618A228462946B5
:106E100009F0A8F805B0F0BDF8950102598400000A
:106E200062A90102B0980102A49601029C96010297
:106E30009E960102A0960102A2960102C9E8B1B88D
:106E400049443A202578202E0D0A0000B9CCBCFE1A
:106E5000B0E6B1BE3A5557422D3447CAD6BBB7202B
:106E60005625642E25642E200D0A0000B7FECEF1B3
:106E7000C6F7B5D8D6B73A2025642E25642E2564EA
:106E80002E25643A25642E0D0A000000F0B583B06B
:106E900030480068C16B0901890F01D003B0F0BD13
:106EA000C16BC06B2C4D05404800400F0826029670
:106EB00086400227384602F0F1FD01907043C10B75
:106EC0004A1B26485043F9F71BF9044607F030FFE8
:106ED000032123A238461F4F0091234609F042F8B0
:106EE000F88A002817D0019840012946F9F7F2F8EE
:106EF00046431822324001200F2A014600D80021C3
:106F000073095B181B4CA3420DD8194DED1A6D0582
:106F10000F2A0CD80CE038680021C160112002F063
:106F2000ADFD03B0F0BD5D1C6D050F2A00D95642C2
:106F30002A0C029D2E4009018919A34202D800980B
:106F4000000400E04004081880183968086303B0A2
:106F5000F0BDC046C0940102FFFF1F0040420F0079
:106F600052434F33324B2070706D2025640D0A0060
:106F7000FF070000FE7F0000B0B582B01549086829
:106F80008269D2070CD00122C2610D69002D07D0A1
:106F900000686C46214607F057FC00212046A847B0
:106FA00002B0B0BDB0B582B00A490868026C920761
:106FB0000ED5026C012313430364CD68002D07D066
:106FC00000686C46214607F03FFC00212046A84798
:106FD00002B0B0BDC094010206480168032291438B
:106FE0000160016801220A43026000F04FFB07F0D4
:106FF000C1FEC0462800004080B50D490868002841
:1070000010D5224802680423032A01D01A4300E065
:107010001A460A601E490A68002A02D04168002008
:10702000904780BD03A00CA19E2211A307F03EFF54
:107030002C100140696E636C7564652F647269760B
:107040006572732F6D6B5F736C6565705F74696DCE
:1070500065722E6300000000534C4545505F544953
:107060004D45525F49525148616E646C6572000033
:10707000556E657870656374656420736C656570C2
:1070800020696E7465727275707400000C90010254
:10709000A0D40102B0B582B004460078002811D017
:1070A000094D01A908702868416A0029FCD101A98D
:1070B00001220020034609F01BFD611C60780028B6
:1070C0000C46EED102B0B0BDF8940102F0B50C78D8
:1070D0004D782D022C198D78C978090249190904B7
:1070E0000C1981000E4D6C509478D5781678527832
:1070F0000C4F7B50120292192B021B191B049A1879
:10710000094B5A50059A13785278084C079D6550E0
:107110004000074908181102C91848228152F0BDE1
:10712000C49F010288E0010228A0010224E00102BC
:107130001096010210B5CE4C216806290FD8012007
:1071400002468A4058210A4209D020600020A060EF
:107150002369002B03D06269002002219847C348AD
:107160002258062A12D801210B4693405822134276
:107170000CD021502018002181600369002B05D01C
:10718000AD20C000225801200221984747482258CC
:10719000062A11D801210B469340582213420BD0E6
:1071A00021502018002181600369002B04D003487E
:1071B0002258022001469847002010BDBC0A00005A
:1071C000F0B581B00024022803D9E443204601B081
:1071D000F0BD17460B46094E464309488519284617
:1071E00018302A2107A2FCF74FFF42202F5203201C
:1071F00003498851204601B0F0BDC0465405000047
:107200008CAE010225730000F0B585B0E04D2C680E
:10721000002C0CD0DD4FDE4CE659002E0CD0234F55
:10722000E659002E0DD00020C04305B0F0BD01ACE2
:107230000FC400272E4608E001AE0FC6E61901274D
:1072400003E001AE0FC6E6190227D04C30462146B6
:10725000FCF700FE022030607C432919029D4D603E
:10726000CF60039808610498486108464430CC31E7
:107270000122560210233246FCF7E2FFE4480019CF
:10728000B32189004118012D05D1B83001233246C0
:10729000FCF7C1FB04E0743010233246FCF7D0FF4A
:1072A00001980760002005B0F0BDC046A80A0000A4
:1072B00001460020022901D9C0437047E24A4A43EF
:1072C000E24988507047C046022806D8E649414343
:1072D000E64840180249401870474B20800070472C
:1072E000D4040000022802D94B2080007047DE49F8
:1072F0004143DE4840184D21090140587047C046BF
:10730000032801DB03487047D7494143D748401859
:1073100018307047413B0100022806DCD249414346
:10732000D24840184221405A704700207047C0465A
:10733000032801DB00207047CB494143CB4840186C
:1073400044307047022804DCC7494143C7484058CD
:10735000704700207047C046022805DCC2494143FF
:10736000C24840184068704700207047B0B50024FC
:10737000E14302280FD8BC4A4243BC4B9D58042D20
:1073800009D0991801220A600B69002B05D04A69BF
:107390000221984721460846B0BD2046B0BDC046F0
:1073A00010B50024022801D9E04310BDAE49414385
:1073B000AE4A0723535051180B69002B03D04A697A
:1073C000002421469847204610BDC046F0B581B044
:1073D0000024022803D9E443204601B0F0BD05464D
:1073E000A1486843A14906220A500F183846443084
:1073F0003946CC310122560210233246FCF720FFD9
:10740000786801280CD1B320800039183846B8308C
:1074100001233246FCF7FFFA3B69002B0CD1DBE776
:10742000B320800039183846743010233246FCF7F8
:1074300007FF3B69002BCFD07A6901212846984786
:10744000204601B0F0BDC04610B50024022801D985
:10745000E04310BD84494143844A51180B69002B15
:1074600002D04A6903219847204610BD5405000008
:107470008CAE0102F0B583B017460024E243022827
:107480001AD8002B18D00D46774941437748461843
:1074900070680128029312D1002F0AD0B836002458
:1074A00029193046FCF7BFFA002825D1641CA742F1
:1074B000F6D1029807600022104603B0F0BD019299
:1074C00074363046FCF777FE002811D00346426838
:1074D000BA4209D2196828461D46F8F74BFE2B46DA
:1074E000686802990860019430461946FCF739FE35
:1074F000019A104603B0F0BD0298046000221046C5
:1075000003B0F0BDF0B581B004460020C343022CA7
:1075100002D9184601B0F0BD15460E461B4A62431B
:107520001B498F187968012910D1002D28D01C46DD
:107530000090B83738463146FCF74EFA002821D182
:10754000761C6D1EF6D1009801B0F0BD0090743726
:1075500038462946FCF74AFE00280CD0044600684D
:1075600031462A46F8F706FE38462146FCF70EFE5D
:10757000009801B0F0BD07A02146FCF7EBFA009897
:1075800001B0F0BD204601B0F0BDC046540500007A
:107590008CAE0102536F636B65745B25755D205281
:1075A000656376204275666665722046756C6C0D63
:1075B0000A000000F0B583B0154607460022D0430C
:1075C000022F19D8002D17D000AB07C30F487843FE
:1075D0000F490E18443630462946FCF707FE0028AE
:1075E0000CD00446006801992A46F8F7C3FD3046DE
:1075F0002146FCF7CBFD029803B0F0BD05A039464B
:10760000FCF7A8FA009803B0F0BDC046540500008E
:107610008CAE0102736F636B65745B25645D2073D0
:10762000656E64206275662066756C6C0D0A0000DC
:1076300002460020022A04DC0B4B53430B4AD15074
:107640007047C0437047C046540500008CAE01022D
:10765000022801D9002070470349414303484018DC
:10766000034940587047C046540500008CAE0102E3
:10767000CC04000080B504480168491C0160006921
:10768000002800D0804780BD0CE00102014802497B
:10769000016070476C9001020026B80310B5C54820
:1076A0000024446110300221024A2346FFF7ACFD5A
:1076B000204610BD6977000070B584B0FDF732F93F
:1076C000012814D1FCF774FB204D6969022914D0FC
:1076D000002909D12978002921D0A969411A062950
:1076E00002D300212970A861002004B070BD1748A2
:1076F00000214161002004B070BDE969421A1449BB
:10770000144B9B8B9A4202D20A78002AECD0E86193
:107710000020087000F006F9002004B070BD0126BA
:107720006E61AB88E88829896A8900AC07C4B10218
:10773000094C0AA22046FCF7A7FC2869AA89214621
:10774000FFF73EFD2E70002004B070BD9896010238
:107750004093010262A9010278C5010225752E2518
:10776000752E25752E257500F0B58DB0032909D825
:107770007944097949008F4401070F155948416937
:1077800001290AD00DB0F0BD564841690129F9D14F
:10779000022141610DB0F0BD5248002141610170EC
:1077A0000DB0F0BD002500954E4C20694E494F4A62
:1077B0006B46FFF75FFE0028E4D103204CA2014690
:1077C00008F0D0FB48484DA10A22F8F708FD002830
:1077D00012D045484CA10F22F8F701FD0028D1D165
:1077E00041482C2101AA0C23FCF75FFC0298FCF70E
:1077F00035FB60870DB0F0BD3B482C2101AA0C235E
:10780000FCF753FC0498FCF729FB608780B2684EB4
:10781000B1888142B6D10298FCF769FCE062039816
:1078200001794279120251188279C3791B029A18A0
:10783000120451188278C378077840780002C01982
:107840001B029A1812041018206261620598FCF756
:1078500005FBA0870698FCF74AFCE0870798FCF731
:1078600046FC4027E0530898FCF741FC4221605455
:10787000E16A491E062901D80122A270062926D8EC
:107880007944097949008F440318111C221E150000
:10789000E08FB082E05BF082A08FB18D814216D084
:1078A0001E4902220A60B0851D4800E01A480121E5
:1078B00001700CE00120B08709E018480560B5852B
:1078C00005E0B58703E0C0B23C214143B18301200C
:1078D000A07000F027F807F0B3F925626562A57083
:1078E0000DB0F0BD9896010278C50102FF030000BB
:1078F000CAD5B5BDCAFDBEDD0D0A000024696E7390
:1079000074727563742C0000246D65737361676510
:107910005F7265706C792C00DC960102D0980102D0
:1079200038900102F0B5C7B0214CA0881490214DC9
:1079300068781390FBF7E2FE1290A08D11906878A2
:1079400010901D4800780F90A08A0E90E08A0D904C
:107950001A48C0C81A490A684968AB78194C2468A3
:107960002035089209910A950B930C941298009077
:1079700011980190109802900F9803900E9804901F
:107980000D9805A9C1C11398002801D00F4A00E045
:107990000D4A15ADC8212846149B09F0BBFD0246CF
:1079A000044800692946FFF705FE47B0F0BDC04610
:1079B00062A9010298960102B89801024099010259
:1079C00038990102849901024D3201000C32010004
:1079D00080B582B00E4908680022C2600192CA6870
:1079E000002A02D0016801A8904702B080BDC046BD
:1079F00080B582B0064908690022C2600122019266
:107A0000CA69002A02D0016801A8904702B080BD6F
:107A100018930102F0B582B0144C20780090002831
:107A20001DD0134B24330025019504E09B1C6D1CD5
:107A30000098854215D262196026905D471C9755C3
:107A40000928F3D80199C8B222181C88975540001C
:107A5000074A10188484054C491C0191E6E7002070
:107A600001900198207002B0F0BDC04660990102FB
:107A70003C9A0102F0B589B009F092FCE94C6078BB
:107A800009F034FAE8498A8807A882800A88498878
:107A900009048918079105F0B5F96078052804D024
:107AA0000222E249092804D104E00122DF49092821
:107AB00000D0891849792078621C09F0DBFA607AD5
:107AC00006F0C8FCDA48DB4904F0A0FCDA4C207868
:107AD0000026002806960AD0D8491A31D84A03460B
:107AE00010CA0C80891C5B1EFAD14600D24CD54DC1
:107AF000A872D54800886871D449097829706178DE
:107B0000E970000AA871481C607028460B30CB4F02
:107B100039464C3103913246F8F72CFB70190B3083
:107B200039461A313246F8F725FB2020687206984C
:107B30002071E0886870000AA870C3200690840154
:107B400006F0F8F90319BC48C362BB48007881000D
:107B50000D3101222846059209F07EFCB649886263
:107B6000B548C46A06F07CF90019B34C06F0D4FDA0
:107B700005460E46AB48007B06F05AFC81B2C90BA5
:107B8000401800B2C11740102818A0657141E16586
:107B900006F0D0F9A06104F0ABFB0028FBD106F0A1
:107BA000C9F9E0617D200601002738463946324692
:107BB00009F028FCA06225460698040206F0BAF9EE
:107BC000297861434118A3480818421C01D1A048F4
:107BD0000818994C206306F0ADF96063216B884268
:107BE00004D39D4A8918884200D897E006F0A2F98C
:107BF000606306F09FF9E06104F07AFB0028FBD196
:107C000006F098F92062607902284FD001287DD1D2
:107C100000206071914D697A212971D16979AA7921
:107C200012025118884A1288914269D1874909780D
:107C30002A788A4264D16978AA7812025118A181FF
:107C4000E278002A40D02278002A0BD07B4B4C33BC
:107C500000201C888C4204D09B1C401C8242F8D11E
:107C60001046754CC0B2E081236EA16BA26D7B4DB6
:107C70002C4622340094704C0191029229461A310C
:107C80001E352A46FFF722FAE089E178884208D3B8
:107C900041006A4A5118A2894C23CA522178491CD2
:107CA00021700521654A11546C4824E00020607160
:107CB0000146324609F0A6FBA06206F03BF92062BD
:107CC00006F038F9A06121E04C205C4A1152059879
:107CD000207005201070236EA06BA16D2A46223201
:107CE00000920190029129461A312A461E32002044
:107CF000FFF7ECF928469621F8F755FA0020208284
:107D000000200146324609F07DFBA062226B606BC9
:107D100051495118904200D365E767E7A06DE16DC6
:107D2000FBF7E8FAA770207800282FD044484C21B0
:107D30003D463C46414B05E0891C001DFAB26D1CD6
:107D400095421AD25E5D002EF6D0761E5E55A300D7
:107D50000693F6B22246424CE650384B5E5A530028
:107D6000404CE6527F1C344B9F7003683E4C069E8D
:107D7000A3511446314B541CDEE705922E48C770C0
:107D800007700497F8B2022806D228E0E778059732
:107D90000497F8B2022822D30598441E00210694C5
:107DA00003E0491C069CA14219D02F4A10682D4BB4
:107DB0002B4F0FE0156050605D881E885E801D802F
:107DC00060CF083F3E607D60641E121D9B1C3F1DFE
:107DD000002CE6D05568A842ECDC2846F4E704986D
:107DE0000006059C10D062001E490398F8F7C2F9FE
:107DF000A20013481C49F8F7BDF9104A184802C8F8
:107E00001170521C641EFAD10B488389174801680F
:107E1000406800910190032015A2014608F0A2F8E5
:107E200009B0F0BDC0900102DC1F0100F4A0010206
:107E30009D0101008DEB0000E096010230980102E7
:107E400050D20102FEE90102DC980102B49801025D
:107E500081E7010080E701000026B803A0D30102FA
:107E600004E90102CCE9010268E90102509601022D
:107E7000BBF9D5BE4944A3BA25582CBEE0C0EB3AA5
:107E800020256C660D0A000080B5002008F0E8FA95
:107E900080BD80B5012008F0E3FA80BDF0B581B067
:107EA00003F06CFD164CE060A178002901D001B010
:107EB000F0BD21790029FAD10121217100281BD0C0
:107EC0008D02281AA168814216D0624E2F46A06802
:107ED000305C21698847A068401CA060681EA168CA
:107EE000814201DD0020A060E168A068022F03D379
:107EF000691A7F1E8842EAD10020207101B0F0BDCE
:107F0000E8950102B0B5294C2368002B07D0022B5D
:107F10000DD0012B39D109F00FFA00F011FC09F056
:107F2000E9F92368022B1FD0012B18D02DE0204D3A
:107F3000287800282FD003201EA2014608F012F84E
:107F40000020287009F0F8F900F072FD1C4D28702F
:107F500009F0D0F928780028E3D0012020601948E2
:107F600000214181012310E011480178002909D145
:107F700014494A89531C4B81152A03D301220270EC
:107F80000020488108F07EFF2368032014A20146E8
:107F900007F0E8FFB0BD0B48408914210B1A0320FD
:107FA00009A2014607F0DEFFBBE7C046D0980102F8
:107FB00038900102BFAAC6F4CBD1CBF70D0A00005E
:107FC000B598010260990102B5C8B4FDBDF8C8EBCF
:107FD000CBD1CBF7C4A3CABDA3BA25640D0A000058
:107FE000555742D7B4CCACA3BA25640D0A000000A3
:107FF00080B506480068022805D809F09DF9FFF70A
:1080000039FD09F077F908F03DFF80BDD0980102F5
:1080100070B50E2500242846214603F0ABFD0D2047
:10802000214603F0A7FD0124204608F021F904268B
:108030002846314603F09EFD0920314603F09AFDA3
:10804000204601F041FBA2020249034B204608F002
:108050000DFC70BD10CE0102A50A010080B50328F9
:1080600010D800290ED07C224243BF488018C26835
:10807000012A07D12030FBF7D6FC002801D00020D0
:10808000C04380BD0020C04380BDC046F0B589B06C
:108090000022D543032800D9ABE00C46002900D1CB
:1080A000A7E00095216A0727534DA9420EDC574DE2
:1080B000A9421ADD564A91422FDC4B22D501A94232
:1080C0003ED0120291424BD1042246E04B4A9142EB
:1080D00017DD4B4A91422ADCE1221203914231D052
:1080E000494A91423CD10C2237E04B252E01B14246
:1080F00033D06A01914227D0AA01914230D10222A5
:108100002BE0E1225502A94220D09502A9421FD0BE
:10811000D202914224D109221FE04B225202914205
:1081200018D0E122120291421AD1062215E0E12272
:108130005203914210D0334A914211D10D220CE0EA
:1081400003220AE00A2208E0012206E0072204E0F6
:10815000082202E0052200E00B22D1002D4A5758E8
:108160007C214143804A505056182068B0606068B6
:10817000F060A1683161E268726100250595032312
:1081800004930395029501970695079501231B0219
:108190000893012807D000280AD18818009A80186F
:1081A000B161F06104E0304620300123FBF733FC7D
:1081B000206970636069B063E069B067A069F063CB
:1081C000706801A908F07EFA2068012806D83046B8
:1081D0004030234610330ECBFCF732F8606801289C
:1081E00007D1301D7036006801220B4B314608F074
:1081F0003DFB284609B0F0BDFFC10100FF0F0E0096
:10820000FF1F1C0080841E0040420F007F250000DD
:10821000FF9500000C200100BD0A0100B0B50C461E
:108220007C214843504A15182846FBF713FE6C6022
:108230000020B0BDF0B583B00024E743032800D987
:108240008EE00E46002900D18AE01546002A00D1B2
:1082500086E07C214143444841188868022832D096
:1082600001283AD000282BD1EFF31080C00702D1AB
:10827000EFF3108072B60291084640300190294613
:10828000FBF7B4FF002863D0014601980F46FBF7C7
:108290007DFF386831462A46F7F76CFF0198FBF7F7
:1082A0008AFFEFF31081C90703D1EFF3108172B693
:1082B00062B602994D6806C82C4B284608F018FC97
:1082C000204603B0F0BD4868002431462A462346C4
:1082D00008F00EFC204603B0F0BDEFF31080C0079D
:1082E00002D1EFF3108072B602910846403001903F
:1082F0002946FBF77BFF00281ED0014601980F4658
:10830000FBF744FF386831462A46F7F733FF0198F8
:10831000FBF751FFEFF31081C90703D1EFF3108191
:1083200072B662B602994D6806C8104B284608F02E
:10833000DFFB204603B0F0BDEFF31080C0070FD184
:10834000EFF3108072B662B63C46204603B0F0BD33
:10835000EFF31080C00703D1EFF3108072B662B65E
:108360003C46204603B0F0BD88BE0102C10D0100AD
:10837000B0B582B0602833D0622843D0642854D18D
:1083800001A82F490180EFF3108072B60024204627
:10839000214602F0DDFA2B4D002805D10120020311
:1083A0000020294602F02EFA103501AA02232046A9
:1083B000294602F005FF62B623A0FEF76BFE64209B
:1083C0001B490C5206F03CFC1A4801F037FCBFF385
:1083D0004F8F194819490160BFF34F8F00BFFDE768
:1083E0006020134900220A5206F02AFC114801F0CD
:1083F00025FCBFF34F8F104810490160BFF34F8F2A
:1084000000BFFDE762200A4900220A520A8006F0F6
:1084100017FC084801F012FCBFF34F8F06480749CC
:108420000160BFF34F8F00BFFDE702B0B0BDC04693
:1084300062A90102A08601000CED00E00400FA052B
:10844000AAAA000000D00204BDF8C8EBC9FDBCB662
:10845000C4A3CABD0D0A0000F0B5D1B0A74EA8490B
:108460000A78002A25D0F28B002A22D1A54FBA68BB
:10847000082A00D990E0930001A4E3589F46C04623
:10848000A58400009985000099850000A985000059
:10849000D3850000DD850000E7850000B78500007A
:1084A000F1850000552800D0BBE00120B86051B034
:1084B000F0BD4978002900D1B7E0924D6A7996491C
:1084C0008854A979A871E971521C6A710A2800D0F0
:1084D000ABE00D2900D0A8E003A8019037A80090D8
:1084E0002C4630348C488D491DAB2246F7F794FE5C
:1084F000E8608BA105222046F7F771FE00282AD1FB
:10850000F08B002805D0032087A2834B014607F09B
:1085100029FD1DA80024214609F0C5FCA861E961D8
:10852000824B2246F8F7C4F9002814D1804800F0A5
:10853000F1FF1DA80024214609F0B5FC28626962FC
:1085400037A8214609F0AFFCA862E96203A8F7F753
:10855000F5FE286100E0286900266E71002806D02B
:1085600074480670744801210170744806806A4896
:108570009621F7F718FE1DA864242146F7F713FE8D
:1085800037A82146F7F70FFE03A82146F7F70BFEA1
:108590006E71EE8051B0F0BDAA2838D1012A36D1D3
:1085A0000220B86051B0F0BD0421B9600021B9705B
:1085B000787051B0F0BD3979534A5054481C387125
:1085C0007978491FC0B281422FD10820B86051B0DC
:1085D000F0BD0522BA60887051B0F0BD0621B960C7
:1085E000B87051B0F0BD0721B960387051B0F0BD1E
:1085F0007A78062A02921AD3531F0025424A2C4643
:10860000565DA419A4B26D1C9D42F9DB10E003284D
:1086100007D1022A05D10120F8700320B86051B0BB
:10862000F0BD0020B870B860787051B0F0BD002483
:108630002018029A821888781118BD7849193C7858
:108640000919FA78002A00D0C91C2C4EC9B2FF299A
:1086500035D1012809D0022831D11E2D36D1FFF79E
:10866000D7FC0120F08351B0F0BD284A947103205B
:1086700010719070AA2050705520107068085071C9
:10868000651DD570400031181646D01D2246F7F7FB
:1086900071FD301DE11CEAB2D21C037892B2D218EF
:1086A000401C491EF9D1A019D143C171090A0172B8
:1086B0000934012000233146224608F019FA00202F
:1086C000B870B8603871787051B0F0BD70190E4E46
:1086D00031462246F7F74EFD3078012802D1284670
:1086E000FFF746FE06F0ACFABFF34F8F0848094982
:1086F0000160BFF34F8F00BFFDE7C04662A90102D2
:108700001890010218990102ACCD01020C9B0102E4
:108710000CED00E00400FA0514CD0102A9310100BE
:10872000474E474741000000257300000000F03F1E
:10873000C9AD010228940102DF960102CAAD01020F
:10874000F0B589B008F02CFE9B489C4903F05EFE12
:108750009B4D00242C71EC7005F0ECFBE8610420CB
:1087600003F094F9974E728820460694214608F04B
:1087700049FE05F0DFFB044628632720410170888D
:1087800048430A21F7F7A6FC68630119481C00D08A
:108790000846A86305F0CEFBE863A96B8A4C8842C3
:1087A00002D30919884233D9884F894E05F0C2FB9C
:1087B000E86303F09DFD00280AD0FCF771F805F08E
:1087C000B9FBE863A96B8842F3D909198842F0D252
:1087D000E87801280FD138783178814211D1787A40
:1087E00020280ED17879B979090208187949898D3C
:1087F000884206D115E0734842880020014608F0FF
:1088000001FEA96BE86B8842D0D309198842CDD804
:108810002879002800D1B1E0042003F027F909B03D
:10882000F0BD0120287105F085FBA861B87AA87019
:10883000024605907879B97909020C18EC8039461E
:108840000B315600644802913246F7F793FCF11958
:10885000059F0B31604832303246F7F78BFC002F12
:10886000069872D05B48808904905C4803680026B3
:10887000594A039326E0A91860230027CF545100DA
:10888000574A51188C8400B2F8F750F83A46554BC5
:10889000F7F7E8FE08900791686AF8F747F83A4654
:1088A000504BF7F7DFFE02460B4608980799F7F79B
:1088B00027FEF8F7A1F86862059F474A039B761CDC
:1088C000BE4227D07000115A8B42F8D11118488E41
:1088D000049A80184886297800290ED0404B24330A
:1088E00000221F88A7420DD09B1C521C9142F8D138
:1088F0000B460A46172908D9BDE700231A4617294F
:1089000003D9B8E7D3B21729B5D88B42B3D1491CE4
:108910002970B0E7002F0FD0304801680020029C7A
:10892000227863781B029A18914207D0A41C401C3D
:108930008742F5D1384608E0002006E0C4B2204660
:10894000FAF756FCA878A04201D1FAF751FC264864
:10895000002101702548623006F0EEF90520285606
:108960001C498B8D696A00910190032020A2014669
:1089700007F0F8FA2879002800D04DE71B4806F0E8
:10898000DBF9194C2378032022A2014607F0EAFA0A
:108990002078411C2170062800D23DE7234802219F
:1089A0000160069820706881012006490870042043
:1089B00003F05CF809B0F0BD75010100E5EA0000C4
:1089C0006099010238900102007C312508D3010230
:1089D000B498010262A90102949A0102DC98010292
:1089E0003C9A01020000E03F06D301021A3F00005A
:1089F000B1EAC7A94944A3BA25582CBEE0C0EB3A56
:108A000020256420D0C5BAC5C7BFB6C8A3BA25649F
:108A10002E0D0A00B2E2BEE0CAA7B0DCA3ACBCC611
:108A2000CAFDA3BA25640D0A00000000D098010217
:108A3000F0B587B008F0B4FC8C4C607808F056FABA
:108A40008B498A8805A882800A8849880904891880
:108A5000059104F0D7F96078052804D002228549F1
:108A6000092804D104E001228249092800D089188C
:108A700049792078621C08F0FDFA607A05F0EAFC7A
:108A80007D487E4903F0C2FC7D4E0025F57005F05F
:108A900051FAF061042002F0F9FF7A4A284629468B
:108AA00008F0B0FC05F046FA77493063716341186D
:108AB000481C00D00846B06305F03CFAF063B16B87
:108AC000724C884203D30919884200D8BFE0704F26
:108AD00003F00EFC00280AD0FBF7E2FE05F02AFAAC
:108AE000F063B16B8842F3D909198842F0D205F0DE
:108AF00021FAB061F07801280FD1387865490978FA
:108B000081420AD1787A202807D17879B979090287
:108B100008186149898D884210D005F00BFAF06180
:108B2000002528462946574A08F06CFCB16BF06BCB
:108B30008842CDD309198842CAD888E005F0FAF9ED
:108B4000B061B87AB070024602907879B9790902BA
:108B50000C18F48039460B315500504800912A46D4
:108B6000F7F708FBE919029F0B314C4832302A46CF
:108B7000F7F700FB002F62D0494803680025474AF9
:108B8000019326E0B11860230027CF545100454AD5
:108B900051188C8400B2F7F7C9FE3A46424BF7F7FA
:108BA00061FD04900391706AF7F7C0FE3A463E4BB0
:108BB000F7F758FD02460B4604980399F7F7A0FC17
:108BC000F7F71AFF7062029F344A019B6D1CBD4289
:108BD00024D06800115A8B42F8D11018408E317899
:108BE00000290ED02F4B243300221F88A7420DD01E
:108BF0009B1C521C9142F8D10B460A46172908D9F2
:108C0000C0E700231A46172903D9BBE7D3B21729B7
:108C1000B8D88B42B6D1491C3170B3E7002F0ED0C3
:108C20001F4801680020009C227863781B029A1874
:108C3000914212D0A41C401C8742F5D100E00027CD
:108C40003846FAF7D5FA194806F076F801250420D7
:108C500002F00CFF284607B0F0BDC4B22046FAF778
:108C6000C7FAB778A742EED1EAE7C046B290010250
:108C7000E21F0100F4A0010275010100E5EA000015
:108C80006099010280841E000098E00E007C31256E
:108C900008D30102B498010262A90102949A010268
:108CA000DC9801023C9A01020000E03F7C3F00009A
:108CB00080B582B0002001900448C268002A02D02A
:108CC00001A80021904702B080BDC04688950102EE
:108CD000F0B583B000242046FDF7E0FFFEF703F86F
:108CE000274EB060FDF7FCFF7060264F0BE001A837
:108CF000C1888088084319D101A840882418083405
:108D0000B068844235D201AD082128462246FDF7DD
:108D1000D1FF28880028EAD0B8422AD001AD04212A
:108D2000284600F075FFA9888842E5D03460B06815
:108D300084420CD201AD022128462246FDF7BAFF3B
:108D40002888B84203D0A41CB0688442F2D370686B
:108D50002118491E4042084030600DD000242546AD
:108D600001202946FDF77EFF03CE4D19083E8542BE
:108D7000F6D3346003B0F0BD0024346003B0F0BD1E
:108D800048970102FFFF000010B5054C6070FEF728
:108D9000C9FD6078022801D10020607010BDC04676
:108DA00098960102F0B585B01F4604920646C81792
:108DB0000C1844400A2C039114D301250A212046A3
:108DC000F7F788F96D1C632C0446F7D804998D4297
:108DD00000D329460A9C002F09D00398002808D404
:108DE000002207E0012504998D42F2D2F2E7002229
:108DF00005E00122042323409B081343FA1A0223AF
:108E0000234004980028029412D1002B10D0F4685B
:108E1000002C62D40398002825D40298400734D54A
:108E20007068B5686F1C87422FD830682B2423E008
:108E3000E407ECD1002A0AD1E9E737682020385549
:108E4000B560F068441CF460521E002CDFD49142DF
:108E5000DDD27768B468651CBD42EED9F468521E55
:108E6000002CF4D5D3E7404203907068B5686F1CBE
:108E700087420AD830682D244455B760F068441CF6
:108E8000F4600025ED43A84227DB002B1CD0012015
:108E9000029B1840049B184316D1002A03D113E00B
:108EA000521E002C0ED491420CD27068B3685D1C27
:108EB0008542F5D830683024C454B560F068441C4D
:108EC000F460EDE7002C08D40092029801900A2289
:108ED00030460399049B00F003F805B0F0BD000094
:108EE000F0B587B01F4615460290012406919142C5
:108EF000009407D3012406982946F7F7EBF8641C81
:108F0000A842F9D20D980C9ABC42039700D303945F
:108F100000990140002A009109D00029029C25D126
:108F20002021800705D40846002F11D004E0029CC0
:108F30001CE03020002F0BD0084609E0236858546D
:108F4000A260E168491CE1603246721E00290DD41E
:108F5000039991420AD216466368A1684A1C9A4254
:108F6000ECD9E1683246721E0029F1D5E06800288C
:108F700059D40590012401E07F1E6C43022FFBD2DF
:108F8000069821461646F7F7A5F83246A842F4D2CD
:108F9000029880680490069F0195069738462146FE
:108FA000F7F798F8049D691C029F7A68914206D9E8
:108FB000069F059A019D0592002A0ED516E01B4AD0
:108FC000125C3B685A55B960FA68521CFA60049109
:108FD000069F019D0592002A08D460433F1A20464F
:108FE0002946F7F777F8AC420446D6D20098002815
:108FF000029C059B049D16D0002E14D0701C01E02D
:10900000002B10D4401E039981420CD2691C626867
:109010009142F5D8226820235355A160E268531C81
:10902000E3600D46ECE707B0F0BDC046E822010062
:10903000F0B583B001900291002923D00025124F92
:109040002E460AE013480818410F4018C010387225
:10905000761CB0B20299884214D2019800884B2441
:10906000210100B200F018F8400061014018388377
:1090700001B2064881422846E9DB05488142E1DD2C
:109080006420E4E703B0F0BDB0980102E40C0000F6
:10909000041000001CF3FFFF074A904201DD054A5F
:1090A000801800B24143C817400D0818C00A00B22A
:1090B0007047C04600F0FFFFFF07000010B50078C2
:1090C000012819D1AC480269012A04D1614A136808
:1090D0000124A3431360032905D080214161C269A3
:1090E000002A05D107E001214161C269002A02D0AE
:1090F00001898069904710BDFF222E32024803A1EA
:1091000007A305F0D3FEC0469C2E01006164635F97
:10911000646D615F63616C6C6261636B0000000091
:10912000556E657870656374656420646D61206355
:1091300068616E6E656C0D0A00000000F0B58DB0C0
:109140000D460124EFF31081214002D1EFF310838B
:1091500072B6894E73690F2B06DD102B37D0402B6A
:109160002FD0802B2DD005E0002B2AD0012B01D150
:1091700010237361B5813581B061F261002900D19E
:1091800062B63179002929D00294304C05A90A46EB
:1091900004950390E8CCE8C2E8CCE8C2029C2046E3
:1091A00000F0BCFD2A4800902A4D2946083120468F
:1091B000039A049B00F022FE2C60002420460DB090
:1091C000F0BD0029FAD162B620460DB0F0BD0224F0
:1091D0000029F3D162B620460DB0F0BD31780029E8
:1091E00007D01C48072181610460002420460DB08F
:1091F000F0BD3269B3891749002B15D0B5693089A4
:10920000012A02D0002A03D003E09FB2874200D196
:109210000C604F68FF07FCD08F6880C55B1E1F0481
:10922000EED10023B381B561012A02D10A68A243BD
:109230000A607461F2690024002ABFD0B3693189E1
:109240008800181A904720460DB0F0BD2823010071
:10925000BD90000008D00140F0B581B0002856D084
:109260000446424EF068800754D41325284600F087
:109270000DFC284605F0DAFA2768616801253846B2
:109280002840CA07920F1018227C1207120E80186D
:10929000627C1207120D8018A27C1207120C801833
:1092A000627D13071B0AC01812091206801830606D
:1092B0007D2006020029304600D12D48E3681A0AB5
:1092C0007D2A1A4629D22B4EB3422AD200292BD00E
:1092D000002A2946254E00D01146F6F7FBFE401E17
:1092E00080B2706024480761E27C0270237D0371C4
:1092F000224F3E686902A468012C1BD02C02264331
:109300003E60002B1ED00121184A116329E0012084
:1093100001B0F0BD022001B0F0BD3246154EB3429F
:10932000D4D333460029D3D11A46002A29460F4EFA
:10933000D2D1D2E73F242401A6437618F0363E600E
:10934000002BE0D1002A0CD0FF2212020C4B1C682B
:1093500094430122D203A2181A60304A1160304AA5
:10936000116001214161002001B0F0BD00D0014039
:109370000026B80380841E00989501022C06004048
:1093800008E400E070B5002801D0012070BD0C4653
:109390001625284600F07AFB284605F047FA002CEF
:1093A00005D01B48183014222146F6F7E3FE282189
:1093B0001748415C002915D04168002916D40322C2
:1093C0000B469343144A9C588D07ED0EFF26AE4082
:1093D000B4439C501F220A40012191400F4A116062
:1093E0000F4A116001210161002070BD8A07D20E71
:1093F000FF2393400F220A40083A03218A4305497C
:1094000054589C43545001210161002070BDC04656
:10941000709001021CED00E000E400E080E200E05A
:1094200000E100E080B568480021017061480078E3
:10943000C001614909788901014360480078400111
:1094400008435F490978090101435E480078C0007C
:1094500008435E490978490001435D4800780843A4
:10946000C0B2FBF759F980BD80B5574801210170A2
:109470005148007880014F490978C90101434F489C
:109480000078400108434E490978090101434D48DD
:109490000078C00008434D490978490001434C4811
:1094A0000078084304210143C8B2FBF735F980BDB9
:1094B0005A21014A505270478CA00102F0B581B088
:1094C00013490A78002A13D0052A01D104220A7010
:1094D0009300CD18561C00231C462F686F60F917A7
:1094E000DB194C412D1F761E012EF6DC084902E0E7
:1094F0000022134614464860521C0A70C1171818FF
:109500006141D2B20023F6F70FFE01B0F0BDC046B4
:10951000B8950102F0B581B004460078414241415E
:10952000217024480078C00123490978890101434A
:109530002248007840010843214909780901014384
:1095400020480078C00008431F4F39788900014344
:109550001E4D2878400008431D4E31780143C8B2A3
:10956000FBF7DAF87D20C00000F068FB207841426C
:10957000414121700F480078C0010F4909788901E5
:1095800001430E480078400108430D49097809015C
:1095900001430C480078C000084339788900014332
:1095A00028784000084331780143C8B2FBF7B4F88B
:1095B00001B0F0BD109F0102DE9601022994010264
:1095C00094EA0102C9AD0102119F010254A30102F4
:1095D00055A30102B0B5094D2860022400212046A0
:1095E0000A4602F05BFA01210522204602F0EAFA5F
:1095F0002A680321204602F0C9F9B0BD0C9F010280
:109600005C219D480022425282847A214184028456
:10961000C2830283C2820282114941608260C260B9
:109620003D21490441834182090C81838182704735
:109630005C2191480022425282847A214184028432
:10964000C2830283C2820282054941608260C26095
:109650003D21490441834182090C81838182704705
:109660004C37373770B5BF484C21016001252C02BB
:10967000601C00F08BF9322000F0E0FA00F044F9B1
:10968000284600F04BF9284600F05AF800F036F969
:109690000C4800F07BF900263046314600F086FA8F
:1096A0002846314600F082FA204600F06FF9022089
:1096B00000F06CF94834204605F070FB05F0CEFB55
:1096C00070BDC0460102000010B50446072106F037
:1096D000A7FA0148046010BD8C96010270B5052000
:1096E0000424214602F046FA0620214602F042FAFE
:1096F0000A20214602F03EFA0920214602F03AFAF9
:1097000000240121204602F035FA02252046294690
:10971000224602F057FA0B2630462146224602F036
:10972000BDF930462946224602F04CFA70BD0000D1
:1097300002480168012291430160704758000040CF
:1097400002490A6802408242FBD17047046000402F
:10975000B0B5494D28688107484C0ED528797F213E
:10976000084022688A431018206023680B400220BA
:109770000321434A06F0F6FB286880040ED55E20DC
:10978000285C7F21084062688A4310186060636823
:109790000B40022003213B4A06F0E4FB172000F0B7
:1097A00075F93948016802220A4301218A4302609F
:1097B00036483749016037480021C17181791F253A
:1097C00029408171817A427C837C1B029A18C37C78
:1097D0001B04D218037D1B06D2182F4B9A4218D1B6
:1097E000427B837B1B029A18C37B1B04D218037C29
:1097F0001B06D218294B9A420BD1C27A037B491E11
:10980000122906D819028918254A914201D120212E
:1098100001720178CA0602D11022114301701C3C6A
:1098200020682021884320601E481F49016041684C
:109830000029FCD503F04AFA0446022003211BA2AA
:10984000234606F08FFB0A20C441032C05D80220D2
:1098500003211DA206F086FBFEE71848C1680F220F
:109860009143C1600168164A0A4002601920000154
:10987000144948600D60B0BDF4A0010248000040EA
:10988000E42E0100CE2E0100040200400C06004030
:10989000AF6B100A6B0001404D383650312E323616
:1098A0000734000000600040FE1C008043686970BF
:1098B0002049443A20253038780D0A00C86000401D
:1098C000FEFFC3FF0C0400404F6C642063686970A6
:1098D000206D6F64656C206973206E6F74207375E2
:1098E00070706F7274656420627920746869732087
:1098F00053444B2121210D0A0000000080B51720A0
:1099000000F0BCF8002080BD10B51724204600F000
:10991000BDF8204604F08AFF002010BD0121C907D0
:1099200001430148016070470060004010B582B0FB
:1099300003460C480168022B01DD012204E00222EB
:10994000D24393420CDCFF227F248A18A143224099
:109950008918016000920448032104A206F002FB6A
:1099600002B010BD48000040020800005854414CAD
:10997000206C6F6164206361702074756E652025B2
:1099800064203A2025640D0A0000000010B5C1B221
:10999000000AC2B202290CD0012913D0002930D10B
:1099A000911E7F4802291BD20121032A2AD0490493
:1099B00029E07B484168002A1FD00246203A114323
:1099C000416010BD76480168D31E022B10D3012AD6
:1099D00029D0002A41D1012292079143016010BD94
:1099E000002A16D10121490702688A43026010BD8E
:1099F0000123042A1FD05A041EE00122920791433A
:109A0000416010BD0904194A7F32C36A13405918D6
:109A1000C16217498A699207FCD50121490702688A
:109A20000A43026010BD0522120791430246203A04
:109A30000A43026010BD1A04836A0C4C1C40A21831
:109A400082620B4A131F00241C600A4B0A4C1C60E4
:109A50000D235B0214681C431460054A93695B067E
:109A6000FCD5052212071143016010BD80FFFCFFE9
:109A70001402004004010040FF0F0000012181405A
:109A8000474802688A4302607047C046012181400E
:109A9000434802680A4302607047C04610B5052873
:109AA00011D8C0467844007940008744020E19243A
:109AB00034393B490A680868C0003CD53A48203927
:109AC0000A425DD03BE0002010BD35490A680868B5
:109AD000C00035D534480B46203B1A4237D134E01C
:109AE0002F490A680868C00036D52F480B46203B2E
:109AF0001A424CD135E02A494C680120C0030A685B
:109B00000B46203B1C421AD00C68E4003BD5264C87
:109B10001A423CD03AE0224800680120C00310BD40
:109B20001F490A680868C0001ED51F480B46203B25
:109B30001A4220D11DE01B4820390A4220D010BD16
:109B400018480B46203B1A4201D10120C003496846
:109B50008900890FC84010BD12480B46203B1A42AD
:109B600015D10120C00312E00E480B46203B1A42DB
:109B700001D10120C00349680903890FC84010BD05
:109B80000120C00310BD074C1A4200D020464A688D
:109B90009200920FD04049680901890FC84010BD5A
:109BA00020000040006CDC020026B80304282CD8FA
:109BB000164AC0467844007940008744020A121AC7
:109BC00021000320000713688343880780081818C2
:109BD0001AE00320800613688343880700091818D9
:109BE00012E003208004136883438807000B1818D1
:109BF0000AE0FF200002136883430802181803E0FC
:109C00001068FF23984340181060704724000040FC
:109C1000B0B5002200290CD0074B047895B22D0A6C
:109C200065406C001C5B12026240491E401C00290A
:109C3000F3D190B2B0BDC046E820010000280AD0A0
:109C400030B407252C02CD25641960434009123831
:109C5000001FFDD830BC7047F0B583B01F461646D4
:109C60000D460146E8680291F6F7CEFB04460F2E3A
:109C700011D8082E04D320462146F6F76CFB09E0E4
:109C8000042E02D38120C10501E0412001062046B7
:109C9000F6F7BAFB04460999089E2B20C043874279
:109CA00005DB20460F462146F6F755FB0DE03F2029
:109CB000C04387420BDA4920C04387420CDBFF20B8
:109CC0000F4681052046F6F79FFB39460446688A11
:109CD0000880346003B0F0BD01915320C043874237
:109CE00006DB20462146F6F736FB0446688A10E07C
:109CF000A8690299F6F7B2FD002801D1A88B00E00F
:109D0000E88BF6F70CFE01462046F6F77DFB04468D
:109D1000002001990880346003B0F0BDF0B581B037
:109D200005460120072D66D80C46002963D04A4F0E
:109D300038680169C90736D105263046FFF7A6FE07
:109D4000304604F073FD03CF03690122134303611E
:109D5000002918D403200B4683438E481E588807D9
:109D6000C00EFF278740BE434027874037438948BE
:109D70001F501F20084082408748026087480260C9
:109D8000354800680FE08A07D20EFF2696400F2361
:109D90000B40083B03218B437D495F58B743402666
:109DA00096403E435E506901401801210902421865
:109DB000E369DB069B0CA569ED00EDB2EB1853607F
:109DC00062685207520B23685B075B099A18A36805
:109DD0005B079B0CD218E3685B075B0DD218236905
:109DE0005B01DBB2D21863699B07DB0ED2188023BC
:109DF00013434350002001B0F0BDC046F0B581B020
:109E0000002A23D005460835134C2668F668EE4034
:109E1000F50702D0022001B0F0BD069D8600A6190C
:109E2000B560400124682018009301231D024619E3
:109E300077680724A7437760F16032610099B160C9
:109E4000415919434151002001B0F0BD03A00AA1BE
:109E500074220DA305F02AF8D0920102696E636C9A
:109E60007564652F647269766572732F6D6B5F64BC
:109E70006D612E6300000000646D615F7472616E3D
:109E80007366657200000000496E76616C6964203B
:109E90007472616E736665722064737420616464A9
:109EA0007200000000015849085840687047C046D9
:109EB000F0B581B005460120012D4CD80C46002993
:109EC00049D0002D03D0012D04D10F2000E00E2039
:109ED000FFF7DCFDA668012E04D0002E4FD1E089EB
:109EE00000284CD12901294843580020D860F507A3
:109EF000AD0F27686668B607360F76192569EA0739
:109F0000920EB618022F04D0012F03D1012216435E
:109F100000E040361D4F9E60E2681A6079188D603F
:109F20006269CA604968002917D403220B4693432B
:109F3000184A9C588D07ED0EFF26AE40B44380268C
:109F4000AE4026439E501F220A4001219140124AF2
:109F50001160124A116001B0F0BD8A07D20EFF24D1
:109F600094400F230B40083B03218B4308495D5865
:109F7000A543802494402C435C5001B0F0BD08A060
:109F80000FA1492212A304F091FFC04618930102C9
:109F90001CED00E000E400E080E200E000E100E011
:109FA000696E636C7564652F647269766572732F70
:109FB0006D6B5F6475616C5F74696D65722E6300B3
:109FC0006475616C5F74696D65725F6F70656E005A
:109FD000636F6E66696720697320696E76616C696C
:109FE000640000000001084A105801608168802266
:109FF0000A4382607047C0460001034908588168DF
:10A00000802291438160704718930102F0B58DB0B2
:10A01000019315460E460A90129800240890048079
:10A02000149F3C8013980990046015980490048054
:10A03000FF2081053046F6F7E7F902903046039697
:10A040003146F6F788F92B463D4606902746079598
:10A050000B9311E011801888800028580999086036
:10A060000120079D28800520049908807F1CBCB230
:10A070001888844200D9A0E028880028F6D1A000E2
:10A080000A9D2E5830460699F6F7DAFB002817D0BD
:10A0900030460399F6F7D4FB00280B9B079DE5D1CA
:10A0A000089A1780099D2E601888011B012934D158
:10A0B0001080198889000A9A51582960059035E066
:10A0C000089A1780099806600B9B1988081B0128BD
:10A0D000C0D00C96019825187E1CB0B28542BFD323
:10A0E00089B2B2B28A420ED880000A990C58204632
:10A0F0000C99F6F797FB0B9B002804D10998046094
:10A10000089806800C94761CB0B28542A8D31988B2
:10A1100089B2B2B28A42E7D9F5E70C960199621882
:10A120007D1CA9B216468A4205972CD2059884B2A6
:10A13000A5000A9E7259002C104609D0A819001FCC
:10A14000016810460C92F6F706F90C9A062C07D80F
:10A150000446A81941681046F6F7FDF80C90204611
:10A16000079D0299F6F77AFB00280B9B07D10C9804
:10A170000299F6F765FB0B9B002800D076E70120DB
:10A180002880032070E780B2AAB282420FD88800EC
:10A190000A990C5820460C99F6F744FB0B9B0028B3
:10A1A00005D1099804600898058005950C946D1CEC
:10A1B000A9B28E42BAD31888E5E70DB0F0BD000011
:10A1C0000A490A680A4802400A60FD214900094A12
:10A1D0001268515C002908D007490A6C02400A64E1
:10A1E000012000060A6882430A60704700040040AC
:10A1F000FFFFFF7F409401022000004000207047D5
:10A20000F0B583B00D4604467C2646435048871976
:10A21000F869396AF5F75EFFA84200D892E0019527
:10A2200002940121EFF31080084002D1EFF3108275
:10A2300072B63C4610343B690025062B0CD80A4602
:10A240009A40D3065B0F06D161231A4275D00D46A2
:10A25000002803D003E00225002800D162B6002DBB
:10A2600002D0284603B0F0BD00943C462034384864
:10A2700080591021C1613E46143604F0E9FD0546BF
:10A280003868C069C00605D504F0E2FD401B31887E
:10A290008842F5D90621029D284600F00BFF206870
:10A2A00001994143B86909183868816017217956C6
:10A2B0003C461734002909D5C16920220A43C261EE
:10A2C0000121F966890502680A43026005212846D2
:10A2D00000F0F0FE207840B200250028C1D42B48C1
:10A2E00000687D24E100F5F7F5FE61014143029825
:10A2F00000F0B2FE04F0ACFD04463868C069C00747
:10A3000005D004F0A5FD001B31888842F5D904F082
:10A310009FFD04463868C169890706D504F098FD99
:10A32000001B31888842F5D938680121009A1160F4
:10A3300053498161284603B0F0BD03212160002804
:10A340008CD08CE7034804A1084A09A304F0AEFDB1
:10A3500044930102142F0100666C6173685F626CA4
:10A360006F636B5F65726173650000005D020000E2
:10A37000626C6F636B20696478206973206F766507
:10A38000722072616E67650D0A00000020E0010214
:10A39000F0B583B002907C214143934A5418E56E96
:10A3A000EAB2511E02291FD229040126090E18D033
:10A3B00001960092022100F07DFE2746143704F03A
:10A3C00047FD06462068C169890606D404F040FDB1
:10A3D000801B39888842F5D92068007DC007019E1E
:10A3E00008D0304603B0F0BD032A36D100922804CD
:10A3F000000E36D020466C302D0C002101910160FA
:10A400002746143704F024FD06462068C069C007BB
:10A4100005D004F01DFD801B39888842F5D904F071
:10A4200017FD06462068C169890706D504F010FDAE
:10A43000801B39888842F5D9206811498161E9B2C9
:10A440000120002911D003290099019E00D0062087
:10A450002061226F002A0ED1C3E70026304603B0E8
:10A46000F0BD0126304603B0F0BD0099019E206189
:10A47000226F002AB5D002A89047304603B0F0BD45
:10A48000000093EB70B5002801D0012070BD782545
:10A49000CD4E705D00280ED000240921204600F02A
:10A4A00009FE0F20FFF7CAFB1520FFF7E7FA7455E6
:10A4B0003461204670BD042070BDC046F0B581B047
:10A4C0000C460078484EF16881422CD1032C54D1BF
:10A4D000706EB16E884261D900240621204600F0DA
:10A4E000E9FD3068F16D81602046214600F0E2FD13
:10A4F000354660352CCDF0683168B48C414F0097FB
:10A500005B1BA34200D81C46A3081431FFF776FC5E
:10A51000B06E0019B066306E00193066F06D00192B
:10A52000F06501B0F0BDB168814255D1032C45D131
:10A53000F08CF16D0918F165316E09183166B16E54
:10A540000818B066716E814238D900240621204671
:10A5500000F0B0FD3068F16D81600121204600F00F
:10A56000A9FD316EB068F38C3268264C0094143229
:10A570009B08FFF743FC01B0F0BD30681021C161BA
:10A5800004F066FC05463068C069C00616D504F0C4
:10A590005FFC401BB18A8842F5D90FE0306810217A
:10A5A000C16104F055FC05463068C069C00605D598
:10A5B00004F04EFC401BB18A8842F5D90120C10746
:10A5C000326813688B431360F16E22040A43000261
:10A5D0001043F06601B0F0BD4D200201034804A114
:10A5E000844B04F063FCC04644930102142F010025
:10A5F000666C6173685F646D615F63616C6C6261FE
:10A60000636B0000BDA40000F0B581B000786E4D12
:10A61000AA68824200D0D0E001263002032942D14C
:10A620006A6DAA66AB6DAC6AA418EB652C66AB6C60
:10A630005B1CAB646B6E934235D95E30FFF7FEFA5C
:10A64000686CA96C02293AD3814238D1E88C696DD3
:10A65000081868650020062100F02CFD2868E96DC7
:10A6600081602F6D04F0F4FB04462868C069C007C0
:10A6700005D004F0EDFB001BA98A8842F5D904F04F
:10A68000E7FB04462A68D069800706D504F0E0FBA2
:10A69000001BA98A8842F5D92A687420285C012801
:10A6A00041D0F10440E0F2072B681C6894431C6021
:10A6B000EA6E090411430143E96601B0F0BD0229C5
:10A6C000FBD38142F9D2E88C696D09186965A96DDF
:10A6D0000818A8650020062100F0ECFC2868E96D48
:10A6E0008160EF8C04F0B4FB04462868C069C007A1
:10A6F00005D004F0ADFB001BA98A8842F5D904F00F
:10A70000A7FB04462A68D069800706D504F0A0FBA1
:10A71000001BA98A8842F5D92A687420285C012880
:10A7200022D0F10421E03105334B3B405918012878
:10A7300002D01920400601E00720C00608182F4962
:10A7400040185060002F0DD004F082FB04462A68A8
:10A75000D069800706D404F07BFB001BA98A8842DD
:10A76000F5D92A682B6D1FE03105234B3B40C918F2
:10A77000012802D01920400601E00720C006081871
:10A780001E4940185060002F0DD004F061FB0446B4
:10A790002A68D069800706D404F05AFB001BA98AF6
:10A7A0008842F5D92A68EB8C296EA868144C00946D
:10A7B0001432FFF723FB01B0F0BD044804A10C4A9A
:10A7C0000C4B04F073FBC04644930102142F0100AC
:10A7D000666C6173685F646D615F77726974655FF1
:10A7E0006E62797465735F63616C6C6261636B0048
:10A7F00072040000FB2E0100FF3F0000008080007B
:10A8000009A60000F0B587B004460126880E14D0D2
:10A810001546002A11D00F468120C004401B8842F3
:10A820000BD37C206043F04908180590818C384692
:10A830000691F5F74FFC002902D0304607B0F0BD75
:10A8400028460699F5F746FC0029F6D10598806957
:10A850003E1A30460699F5F73DFC074603967019F7
:10A860000190069E3146F5F735FC0546C01B049065
:10A870000598006A02903146F5F72CFC0499814254
:10A880000FD20026BD42D8D92046394600F018FB29
:10A890002046FFF77DFD0028FAD17F1CAF42F3D39D
:10A8A000CBE700900398029D2946F5F713FC064676
:10A8B000284670430399081A019800D0761C29464F
:10A8C000009D7543F5F706FC0590029941430198F8
:10A8D000401A03900699F5F7FDFB0490AF420BD2A6
:10A8E0002046394600F0ECFA2046FFF751FD0028DB
:10A8F000FAD17F1CAF42F3D305988642069D009F94
:10A900000CD220463146FFF77BFC2046FFF740FD86
:10A910000028FAD1761C05988642F2D30398A84203
:10A9200003D20026304607B0F0BD05984743002506
:10A93000E919204600F0C4FA2046FFF729FD002857
:10A94000FAD16D1C002604988542F1D375E7C04604
:10A95000F0B585B0002803D00124204605B0F0BD35
:10A960007822A14FB85C002803D00024204605B00F
:10A97000F0BD0492002905D0384614300CC90CC033
:10A980001CC91CC00020F86615242046FFF77EF87D
:10A99000204603F04BFF38681021C16104F058FADB
:10A9A00004463868C169C90607D504F051FA001B8E
:10A9B000B98A8842F5D9386800E0B98ABA7D1207A9
:10A9C000120B5218F97DCB07DB08D2188B07DB0F6F
:10A9D0005B05D218CB06DB0FDB05D2184B07DB0F6C
:10A9E000DB06D2188B06DB0F5B07D2180907C90FED
:10A9F00089071143016000240A21204600F05AFB18
:10AA00003220FFF71BF90821204600F053FB04F029
:10AA10001FFA05463868C169890606D404F018FA99
:10AA2000401BB98A8842F5D93868017D0A46C23A86
:10AA30005342534174257B550904027D120251187B
:10AA4000007D0B180220032668A2314605F08AFA21
:10AA5000785D0128039619D1F87D02900026062121
:10AA6000304600F027FB0721304600F023FB012190
:10AA700002988143785D012847D1386889010175C2
:10AA800006757521795C012938D048E00020032142
:10AA900000F010FB04F0DCF906463868C16989064D
:10AAA00006D404F0D5F9801BB98A8842F5D93868F4
:10AAB000007D46080122F87D014631431640C90752
:10AAC00001D0304036D0029500250621284601925B
:10AAD00000F0F0FA07210095284600F0EBFA019803
:10AAE00046400298385C012813D13868B1010175DD
:10AAF000009901757521795C012910D114307621F6
:10AB0000795C4A424A41510008E0386806754900BC
:10AB100003E03868009901757100143001703748FE
:10AB200000687D21C900F5F7D5FA282141430020AE
:10AB300000F092FA7720385C012803D1022000212E
:10AB4000FFF734F804F084F906463868C069C00796
:10AB500005D004F07DF9801BB98A8842F5D904F04C
:10AB600077F906463868C169890706D504F070F997
:10AB7000801BB98A8842F5D93868D049816117208D
:10AB80003856002829D57868002816D40146039A3B
:10AB900091431C4A8B588507ED0EFF26AE40B34308
:10ABA0008026AE401E438E501F2101400120884068
:10ABB00015490860154908600FE08107C90EFF229A
:10ABC0008A400F230340083B039883430C481D58D9
:10ABD000954380228A402A431A50012004997854D0
:10ABE0003861204605B0F0BD449301026A65646592
:10ABF000635F69642025780D0A00000020E00102EF
:10AC00001CED00E000E400E080E200E000E100E094
:10AC1000F0B593B07C270A9047439348C61998072C
:10AC200004D0F07D4024044000D017E10125880EB7
:10AC30002ED0002B2CD08120C004C01A884227D3EC
:10AC400009920122EFF31084144002D1EFF3108037
:10AC500072B63046103005903069002506280891FC
:10AC6000069310D8079414468440E106490F04D196
:10AC700061210C4203D0154604E0022502E00221C6
:10AC8000059B1960079C002C00D162B6002D02D0F4
:10AC9000284613B0F0BD344617347348C05910210C
:10ACA0000491C1613746143704F0D2F80546306884
:10ACB000C069C00605D504F0CBF8401B398888422E
:10ACC000F5D92078400665D40297B78C069C2046BB
:10ACD0003946F5F7FFF9079039464143601A03906A
:10ACE00035462435A74200D894E0039800281CD0AC
:10ACF00006210A9C204600F0DDF928880799484380
:10AD0000089940183168886000272046039C39461E
:10AD100000F0D0F9079B099A28885843C019316878
:10AD2000097D11547F1CA742F6D330680499C16194
:10AD300004F08EF80446029D3068C069C00605D54F
:10AD400004F086F8001B29888842F5D904F080F8C1
:10AD500004463068C069C00705D004F079F8001BCC
:10AD600029888842F5D904F073F804463068C1692F
:10AD7000890706D504F06CF8001B29888842F5D9AC
:10AD800030680121059A1160B24981610025284689
:10AD900013B0F0BD03200025089FF76509993166BF
:10ADA00006997166B566F0660120C00731680A68C9
:10ADB00002430A6006210A9C204600F07BF93068B5
:10ADC00087602046294600F075F93A4F0BAA0A928F
:10ADD0001BCF1BC21BCF1BC2B48CF0680A99FEF7B5
:10ADE0009DFFF0683168344A0092069A944200D37D
:10ADF0001446A3081431099AFFF700F8B06E001941
:10AE0000B066306E00193066F06D0019F0652846A6
:10AE100013B0F0BD002404E0641C0798844200D302
:10AE200063E706210A9800F045F9288860430899ED
:10AE300040183168886000270A98394600F03AF9CE
:10AE400028880028099AE7D0604310183168097DE6
:10AE5000C1557F1C28888742F6D3DDE7034804A14B
:10AE6000064A07A304F022F844930102142F0100BC
:10AE7000666C6173685F726561640000C603000000
:10AE800054686520444D412072656164206C656E94
:10AE90006774682073686F756C64206265207468DD
:10AEA00065206D756C7469706C65206F6620340D5B
:10AEB0000A00000088230100BDA40000000093EBFD
:10AEC000F0B583B00D4604467C26464351488719A9
:10AED000F869B98CF5F7FEF8A84200D894E001951E
:10AEE00002940121EFF31080084002D1EFF31082A9
:10AEF00072B63C4610343B690025062B0CD80A4636
:10AF00009A40D3065B0F06D161231A4277D00D46D3
:10AF1000002803D003E00225002800D162B6002DEE
:10AF200002D0284603B0F0BD00943C462434394892
:10AF300080591021C1613E46143603F089FF054651
:10AF40003868C069C00605D503F082FF401B318810
:10AF50008842F5D90621029D284600F0ABF82088EA
:10AF600001994143B86909183868816017217956F9
:10AF70003C461734002909D5C16920220A43C26121
:10AF80000121F966890502680A4302600421284606
:10AF900000F090F8207840B22C4600250028C0D45C
:10AFA0002B4800687D21C900F5F794F820492D3120
:10AFB0004143204600F050F803F04AFF0446386849
:10AFC000C069C00705D003F043FF001B31888842E9
:10AFD000F5D903F03DFF04463868C169890706D5F5
:10AFE00003F036FF001B31888842F5D9386801210B
:10AFF000009A116017498161284603B0F0BD032112
:10B00000216000288AD08AE7034804A1084A09A3DE
:10B0100003F04CFF44930102142F0100666C61732E
:10B02000685F736563746F725F657261736500005A
:10B030002B020000736563746F7220696478206965
:10B0400073206F7665722072616E67650D0A00006D
:10B0500020E00102000093EBF0B583B001917C2267
:10B060000290424353498C182546143503F0F0FEF4
:10B0700006460221029800F01DF803F0E9FE07469B
:10B080002068C169890606D403F0E2FEC01B298846
:10B090008842F5D92068007DC00708D06420FEF7FB
:10B0A000CDFD03F0D5FE801B01998842E1D903B0A4
:10B0B000F0BDC046F0B585B0049104467C206043E5
:10B0C0003C490F183D46143503F0C2FE0646386869
:10B0D000C069C00705D003F0BBFE801B29888842E9
:10B0E000F5D903F0B5FE06463868C069800705D576
:10B0F00003F0AEFE801B29888842F5D91421049BF9
:10B100005943DC2060432C4A1018039002914018E8
:10B11000018A8268C47C7426BE5D012E0DD1019126
:10B12000012B02990CD0012B0DD07526BE5D012E8E
:10B130000ED0019E072B0ED10EE00E4602990BE0B9
:10B140000222012BF1D138247526BE5D012EF0D1EB
:10B150000326072B00D0019E184B3340240692078C
:10B16000D20A1219D218039B5958C907490C521810
:10B170004168CB071B0CD218837C5B075B0BD21892
:10B18000C0684007000A10183A685060002E0ED0C0
:10B1900001290CD103F05CFE04463868C0698007C1
:10B1A00005D403F055FE001B29888842F5D905B067
:10B1B000F0BDC04644930102D0240100FF3F0000CF
:10B1C000F0B59DB00D460126890E2FD0002B2DD055
:10B1D00011928121C9041093C91AA94226D30121D1
:10B1E000EFF310840C4002D1EFF3108272B67C2290
:10B1F0000F904243E74814928718384610303B6955
:10B200000026062B0DD80A469A40D3065B0F07D1BD
:10B2100061231A4200D16FE30E46002C03D003E0F5
:10B220000226002C00D162B6002E02D030461DB09E
:10B23000F0BD0290BD650021139179651098401E04
:10B2400012904019B964B9690D916E1A1199B962D9
:10B25000FD6238637E63F98C0E913046F4F73AFF55
:10B260000446B863129830180E9E3146F4F732FF48
:10B27000109B011B4A1CF86339647A64139A0029F5
:10B28000194608D0704359190D9BC91A0A1A7443FC
:10B29000581B80190119384648300E903846443002
:10B2A0000D90384640300B90384626300590384691
:10B2B00058301390384654301290F9643A65149817
:10B2C000B44908581021C1613846143014903846EA
:10B2D000503004903D464C3503F0BAFD04463868C2
:10B2E000C069C00606D503F0B3FD001B1499098898
:10B2F0008842F4D9F87D40060C9500D574E201230C
:10B300000E9803600D98016800290F9800D1CDE2D6
:10B310003A4674320A92DA0407921A0509921922FF
:10B32000520606920722D206089216E09A48006852
:10B330007D21C900F4F7CEFE109941430F9C2046B1
:10B34000FFF78AFE20460C9D0E9A11684B1C136075
:10B350000D9909688B4200D9A8E20B9A1268012A5C
:10B3600055D0002A00D0A8E02E6812990C681399D5
:10B370000D6806211091FFF79DFE386885601198D1
:10B38000051903F065FD04463868C069C00706D09A
:10B3900003F05EFD001B149909888842F4D903F07C
:10B3A00057FD04463868C169890707D503F050FD89
:10B3B000001B149909888842F4D938680A990A78D8
:10B3C000012A089900D00699012A099A00D0079A03
:10B3D0003346724C234013430B4371490B43436084
:10B3E000002EA3D003F034FD04463868C0698007FE
:10B3F00006D403F02DFD001B149909888842F4D966
:10B400003868297801756D1C761EFAD18EE7012BFC
:10B4100000D0C7E02E6812990C6813990D680621B8
:10B420001091FFF747FE386885601198051903F001
:10B430000FFD04463868C069C00706D003F008FD58
:10B44000001B149909888842F4D903F001FD0446D1
:10B450003868C169890707D503F0FAFC001B149905
:10B4600009888842F4D938680A990A78012A089923
:10B4700000D00699012A099A00D0079A3346474C12
:10B48000234013430B4346490B434360002E69D0CE
:10B4900003F0DEFC04463868C069800706D403F078
:10B4A000D7FC001B149909888842F4D93868297898
:10B4B00001756D1C761EFAD154E0012B00D0C9E055
:10B4C0002E6812990C6813990D6806211091FFF7E8
:10B4D000F1FD386885601198051903F0B9FC044640
:10B4E0003868C069C00706D003F0B2FC001B14998D
:10B4F00009888842F4D903F0ABFC04463868C16976
:10B50000890707D503F0A4FC001B14990988884219
:10B51000F4D938680A990A78012A089900D006995E
:10B52000012A099A00D0079A33461C4C2340134342
:10B530000B431B490B434360002E13D003F088FCE0
:10B5400004463868C069800706D403F081FC001BFC
:10B55000149909888842F4D93868297801756D1CD6
:10B56000761EFAD10C4800687D21C900F4F7B2FDBF
:10B57000109941430F9C2046FFF76EFD20460C9D1D
:10B580002A68139B196889181960129B1968891811
:10B590001960D9E64493010220E00102FF3F000058
:10B5A000008080008B4200D0CEE604990E6812998C
:10B5B0000C6813990D6806211091FFF77BFD386820
:10B5C00085601198051903F043FC04463868C0698A
:10B5D000C00706D003F03CFC001B14990988884280
:10B5E000F4D903F035FC04463868C169890707D5EA
:10B5F00003F02EFC001B149909888842F4D938689E
:10B600000A990A78012A089900D00699012A099A0C
:10B6100000D0079A3346D44C234013430B43D349FD
:10B620000B434360002E00D180E603F011FC04467A
:10B630003868C069800706D403F00AFC001B14991F
:10B6400009888842F4D93868297801756D1C761EFE
:10B65000FAD16BE6129A1268119CA618139A156813
:10B660008B425FD104990C6806210391FFF722FDFC
:10B670003868856003F0ECFB05463868C069C00790
:10B6800006D003F0E5FB401B149909888842F4D9E1
:10B6900003F0DEFB10900C9D3868C169890708D55E
:10B6A00003F0D6FB1099401A149909888842F3D9FF
:10B6B00038680A990A78012A089900D006991091E9
:10B6C000012A099A00D0079A2346A7490B40134341
:10B6D00010990B43A5490B434360002C14D003F091
:10B6E000B7FB10903868C069800707D403F0B0FB3F
:10B6F0001099401A149909888842F3D9386831782A
:10B700000175761C641EFAD19A4800687D21C90033
:10B71000F4F7E0FC039941430F9C2046FFF79CFCA3
:10B72000204611E605990C8806210391FFF7C2FC1B
:10B730003868856003F08CFB05463868C069C0072F
:10B7400006D003F085FB401B149909888842F4D980
:10B7500003F07EFB10900C9D3868C169890708D5FD
:10B7600003F076FB1099401A149909888842F3D99E
:10B7700038680A990A78012A089900D00699109128
:10B78000012A099A00D0079A234677490B401343B0
:10B7900010990B4375490B434360002C14D003F000
:10B7A00057FB10903868C069800707D403F050FB3E
:10B7B0001099401A149909888842F3D93868317869
:10B7C0000175761C641EFAD16A4800687D21C900A3
:10B7D000F4F780FC039941430F9C2046FFF73CFCA3
:10B7E000204605990A88CCE65E4815A90A4678C81D
:10B7F00078C278C878C20125E8073A68136803431D
:10B800001360B868FEF78AFA02200026139C2168AC
:10B81000BA6AF9653A6610997966BE66F8660C9858
:10B820000068129A1168091811600E9B19684A1C69
:10B830001A60226810182060002900D0F6E41095E4
:10B840003846603013903C465C34384608301290DD
:10B8500006210F98FFF72EFC3868216881600C984C
:10B860000068119003F0F4FA04463868C069C00714
:10B8700006D003F0EDFA001B149909888842F4D928
:10B8800003F0E6FA0446109D3A68D069800707D5B0
:10B8900003F0DEFA001B149909888842F4D93A684B
:10B8A0007420385C01282DD0E9042CE003F0D0FA94
:10B8B00004463868C069C00706D003F0C9FA001B07
:10B8C000149909888842F4D903F0C2FA044638680A
:10B8D000C169890707D503F0BBFA001B14990988D1
:10B8E0008842F4D938680121029A116022498161A5
:10B8F000002630461DB0F0BD04210160002C00D1AF
:10B9000091E491E42905119C174B23405918012813
:10B910000C9D02D01920400601E00720C00608183F
:10B92000124940185060002C0ED003F091FA0446E2
:10B930003A68D069800707D403F08AFA001B14998B
:10B9400009888842F4D93A682B68139801681298DC
:10B950000068074C00941432FEF750FA30461DB0D0
:10B96000F0BDC04648230100FF3F0000008080007A
:10B9700009A6000020E00102000093EB3920C0007E
:10B980000149096808587047D0920102F0B50329AF
:10B9900020D8C0467944097949008F4401080F1521
:10B9A000012181404F4B1B685963D96212E001218C
:10B9B00081404C4B1B681963D9620BE00121814027
:10B9C000484B1B68596304E001218140454B1B68CB
:10B9D0001963996283004349CB18DA608A68002AA8
:10B9E00029D14A68002A16D4032314469C43174BD6
:10B9F000E5589607F60EFF27B740BD438027B740AE
:10BA00002F43E7501F23134001229A40104B1A6026
:10BA1000104B1A600FE09307DB0EFF259D400F24AB
:10BA20001440083C03229443074AA658AE4380259D
:10BA30009D403543A5500122824008680262886813
:10BA400010438860F0BDC0461CED00E000E400E05B
:10BA500080E200E000E100E010B501242046FEF79E
:10BA600015F8204602F0E2FE002010BD01218140C1
:10BA70001C48006842688A43426070471949096857
:10BA80000968C140012008407047C046012181403B
:10BA90001448006842680A4342607047012907D091
:10BAA000002910D1012181400F4802680A430FE0AC
:10BAB000012181400B4800684368002A0DD00B43E8
:10BAC00043600161704701218140074802688A4351
:10BAD000026004480068416170478B434360016124
:10BAE0007047C046D49301020801004080B5114A56
:10BAF0001170114A10708001C90101430F4800788C
:10BB0000400108430E490978090101430D480078B6
:10BB1000C00008430C490978890001430B480078AC
:10BB2000400008430A4909780143C8B2F8F7F4FD18
:10BB300080BDC046109F0102DE96010229940102D9
:10BB400094EA0102C9AD0102119F010254A301024E
:10BB500055A30102012282400548002903D0016853
:10BB60001143016070470168914301607047C0460E
:10BB700000010040124A072809D880000F238340A3
:10BB800081401940106898430843106070470F289F
:10BB90000AD8800020380F23834081401940506824
:10BBA0009843084350607047800040380F2383401B
:10BBB0008140194090689843084390607047C046A0
:10BBC00034000040F0B54307DC0E0726A640C3084A
:10BBD0009D000E4BEF187D68B5433E1D002908D02F
:10BBE00035600122824001290CD118681043186089
:10BBF000F0BD01218140186888431860A2401543B8
:10BC00003560F0BD186890431860F0BD0C0100402D
:10BC100010B582B014460A4601460498009301907C
:10BC20000820234600F092F802B010BDB0B584B0F1
:10BC300014460A4601460898022500950193029091
:10BC40000720234600F052F904B0B0BD70B50028BB
:10BC50005BD031490A783149002A03D14A6801236F
:10BC600013434B60428803881B049A180B46183B09
:10BC70001A60828883891B049B180C460C3C236045
:10BC80000B46083B84681C60446903232340057C01
:10BC9000AD00EB188569AD072D0D5B19457C2D03B3
:10BCA0005B19C569AE07B60A9B19867CB6059B1958
:10BCB0000E1F3360036A122B04D107240C60541E3C
:10BCC000A2410AE0032C05D1012D03D807220A6006
:10BCD000012202E006220A600122114C0025257093
:10BCE0000F2464012034C57C6D0225401B069B0B8C
:10BCF000D218C3791B07DB0ED21880790007C00D5C
:10BD0000101840191439086070BD064806A1862233
:10BD100009A303F0CBF8C0460CCD01021810005067
:10BD20000ECD0102F13B01006C73705F656E6769B7
:10BD30006E655F72756E0000506172616D6574654D
:10BD400072206973206E756C6C000000F0B58BB0CA
:10BD5000109E34043ED00D46D64C21400127019759
:10BD60007F06B9423CD111462140B9423FD11C4027
:10BD7000BC4243D1119902AC0027E781E78066807D
:10BD800027802782A774E1749908A181A908A1805E
:10BD90000A90099708970797900880B20490204668
:10BDA000FFF754FFAA480078002801D00BB0F0BD7F
:10BDB000AB480168C90708D10168C90705D1016806
:10BDC000C90702D10168C907F3D07F480199017002
:10BDD0000BB0F0BDB8480D49AF22C14B03F066F877
:10BDE0000095B5480949B022754B03F05FF8009201
:10BDF000B1480649B122724B03F058F80093AE489F
:10BE00000249B2226E4B03F051F8C046C73B010015
:10BE1000F0B58DB00392139E340446D00A46A54C6B
:10BE20002140012502956F06B94244D10399214072
:10BE3000B94247D11C40BC424CD11499129D04AC6C
:10BE4000E174294921820027E781E7806680278005
:10BE50009908A1819108A1800B95012D01D1612143
:10BE6000CF43A7740C9002200A9009900398800891
:10BE700080B206902046FFF7E9FE7548007800285A
:10BE800001D00DB0F0BD76480168C90708D101683E
:10BE9000C90705D10168C90702D10168C907F3D0F4
:10BEA0004948029901700DB0F0BD83480D49FB224D
:10BEB0008B4B02F0FBFF00927F480A49FC22404B6B
:10BEC00002F0F4FF039800907B480649FD223C4BAA
:10BED00002F0ECFF009378480249FE22384B02F052
:10BEE000E5FFC046D43B01008E8E0000F0B58BB05C
:10BEF000119E340447D00D466E4C21400127019716
:10BF00007F06B94245D111462140B94248D11C4073
:10BF1000BC424CD11299109F02ACE1742949218294
:10BF20000021E181E180668021809908A181A90832
:10BF3000A1800997012F01D0712100E06121C9433F
:10BF4000A1740A90032008900790900880B2049092
:10BF50002046FFF77BFE3E480078002801D00BB05A
:10BF6000F0BD3F480168C90708D10168C90705D17C
:10BF70000168C90702D10168C907F3D012480199C5
:10BF800001700BB0F0BD4C480C49D522544B02F067
:10BF90008DFF009548480949D622094B02F086FFDB
:10BFA000009245480549D722054B02F07FFF0093D8
:10BFB00041480249D822024B02F078FFE33B0100DE
:10BFC000113C0100868600000ECD010210B582B042
:10BFD00014460A460146002000930190042023469F
:10BFE000FFF7B4FE02B010BD10B584B014460A4687
:10BFF0000146002000900193029004202346FFF7A1
:10C0000007FF04B010BD000070B50D4606460424BD
:10C010002046FDF73BFD204602F008FC0B4805607A
:10C020000B480670002E0ED00A48016880220A4391
:10C030007F218A4302600120000307490860074905
:10C04000086007480460002070BDC04610CD0102A2
:10C050000CCD01020CE400E080E200E000E100E031
:10C060001C100050B0B582B0144602461148204062
:10C0700001256D06A8420DD1180413D017480160A0
:10C08000002000930190062011462346FFF75EFE34
:10C0900002B0B0BD0094FF228C320748074908A3C4
:10C0A00002F004FFFF208C30421C034803490C4B74
:10C0B00002F0FCFE0300FCFFF13B0100B93B010074
:10C0C00044737420616464726573732025782069F9
:10C0D0007320696E76616C6964000000081000507E
:10C0E0002F3C010080B582B00B4601460020009233
:10C0F000019003200A46FFF729FE02B080BD000030
:10C10000002801D0042100E00221C24A5172411EE0
:10C110008841800103490A6840239A431018086047
:10C120007047C04650A00050F0B583B002912E4930
:10C13000CD7A0E7B771987424FD90899019118253E
:10C1400045434126F604BF00BE19745B34490C40D8
:10C1500057033C199B07D90C6418324B1B681B7A98
:10C16000745375196C880326B60326409B079B0CF5
:10C170009B193F2404401819029CA3061B0DC018EC
:10C180006880012A184E13D8707B14224243307BFA
:10C190005023434324011B199A18F37AC0181C2317
:10C1A0004343D01880081E4A104007430F432F8096
:10C1B0000198686001F0BEFEA860E8681A4908406E
:10C1C0003030E860286908402721715C40182861F8
:10C1D00000F03EFE686103B0F0BDFF2288320348E4
:10C1E00003A108A302F062FE14D20102803C010008
:10C1F0006D61635F63735F636F6E73747275637495
:10C2000000000000435320696E6465782069732044
:10C210006F7665722072616E67650D0A000000001E
:10C22000FF070000409401020000F0FFF0B581B06C
:10C23000009314460D46074606263046FDF726FCB9
:10C24000304602F0F3FA26211D48475400210170C0
:10C2500041708171017181704171C170C17102229F
:10C260004272C16201634163816304734273C572A8
:10C27000009A561C134A168001724120C004012105
:10C280004903F3F790FF5020604329010818611912
:10C290008A00801818224A438018B2B24A43801894
:10C2A000094940180949884204D200F0B5F8002035
:10C2B00001B0F0BD064807A19A2209A302F0F6FDDD
:10C2C00014D2010210D20102280008020120080243
:10C2D000803C01006D61635F696E6974000000005D
:10C2E000454D206F766572666C6F770D0A00000011
:10C2F000A448C179002901D001207047007A411E6D
:10C3000088417047F0B583B002912A494B7B834244
:10C3100048D9CB7A0C7BE31818245C439B00E318C4
:10C320004124E4041A1914240190054665430026AB
:10C33000565100925519EE882E4F0B467A1C32400A
:10C34000F54E3688497A711A2B4E0E40B618EE809B
:10C350003740997BEF80AA88284F17404A424A41CC
:10C3600091007918264A8918A980264F0F402D1D63
:10C37000029801280AD124490E400921C9027118E6
:10C3800069800121C9037918298000E02F80019874
:10C39000444300980019074A918C4182118C018214
:10C3A00003B0F0BD3520C200034804A109A302F088
:10C3B0007DFDC04614D20102803C01006D61635FC7
:10C3C0006C696E6B5F646573635F636F6E737472C9
:10C3D000756374004C696E6B206465736320696ECD
:10C3E000646578206973206F7665722072616E676C
:10C3F000650D0A00FFFBFFFFFF03000003D0FFFFF6
:10C40000E80F0000EF1F0000FF830000BE4A5063EA
:10C410009163704714D20102F0B581B04348CC213A
:10C42000016003214160B8490A7BD304404C1B19C9
:10C43000CC7AA218541E1C431823534392009A1816
:10C440004B7B14255D43521992012243012463065C
:10C450001343436100228262C262026342638263C9
:10C46000C26342650267334B1A605A609A60324B6E
:10C470001A601A619A61DC61304C1C62304C251DD7
:10C480001D6325460C3D5D632546283D9D632D4E6D
:10C49000DE631C645C642C4D2F461C379F6427466A
:10C4A000143FDF64103C1C65284C5C65284C9C657F
:10C4B0000C369E67274CA5634035E563DA651A663E
:10C4C0005A669A66DA661A67234DDD67022585612A
:10C4D000224DC561C325AD03CD620A63D2435A60C4
:10C4E0001F4A1368FF25AB4326254D5DAD072D0E72
:10C4F000EB1813601B4A102313601B4A136027229A
:10C5000060238B5419498160C160016121607D21E4
:10C510000901016641661649C1641649416416491C
:10C52000016400F085FC01B0F0BDC04604A00050DD
:10C530000000F8FF94A0005034A10050FF185A00EA
:10C5400030040040041000401C20004054300040E3
:10C5500060400040B8A1005014001400FF3F3FFFAE
:10C5600004E400E080E200E000E100E0DC05DC053E
:10C570003F0270020133D007D007D0072921C64AF5
:10C580005054704714D20102F0B58BB00792089155
:10C590000146C14FB8780991FFF7B4FE78793A7B2C
:10C5A00079790691824200D89FE0FB7A9A18182385
:10C5B000534392004124E10404915218D2187B7B2A
:10C5C00014214B43D21850246043155801230A9379
:10C5D000DB022E469E4316504E4B2B4005937D7B2F
:10C5E00003914D433E7B7443F97A0B011B195B1990
:10C5F00071181C24029461435918A84B1B88069C8F
:10C600005C430919C904490D059BC918115010183C
:10C610000799416038787979089A00920322099B3A
:10C62000FFF782FDF87A397B09183878814263D99F
:10C6300083000993049AD45C0894F7212140D154D3
:10C64000D1184D788E7836027619CB781B04F31802
:10C6500007900A9886051E43330CCB70FB7A387B13
:10C66000BC784D709F4D3540039E6643C018029BB9
:10C670004343981940029C4B03405C19200A887080
:10C68000200CC870F023089D2B401B1D3D7B089596
:10C69000FE7A099D5355C8700620079A50438019A9
:10C6A000089A801848701F22D20222400243100AC2
:10C6B00088707879401C7871387B7979814201D310
:10C6C000002179713978491C3970F97A081839785C
:10C6D000884201D80020387028200A993954387AC5
:10C6E000401C3872387A0BB0F0BDA7204200D24807
:10C6F0000649074B02F0DAFBA72042007A32CE4807
:10C700007349744B02F0D2FB14D20102A03C010029
:10C71000493C010000F0FFFF10D201020320000697
:10C7200005490A6882430A600A6802430A600348AE
:10C73000012101607047C0461C0000401CA0005051
:10C7400080B50120FDF758FC80BD0000F0B587B032
:10C7500006930646504C607A504B1B88181A0C9D65
:10C76000A84200DC89E00F460592012E06D156480A
:10C770000021C1620169554A89180160A0783146DB
:10C78000FFF7C0FDE078E178069A2B4600F0AEF89E
:10C790002078E1780097002206923346FFF7C4FC28
:10C7A000E07A217B0818217888426ED94120C204A2
:10C7B00004918800815C0391F7250D400292855415
:10C7C0004549455C4549465C360276194449475C13
:10C7D0003F04F6190127BF0537433E0C4654E67A5D
:10C7E000217BA3783C4A85543E4D3D4014275F434E
:10C7F00089191C234B43D91949023B4B0B405D1946
:10C80000290A364BC1542E0C35494654F02703995A
:10C810000F400599002900D13F1D217BE37A029A40
:10C8200087542F4A86540622049E7243D218511808
:10C83000294A81541F22D20215400D43290A274A52
:10C840008154E078401CE070E07AE178814201D3C5
:10C850000699E1702178491C2170217B0818217804
:10C86000884201D806982070E079401CE071A07AD7
:10C87000401CA072E07907B0F0BD3920C20016322A
:10C88000074808A109A302F011FB3920C20004489F
:10C890000F49104B02F00AFB14D2010210D2010220
:10C8A000803C01006D61635F747800004D4143205E
:10C8B0005458206C656E206973206F766572207203
:10C8C000616E67650D0A00000804004090D0030007
:10C8D000B63C0100673C01000100080202000802AA
:10C8E00003000802FF07C0FF00F83F00F0B589B061
:10C8F0000893019204914F4DEF7A874200D891E05E
:10C90000297B502632464A434124E3040693D21839
:10C91000CC19A10051181822059254430A19697BB9
:10C9200014230793594353180290000119580446E1
:10C930000390504A0A40A97AC90251180898820502
:10C94000D2088A181A514C4911402A7B0096564346
:10C95000384CE57A2C0106982418A719354E54193D
:10C96000A5007D19059844432819747B079D6C43E5
:10C970000519049FD2194148048854432A19089C78
:10C98000D204520D51181D460398195000F06AFA4E
:10C990000146707A001902043E460CD080B2C000F5
:10C9A000002900D1801E029FA5214900F3F792FBC8
:10C9B0001F21014001E00021029F3801281842791F
:10C9C00083791B029A18C3791B04D2182C4B13408D
:10C9D000437109045918090CC171002C20D0154865
:10C9E00035460646007B009B4343F17A0A01069FC9
:10C9F0003A43D21841188B00D218059B4B43D118EB
:10CA0000727B079B5343C91840191C4A1288424342
:10CA100088180199884203D001992246F3F7AAFBAE
:10CA200009B0F0BDFF225C32034804A109A302F063
:10CA30003DFAC04614D20102803C01006D61635F83
:10CA400074785F646573635F636F6E73747275632C
:10CA5000740000005458204445534320696E6465B7
:10CA600078206973206F7665722072616E67650D3C
:10CA70000A000000FF0700E000F8FFFF10D20102EB
:10CA8000EFFFE00082B0FCF7EDFD05200025294610
:10CA9000FFF770F806202946FFF76CF80A202946B0
:10CAA000FFF768F809202946FFF764F801242046BB
:10CAB00003F0DEFB284603F0DBFBFCF70FFE20460D
:10CAC000FCF702FE01F032FE01F02AFE6D4801681B
:10CAD0006D480068890308D403210907084021072D
:10CAE000884202D0FCF78CFD06E0FCF7F1F8FCF779
:10CAF0009FFD0020FDF7C6FCFCF72AFE0025284616
:10CB000004F0D4FC032661A23046314603F02AFA31
:10CB100030462946FBF782FBF7F7FCFEFAF7BEFD2D
:10CB2000FEF79AFF5F4F381DFCF796FBF7F7EAFB1D
:10CB3000F6F722FBF7F77BFE042630462946FFF77F
:10CB400019F8304621462A46FEF7A8FF052230464E
:10CB50002146FFF737F828462146FEF7C7FF674E04
:10CB600030462830504A01902146FCF7E7FAFAF7A0
:10CB7000BDF8A2024D494E4B204603F077FE01F06E
:10CB8000B3FBF6F7E7FA4B4A2046214602F0A4F839
:10CB9000494802F0D1F84948FCF71CFD7878002894
:10CBA0000DD104E0FBF77AF97878002807D1F7F780
:10CBB000A9FE002803D1F079002815D13CE0FCF74C
:10CBC00053FCB079002802D0B571F6F731F9F7F7C8
:10CBD000ADFEF6F7BFFEF7F7EFF8FAF76DFDFCF7DD
:10CBE00021FCF079002827D0F571B078411CB17094
:10CBF0003D2806D30020B070012101982A4AFCF795
:10CC00009DFAFAF707FF2E480470F7F77BFE00281D
:10CC100002D07D70F57007E0F0781E28214600D321
:10CC200029467970401CF070F7F702F97F20C105A2
:10CC3000F069F3F790FBF0610B20FEF71FFF3978E6
:10CC4000002810D00029ADD101201E49087038708D
:10CC500000201D49087003F0E5FAFBF71FF978780A
:10CC60000028ACD1A3E701299CD10020387050499D
:10CC7000C8831449087001201349087003F0AEFA04
:10CC800090E7C04618000040300001405557422050
:10CC900073696D706C65206578616D706C650D0AE7
:10CCA000000000001C9001023190000010CE010233
:10CCB000A50A010089EC00007C3F0000F5CC0000D3
:10CCC000DE960102189001021990010201480068E5
:10CCD0007047C0460C00004081B080B581B003931E
:10CCE00003AB009302F0B8FD01B080BC02BC01B000
:10CCF0000847000001480021C1617047B098010257
:10CD0000F0B581B0002630463146FDF721FE012501
:10CD1000AC022649264F30463A462346FDF778FFB7
:10CD20003988244881423FD064217E5262217E525C
:10CD300060217E524422BE52FD87BD8778227A87C9
:10CD400002223A874322FA86BE83FE811A4ABA81BA
:10CD50007E810A223A81194ABA803880FE830620F1
:10CD60003885F984FF20123078840146E331F98058
:10CD70008730B88450203E523A83EFF3108072B669
:10CD800030463146FDF7E4FD00280CD12A03002689
:10CD90003046064D2946FDF735FD054A3046294601
:10CDA0002346FEF70DFA62B601B0F0BD00E00204C2
:10CDB00062A90102AA550000E1FF00003412000040
:10CDC0000020704710B50024002809D0002905D0A4
:10CDD00003464A0003481946F3F7CCF9204610BD34
:10CDE000E04310BD38930102014600200A2901DA10
:10CDF000C0437047014A11807047C046C09301028A
:10CE00000020704780B50188064A11808178064A63
:10CE10001170C178054A11700079FCF749FB0020B8
:10CE200080BDC0462A9401022C940102C4D20102A2
:10CE300004480549016015210904416003498160E6
:10CE40007047C0469C300040410008003400070095
:10CE50000748006840697047FD20400004490968A0
:10CE6000085C7047024800686221405C7047C04619
:10CE70004094010210B50648046806480068642121
:10CE8000F3F73EF90221C9434143081910BDC046DA
:10CE9000C8D20102CCD201020A491A220A600A4908
:10CEA00048704878FF210902084A13688B438003C1
:10CEB00080B2C0181060064820210160054801605A
:10CEC00000207047702000403094010204E400E02C
:10CED00080E200E000E100E0F0B5A9B016460F46A0
:10CEE0000546C648002B024600D01A463921CC0020
:10CEF0003D21C900511811918242189206D001209B
:10CF00004202BE491898F3F735F9189A61201119B1
:10CF100013910E21119C0A91A170002F0D9501D043
:10CF20000A2100E00921592317938300E170784218
:10CF3000784113990870307810901070F17AE1748C
:10CF400071785170B7789770F178D1703579157123
:10CF500074795471B1799171F179D171317A117219
:10CF6000717A5172B17A91727E1EF0B2002103285B
:10CF7000169106D870B28000A1A210586A00805A9B
:10CF80001690179882001898C0181490F81E02285E
:10CF900004D3012E084604D89D4800E09D4803199B
:10CFA00018781290189DA8181790284630301590C0
:10CFB0002C4656346D2080002950974A974B149E7A
:10CFC00033627262B362F2623176F182139B5970FE
:10CFD00009229A70281841608160C160016110982F
:10CFE00080008F490858F3F753FD012F10900F91DF
:10CFF00004D0022F05D17F217E2004E07C217B20FC
:10D0000001E05B215A20159DA984207003200C901B
:10D01000A080012666701F200B90A8821820A8749B
:10D020000A46083A179BDA76169B129AD2184A4398
:10D030009100189A9163B702791E8B420E9109D91B
:10D04000784860803420688477482882774813992C
:10D05000088339E07F2B10DD802B18D031028B4202
:10D060001BD071028B4227D16E49618068846F4862
:10D0700013990883CF20C00025E0202B17D0402B28
:10D080001AD1684860800420688469481BE06548BC
:10D09000608006206884674815E062486080102040
:10D0A0006884624813990883C520C0000BE0624879
:10D0B00060800220688404E00420688481204000AD
:10D0C0006080FF2002302882104600F0D7FE1298C0
:10D0D000102806D0402808D108201499C8760720C7
:10D0E00000E004201799887002E017980C9981706D
:10D0F0001898169A8078C11E02290CD3022811D0E4
:10D1000001280CD12672BA4200D900266672BA42B2
:10D1100013D8F44812E00D20000211990880012074
:10D12000800201E00C9800022081BA4201D8EE484A
:10D1300000E0FA20179988600EE0FA2017998860BD
:10D14000139800780028119901D0E8484880E848F1
:10D15000139A1083E7480880A88CF3F7FBFB00269E
:10D16000E54B3246F3F77EFA02460B46E34930467A
:10D17000F3F7E0FAE24B3246F3F774FAF3F73CFCCC
:10D180000746E080DF493046109A0F9BF3F7D2FA4A
:10D19000DD4B3246F3F766FAF3F72EFC7843404254
:10D1A000800B608116990E98814208D90C20149F3B
:10D1B000B872D648179988831220189A0EE0480A48
:10D1C000189A149F01D00D2003E0080A00D1DBE279
:10D1D0000A98B872CE48179988831220F872D078CE
:10D1E000052844D878440079400087440227402C21
:10D1F0003339C848B881C8482FE0C046D0900102F2
:10D20000F8220100F8220100082301000823010090
:10D21000E81F0100EF1F010030750000102700001B
:10D22000A820010005020000FF060000040800001D
:10D230000A0400003604000003020000B748F88129
:10D24000B748388013E0B748F881B7483882B74804
:10D2500038600CE0B448B881B5481799C88306E037
:10D26000B4487882B448B8800B9800069064AE4801
:10D270003881A748F880B14802882A84B0480078ED
:10D28000E874B0480078119F7875387D13900028B5
:10D290005ED0AD490A681023DA413A600A794B79C9
:10D2A000CF8867801B029A186A840A7A4B7A8F7A31
:10D2B000C87A0D7B65701B029A183B04D2180006D1
:10D2C0001018179FF860487B8A7BCB7B3B77120254
:10D2D00010186081087C7877487C149A9072887C5A
:10D2E000D072C87C159B1874087D5874487D1190C5
:10D2F0009874C87D0A7E120212181A84887DD87428
:10D3000018464B7EC375887ECD7E2D022818B880C6
:10D31000087F4D7F2D022818F880887FB877C87F56
:10D32000F8772020085C149D28732120085C68731E
:10D330002A20085C2A314D782D0228188D782D047A
:10D340004019C9780906401818998864119801E0B5
:10D35000EB7DA87C7D498B700A8080001F38C882D5
:10D36000C883139800281FD022227748825C034686
:10D3700022335B781B029A180A842422825C0346BB
:10D3800024335B781B029A18CA842622825C0346E7
:10D3900026335B781B029A188A832822825C283005
:10D3A00040780002801888846948032569A22946CC
:10D3B00002F0D8FD189F387814907B78B8780F90D9
:10D3C000FA78B8791390F8791190387A1090787AC1
:10D3D000B97A0890099100930F98019002921698DB
:10D3E0000390129804901398059011980690109845
:10D3F0000790FAA2F8482946149B02F0B3FD3D4677
:10D40000643580212846F2F7CEFEB878C11E022985
:10D410000ED3012800D18FE1022800D0ABE1169194
:10D42000149078787F225043F7494018F74907E075
:10D430001691149078785B225043F1494018F149D5
:10D4400041182846F2F796FE0D9D1898C6870E34AF
:10D45000324602E0641C0F2A0ADA21780029F9D04A
:10D46000491C8907C90F91400E43C687521CF1E73A
:10D470001699022907D31499491E012900D97DE183
:10D480004279D24901E04279CF4989180C78002DC0
:10D4900000D177E1C1790E91032900D94AE142799F
:10D4A000062A00D979E14921890041181191E43017
:10D4B00010900E98401E129019A800190F9000238A
:10D4C0001392149403E01898290600D15AE1052A12
:10D4D0005AD8C0467A44127952009744455C728506
:10D4E00098ABC04688130000E20400000C0800005E
:10D4F000060A0000040F00000000104130C1BD41C9
:10D50000000070400000F0400000D041120C00000C
:10D51000140B000012120000140E00000E16000082
:10D52000130D0000121600000E120000140B0E0A5C
:10D5300012080000101600000E0B00002A940102D1
:10D540002C940102C4D20102D0D2010298940102AB
:10D55000010800004361736520706172616D65743C
:10D560006572733A200D0A001693DFB2002F04D0C3
:10D5700019A801223946F2F70FFE002C00D191E0E4
:10D5800019A8C019BB498AE0E8B2022867D0002771
:10D59000022867D06BE00E98022872D1E8B2022808
:10D5A00000D103461693DFB2002F04D019A8012240
:10D5B0003946F2F7F1FD002C74D019A8C019ACA1BE
:10D5C0006DE0E8B2022800D104231693DFB2002FE9
:10D5D00004D019A801223946F2F7DEFD002C61D0F3
:10D5E00019A8C0199FA15AE0E8B2022800D1062369
:10D5F0001693DFB2002F04D019A801223946F2F7A2
:10D60000CBFD002C4ED019A8C01992A147E0E8B27A
:10D61000022800D10C231693DFB2002F04D019A8E2
:10D6200001223946F2F7B8FD002C3BD019A8C019E9
:10D63000874934E0E8B2811E4A424A4197000228F5
:10D6400004D119A801223946F2F7A6FD002C16D004
:10D6500019A8C0197CA12246F2F78CFD0FE006271D
:10D66000022804D119A801223946F2F795FD002CB1
:10D6700005D019A8C01980492246F2F77BFD1697FC
:10D6800010E01693DFB2002F04D019A8012239460A
:10D69000F2F782FD002C05D019A8C0197349224663
:10D6A000F2F768FD3C193F2C05D80F98C0194021AE
:10D6B000091BF2F778FD12980228189801D2002071
:10D6C00002E0C078411E884115990870611E2E46FF
:10D6D000E8B202280CD1179A517019A9119AB8C949
:10D6E000B8C2B8C9B8C2B8C9B8C2B8C9B8C20DE0E2
:10D6F000179A117019A9109AB8C9B8C2B8C9B8C296
:10D70000B8C9B8C2B8C9B8C2C10709D1800735467F
:10D71000149C139A169B00D4D5E602208543D2E6CA
:10D72000FE20354605401898149C139A169B29062E
:10D7300028D0CCE637A231E01691149078780B9976
:10D740004143334808181F386F21C9430D9D7A188B
:10D750000378D427D3554378D827D3558378DC274B
:10D76000D355002900D170E6C378E027D355103196
:10D77000001D189FEBE70120404A10E00024002D17
:10D7800000D087E629B0F0BD80290ED30F20B872F3
:10D79000104817998883102020E525A20120014612
:10D7A00002F0E0FB189829B0F0BD1020402904D306
:10D7B000B8720849179B998310E5B8720448179905
:10D7C000888314200AE5C046EF1F0100E81F01000E
:10D7D000150F0000140B000001080000256420252F
:10D7E0006420256420256420256420256420256488
:10D7F0002025642025642025642025640D0A00006E
:10D800003C4601001DF7FFFF543D010089FBFFFF6F
:10D81000444501007472785F6D6F646520706172B9
:10D82000616D65746572206572726F720D0A000019
:10D830004E73666420706172616D657465722065F7
:10D8400072726F720D0A0000FFFFFFFF01FF000000
:10D85000A8230100FFFFFFFFFF0101FFFF01FF0100
:10D86000FFFF01FFFFFFFF01FFFF01FF9429010000
:10D87000FFFF01FFC823010018230100F23C010053
:10D88000002800D10148064908607047D090010285
:10D89000F0B586B0002805D10148006802E0C04616
:10D8A000409401023121C900049141188A791F2353
:10D8B0001A40CD79ED06AD0DAA180D7AED066D0C66
:10D8C00052194D7AED062D0B52198D7AED06ED09A0
:10D8D0005219CD7AED06AD0852194D7CED0752195B
:10D8E000BD4C22600A7B1A404E7BF606B60DB2187C
:10D8F0008E7BF606760C9219CE7BF606360B9219C5
:10D900000E79F606F60992194E79F606B6089219BE
:10D9100062604A6AB14D2A40A2608A6A2A40E26087
:10D920002D22D20087183A7E1A4003937E7EF60697
:10D93000B60DB218BE7EF606760C9219FE7EF6067D
:10D94000360B92193E7FF606F60992197E7FF6068F
:10D95000B60892190E7CF60792192261BA7F1A4016
:10D960000597FE7FF606B60DB218049BC35CDB0676
:10D970005B0CD2184B78DB061B0BD2188B78DB06BE
:10D98000DB09D218CB78DB069B08D2186261CA6922
:10D990002A40A2610A6A2A40E2618A7C01252A4063
:10D9A000CB7CDB079B0F9A180B7DDB075B0FD21834
:10D9B0004B7D9B07DB0ED2188B7DDB079B0ED218AD
:10D9C000CB7D1B079B0D9A180B7E1B079B0CD21857
:10D9D0004B7E5B06DB0A13438A7E520612091A430A
:10D9E000CB7E5B075B0813432362CA6A62620A6BE1
:10D9F000A2624A6BE2628A6B22633922D200835CA4
:10DA00001E462E4066635E425E41B304AE04744F10
:10DA10003C68B443E3183B6083185A782A409C78EA
:10DA20002407E40EA2188C8F6401A2186D4C1440D8
:10DA3000C98FC905490A0919DA78D207120A891863
:10DA40001A791207120989185A79D207D208891847
:10DA5000FB4EB1639968F163997904952940DA79AD
:10DA6000D207920F51181A7B5207D20E89185A7B8F
:10DA7000D206920D51189A7B5207D20C8918DA7B84
:10DA8000D206920B89181A7CD206520A89185A7C3F
:10DA9000520792090A43997CC90649085118316412
:10DAA000D97C039A11401A7DD206920D51185A7DE5
:10DAB000D206520C89189A7DD206120B8918DA7D8B
:10DAC000D206D20989187164197E0F2421405A7E2A
:10DAD000120151189A7E12038918DA7E1207120A6F
:10DAE00051181A7F1207120989185A7F12078918CC
:10DAF000B164997F01942140DA7F1207120E511808
:10DB00003D22D200835C5B075B0D59188418627854
:10DB10001207520C8918A278D206120B8918E278E3
:10DB2000D206D2098918F164217907220A40617965
:10DB3000C9008918A2795206920B5118E27992070E
:10DB4000120B8918227AD2078A18BF490A60627AB2
:10DB5000A37A1B029A18E37A1B04D2184A60E2895E
:10DB6000BA4B13400394228AD2049209D2188A60D5
:10DB700003463033598CB64A114002939A8CD20531
:10DB8000D20A51185622825C12068918B14D2960BA
:10DB9000014656314A788C782402A2188C88640594
:10DBA0006409A218CC78240712196A60CA880C7A12
:10DBB000A407A40BA2184C7A6407E40A1219AA60FD
:10DBC0004989E960492189004118FF22663282189B
:10DBD00000921035002207E000300040FFFFFF00F8
:10DBE00004040040FF3F000084186427E65D03271B
:10DBF0003E406523E35C9B071B0F9B196626A65DD1
:10DC0000B607B60EF3186726A65DB601F318DBB2A9
:10DC10006826A65DB607B60DF3186926A65DB60799
:10DC2000360DF3186A26A65DB607B60CF3186B26F8
:10DC3000A65DB607360CF3186C26A65DB607B60BC4
:10DC4000F3186D26A65DB607360BF3186E26A65D93
:10DC5000B607B60AF3186F26A65DB607360AF3189C
:10DC60007026A65DB607B609F3187126A65DB6073D
:10DC70003609F3187226A65DB607B608F3187326A0
:10DC8000A45DA407E31808C51032802AACD1019A1C
:10DC9000D243704EB4180B783B404D78AD072D0F32
:10DCA000EB188D78AD07AD0EEB18CD78AD01EB1804
:10DCB000DBB20D79AD07AD0DEB184D79AD072D0D2C
:10DCC000EB188D79AD07AD0CEB18CD79AD072D0CA8
:10DCD000EB180D7AAD07AD0BEB184D7AAD072D0B98
:10DCE000EB188D7AAD07AD0AEB18CD7AAD072D0A8A
:10DCF000EB180D7BAD07AD09EB184D7BAD072D097A
:10DD0000EB188D7BAD07AD08EB18CD7BAD07EB189D
:10DD1000A3641031121DBDD1009B19785A785207A7
:10DD2000520D51189A78D207120D8918B164059BCB
:10DD30001968F164D97D5A681202511831659968E1
:10DD4000454A0A40998A490589187165D9683D4C48
:10DD50002140B16519692140F165029E3178049D29
:10DD6000294082785207120F5118C2799207920EF9
:10DD70008918427A9207920D5118827A9207120DF1
:10DD80008918C27AD207920C89189A7DD207520C50
:10DD9000891872789207D20B8918B2781207D20AC2
:10DDA0008918F2781207D2098A182C490A60327C45
:10DDB000737C1B071B0D9A18B37C9B069B0BD21818
:10DDC000F37C1B079B0AD218337DDB065B09D21854
:10DDD000737DDB071B09D2184A60B27D2A40C38FCE
:10DDE0005B009A188A60826CCA60C26C22400A6129
:10DDF000F27D7F231340328C5204520AD2184A61BA
:10DE000002698A614269CA6182690A62C2694A62B8
:10DE1000026A8A62426ACA62826A0A63C26A4A63A0
:10DE2000039A927CD201121D0A64027A3A40CA65B2
:10DE3000808F074A10400866002006B0F0BDC0463B
:10DE400000300040FFFFFF009C300040FF1F00003B
:10DE5000FF03000000400040FFFF1F0000200040C3
:10DE600004480068806B800803490968490040182D
:10DE700009307047409401021004004010B52D2174
:10DE8000C9004118027A032A04D10079002807D07A
:10DE9000082006E08378DA1E022A05D2032412E065
:10DEA000142088601C203DE0012B02D1C8228A602A
:10DEB00012E00479042C01D3462404E0032C01D1A0
:10DEC000322400E014248C605B1E022B04D3022A4F
:10DED00010D24279154B01E04279154B9B181B7803
:10DEE000402B04D0102B06D11423442405E02A2310
:10DEF0003E2402E04279342348244B800C80022ADD
:10DF000006D0062A08D0052A08D118224C2301E0A1
:10DF1000142250230B8000E01C224A80C078042881
:10DF200003D1142048806420088010BDEF1F010039
:10DF3000E81F0100134800687047C04610B5104A3A
:10DF4000107091700F49002813D0506808610420A8
:10DF500048619078FF2212020B4B1C6894438003A7
:10DF600080B20019186001204007084A1060084A72
:10DF7000106000200860074901220A6010BDC046F9
:10DF800030940102180400401CE400E080E200E04C
:10DF900000E100E070000040F0B591B0002801D130
:10DFA000C04800688778F91E022913D3012F21D0B9
:10DFB000022F3CD11021CA4344782146193991429D
:10DFC0003DD800970125B94A28462946234601F045
:10DFD000C9FF53E10821CA434478214621399142BF
:10DFE00018D800970125B14A28462946234601F052
:10DFF000B9FF43E10821CA434478214609399142D7
:10E0000034D800970125A94A28462946234601F01D
:10E01000A9FF33E1032F3CD0042F43D1C37801255E
:10E02000042B00D02DE106462A02042343E00125FB
:10E03000A6A2284629463B4601F094FF1EE1C3787C
:10E040000125052B0AD806462A02284698401B219E
:10E05000084230D10021052B08462ED00220009026
:10E06000914A2846294601F07DFF07E10646C3781C
:10E070000021022B1ED3032B1CD0042B08460A467A
:10E080001BD001250095884A2846294601F06AFFE1
:10E09000F4E0C3780125032B00D0FAE006462A02FB
:10E0A000032308E0012583A2284629463B4601F0C8
:10E0B00059FFE3E00A46012148020F9159218900E6
:10E0C0007518FD21490071180291314662313F05F2
:10E0D000D219641E1F2727405C013C1914430443D6
:10E0E00032795207D20C22432B789B065B0BD21855
:10E0F000B379DB071B0B13436D4D2B60F2790323C0
:10E1000010931A40737A9B079B0E9A18B37A5B0799
:10E11000DB0D9A18F37ADB079B0DD218337BDB07F4
:10E120005B0DD218737B1B075B0CD218AA60326997
:10E13000EA6072692A61B2696A61F269AA61326A47
:10E14000EA61726A2A62B26A6A620F980870F06ABB
:10E15000A8623F20C4432C353046E4300F9030464F
:10E16000E5300E903046E6300D903046E7300C90AA
:10E170003046E8300B903046E9300A903046EA30BD
:10E1800009903046EB3008903046EC30079030462E
:10E19000ED3006903046EE3005903046EF3004907A
:10E1A0003046F03003903746F1373046F230F336E0
:10E1B0000F990A194021525C109B1A400E9B1B19A3
:10E1C0005B5C9B071B0F9A180D9B1B195B5C9B07E5
:10E1D0009B0E9A180C9B1B195B5C9B019A18D2B280
:10E1E0000B9B1B195B5C9B079B0D9A180A9B1B19C9
:10E1F0005B5C9B071B0D9A18099B1B195B5C9B07BB
:10E200009B0C9A18089B1B195B5C9B071B0C9A18AC
:10E21000079B1B195B5C9B079B0B9A18069B1B19A2
:10E220005B5C9B071B0B9A18059B1B195B5C9B0790
:10E230009B0A9A18049B1B195B5C9B071B0A9A1884
:10E24000039B1B195B5C9B079B099A183B195B5C42
:10E250009B071B099A1803195B5C9B079B089A187C
:10E260003319595C8907891802C51034A0D1029866
:10E270000078042101430E48C1630025284611B0EF
:10E28000F0BD04200090084A2846294601F06AFEA5
:10E29000F4E703200090044A2846294601F062FE74
:10E2A000ECE7C04640940102C73C01000D3D01006F
:10E2B00000100040556E646566696E6564206D658A
:10E2C000616E205052462025640D0A00496E766129
:10E2D0006C6964206D65616E205052462025640D86
:10E2E0000A0000007047704780B50E490E4802468C
:10E2F000083A1268920000D4603142680A434260D2
:10E300000A490A6808239A430A60091F0122520435
:10E310000A600321890402688A430260FBF708FA55
:10E3200080BDC0462000008028000040040200405C
:10E33000B0B5032000072D490A688243012568070C
:10E340001018086000242046FFF7CDFF2046FFF795
:10E35000C9FFEFF31080284002D1EFF3108172B6AD
:10E360008021C943224A53680B40536093680B4095
:10E370009360D3680B40D36013690B4013615369FA
:10E380000B405361002800D162B6B0BD70B50C4699
:10E3900003210907154A13680B4313600122EFF3A9
:10E3A0001081114002D1EFF3108272B68025EA434A
:10E3B0000F4B5E6816405E609E682E439E60DD686F
:10E3C0001540DD601D6915401D615D6915405D6189
:10E3D000002900D162B6002802D00120FFF783FF98
:10E3E000002C02D00120FFF77DFF70BD000400402B
:10E3F000D09501020D4A002907D001290BD1012136
:10E40000814010688843106007E001218140106856
:10E410000843106001E001218140101F02680A4397
:10E420000121C907114301607047C0464400004004
:10E43000032804D840000649085A00B2704700205B
:10E4400000B27047032802D84000014A11527047B9
:10E45000FED201029E4908707047C04670B58AB06E
:10E460000C460546FF20FC30A8490E68315C592057
:10E470008000335CB278307808AE069609AE059617
:10E480000C4E04962126760603960B4E0296012624
:10E4900001960E2600965B1CDBB2F7F7C5FB0998C8
:10E4A000F2F77CFA28700898F2F778FA20700AB030
:10E4B00070BDC0460000204100000443F0B58BB0A1
:10E4C0000446457C824800788249002822D00020FA
:10E4D0000880814A1080814B01269E761E830A9017
:10E4E0007F4800787F4E36786DB205957E4D049555
:10E4F0007E4D03950AAD02957D4D01950096F7F787
:10E50000D1F80A9D112020567A497B4A00F036FC4A
:10E51000064626E000260E806F4A16806F4B0120CB
:10E520009876188309966E4800786E4F3F786DB2E2
:10E5300005956D4D04956D4D039509AD02956C4D96
:10E5400001950097F7F7AEF8099D112021567F201D
:10E55000C005009001900296664A674B3046F8F776
:10E56000F5F9432001062846F1F74EFFF2F716FAB7
:10E57000089062480078002824D05120800060492B
:10E580004A7D42438D185F480068A8642F46403793
:10E5900050480078B87450480078F87455480078AE
:10E5A000387555480078787557480078F8755048A0
:10E5B0000069F2F7F3F9B87552484069E8644C48CD
:10E5C00000686864FF20FE3050490968085C392201
:10E5D000D2008918022812D303D04E4800780128AF
:10E5E0000DD14B480660434800883A4A10804248A3
:10E5F0000088394A108009200790089605E04448B1
:10E60000089A02603548C08B07900B780022002BD7
:10E6100001D0114600E0D1430125002B01D0042395
:10E6200000E0EB43A67AAD1BEE175B1971416568FC
:10E63000AE0F277AAD00ED195641677A3F1FF817E4
:10E64000ED1970414000EE0F80196D00EB18484144
:10E650008001990E4118980127239B02C31A91410A
:10E660001D4805881B480088854201D00798421B39
:10E6700010202056C001194D2D8C032D07D1E468C0
:10E68000E5176D0A6419E4150519EC170FE0E46845
:10E69000E5176D0A6519EC17ED15C6174519744194
:10E6A00097B2002F00D03446002F00D00546581BEB
:10E6B000A141130409D012B2D2015242D3178018DB
:10E6C0005941089BDA17C01A91410BB0F0BDC04602
:10E6D000C29301026CAD01026AAD0102989401027D
:10E6E000B1900102B090010258A3010254A10102AD
:10E6F00070AD0102BAAD0102B8AD010224A701025A
:10E700005CA401026420004068AD01024094010253
:10E7100064AD0102C8AD0102C10D400280307047F6
:10E720000120C0071B4908607047C04610B5194852
:10E730000068C10710D1810711D4410712D4010725
:10E7400013D4C10614D4810615D4410616D48021F1
:10E75000084016D031A215E001240FA213E00224D4
:10E7600011A210E0032414A20DE0042416A20AE072
:10E77000052419A207E006241CA204E0072421A214
:10E7800001E0254A04090220032101F0EBFB2046A9
:10E7900010BDC0465C00004052657365742062790C
:10E7A00020504F520D0A0000526573657420627943
:10E7B00020424F520D0A0000526573657420627941
:10E7C0002050494E0D0A000052657365742062792D
:10E7D000205744540D0A0000526573657420627915
:10E7E000204C4F434B55500D0A0000005265736595
:10E7F00074206279205357205265626F6F740D0A3E
:10E8000000000000526573657420627920535953EB
:10E810005245510D0A000000722F010052657365C8
:10E820007420627920445644440D0A00012181403D
:10E83000044A1F2802D010688843106010680843FB
:10E84000106070471C000040F0B583B00291044690
:10E850009949F1F73FFC0546984901942046F1F7A4
:10E8600039FC974946189749714300956F189649A6
:10E87000441864212046F1F72DFC3818A108471AE6
:10E8800092492046F1F73CFC381891494518914FC0
:10E8900005D464213046F1F71DFC0C4614E0A6B205
:10E8A00064213046F1F716FCB7204000A20701D1E1
:10E8B000002907D1884B73430422D341874A9342EE
:10E8C00000D3401E0C464519009847430298068025
:10E8D000192001013046F1F7FDFB2A461F3A284670
:10E8E00000DB1046019BFF18B30705D1002C03D0B5
:10E8F0001F2D05DA0120C5E01F2D0BDA0120C1E034
:10E9000005461D3D034600DB2B461C2808DC022083
:10E910001546B7E000290CD01C21451A0CD50CE097
:10E9200019461F39184600DB08461F2B1DDA032045
:10E93000A8E01D21451A00D42846002D08D4014620
:10E940001F39024600DB0A461F2804DA032099E03B
:10E950000220154696E015461E3D104600DB28466F
:10E960001E2A0CDA04200D468CE005461E3D0246A8
:10E9700000DB2A461E280BDA04200D4682E0014601
:10E980001F39024600DB0A461F280ADA052079E013
:10E9900011461F39104600DB08461F2A0BDA0520F6
:10E9A00070E015461E3D104600DB28461E2A0CDA94
:10E9B00006200D4666E005461E3D024600DB2A465F
:10E9C0001E280BDA06200D465CE001461F39024680
:10E9D00000DB0A461F280ADA072053E011461F39D8
:10E9E000104600DB08461F2A0BDA07204AE01546CE
:10E9F0001F3D134600DB2B461F2A0CDA08200D466C
:10EA000040E005461F3D024600DB2A461F280BDA80
:10EA100008200D4636E019461E39184600DB084628
:10EA20001E2B0ADA09202DE011461E39104600DBA4
:10EA300008461E2A0BDA092024E01F28054601DBC0
:10EA400005461F3D1F280CDA0A200D461AE01F2834
:10EA5000054601DB05461F3D1F2806DA0A200D4644
:10EA600010E01E2D05DB0C2004E01E2D06DB0C2023
:10EA700005E00B201E2D05DB1E3D03E00B201E2DA7
:10EA800000DB1E3D029EB070681CF070E1200101A9
:10EA90003846F1F71FFB3071C0B211494143CC1920
:10EAA0003C212046F1F716FB70713B21C9434143DD
:10EAB0000819B07103B0F0BD805101008033E1014D
:10EAC000B207000093FEFFFFB107000070FEFFFFDA
:10EAD000A7FA0A0080AEFEFF295C8FC20BD7A30005
:10EAE000F0F1FFFFF0B581B00446FFF721FCA08AEA
:10EAF00000280ED0FFF71EFA2049086120482CCCD0
:10EB00002CC02CCC2CC02CCC2CC00020888101B077
:10EB1000F0BDE08A194FB881A169BA891948F1F7A7
:10EB200029FB174D204629464CC84CC14CC84CC146
:10EB30004CC84CC1FFF7FEF938616E68FFF790F9D9
:10EB4000301AB8622846FFF7B9FC06460D460E4853
:10EB5000007BFFF76DFC0121F970617C7971396CE4
:10EB6000491C396481B2C90B401800B2C11740106A
:10EB7000301A38658D417D6501B0F0BD60990102A4
:10EB80003C9A010208D30102B290010270B504461A
:10EB9000FFF7CEFBA08A244E7082718A002908D02C
:10EBA000B0820220707100203082FFF7C3F9F0615B
:10EBB00070BDE08A3082A169328A1C48F1F7DAFA26
:10EBC0002046FFF77BFC05460C461948007BFFF703
:10EBD0002FFC81B2C90B401800B2C1174010281A8F
:10EBE00030668C417466FFF7A5F9B061F06C401C8B
:10EBF000F064FEF73FF9F063FAF760FC0446306416
:10EC00000C48406AF1F744FF0B4A0C4BF1F72AFD20
:10EC1000F1F7F2FE01462046F1F772FAFAF786FEA6
:10EC20000120707170BDC046E0960102A0D30102C0
:10EC3000C0900102A82001008DEDB5A0F7C6B03E3E
:10EC4000F0B581B0EFF3108072B600200146FBF7FB
:10EC50007FFE0446002803D062B6204601B0F0BD16
:10EC600001273A030025074E28463146FBF7CAFD27
:10EC7000BB02174A28463146FCF7A2FA62B6204684
:10EC800001B0F0BD00E0020480B5F5F7D0FDF9F762
:10EC900039F9F9F7ADF9F7F719FF0C490120C872F6
:10ECA0000A7B03469343CB71521C0A73084A928F26
:10ECB000002A08D08A7A4B78134304D04A7A501C31
:10ECC0004872012090430349087080BDB09801024A
:10ECD00062A901022994010270B514460D46064648
:10ECE0001120FAF7D3FE2248042101600C48046089
:10ECF0001E4805608660002E0DD0FF2000060949E1
:10ED00000A6882430120C0071018086006480821DD
:10ED10000160064801601A200221FFF76BFB70BDFD
:10ED2000A0D4010200E400E080E200E000E100E0A5
:10ED30000C4908607047C04610B504460948006891
:10ED400060430949F1F7DCF90019084948600848AF
:10ED50000022026002460C3A4B68136009680160A9
:10ED600010BDC0469CD4010240420F000C9001022D
:10ED70002C10014000480047C100000080B582B05F
:10ED800013460A4600900348011D0348F7F78AFD21
:10ED900002B080BDDCD401028CA0010210B50C4988
:10EDA0008A1C90420DD2401E0D4A50600D480368E7
:10EDB0000B4003218C071B19036000209060116039
:10EDC00010BD04480449E622044B00F06FF8C04629
:10EDD000FFFFFF00492F0100632F01002F2F0100CB
:10EDE00010E000E020ED00E0B0B50120EFF310816D
:10EDF000014002D1EFF3108272B6124A1368124C2E
:10EE0000226864688506114800682840850E5D19EF
:10EE10002923DB006B43002C1D4606D1002809D1B5
:10EE20001E20684300290AD0B0BD121BD218551C01
:10EE30000028F5D01D461E2068430029F4D162B693
:10EE4000B0BDC0460CE0010214E000E004ED00E0BB
:10EE500080B50020FBF726F8404280BDB0B586B0F3
:10EE6000104869460A4638C838C238C838C2002433
:10EE70002046FBF71DF803992046FBF7B3F80198ED
:10EE8000012803D00824002804D102E0042400282B
:10EE900000D104460220FAF701FEE0400249086072
:10EEA00006B0B0BDF41F010020E0010290B01C4686
:10EEB00005AB07C3EFF31080C00702D1EFF310805A
:10EEC00072B6EFF310800B9068460E907046089073
:10EED00010AB0F93CF4F3E1D01200490C50230466A
:10EEE0002946224600F0B8FC00213154EFF303809C
:10EEF0000990EFF308800C90EFF309800D90EFF389
:10EF000014800A9000F02CFC3868012833D80028BF
:10EF1000C14F00D0C14F2A20C1497A69920703D559
:10EF20000A783A60401E491C0028F6D1B948041DF1
:10EF30002046F1F74DF9002807D079698907FAD5FD
:10EF400021783960401E641CF5E70220B5497A69D2
:10EF5000920703D50A783A60401E491C0028F6D172
:10EF60002A20AF497A69920703D50A783A60401E91
:10EF7000491C0028F6D1FFF737FF0346AA4A30465E
:10EF80002946FDF7A9FE04463018291B089F3B1FA0
:10EF9000049A9343A5A2FDF79FFE9E4909680129A3
:10EFA00066D8001900299C4C00D09C4C00280AD03F
:10EFB0009849091D6269920703D50A782260401EAC
:10EFC000491C0028F6D10A209F496269920703D59F
:10EFD0000A782260401E491C0028F6D10598F1F7F6
:10EFE000F7F8002809D061698907FAD5059A1178E0
:10EFF0002160401E521C0592F3E702208949626994
:10F00000920703D50A782260401E491C0028F6D1D9
:10F010000A208EA16269920703D50A782260401EF9
:10F02000491C0028F6D10698F1F7D2F8002809D03B
:10F0300061698907FAD5069A11782160401E521C31
:10F040000692F3E7022077496269920703D50A78AE
:10F050002260401E491C0028F6D10A207EA1626968
:10F06000920703D50A782260401E491C0028F6D179
:10F070007CA230462946079BFDF72EFE65490968AC
:10F0800001290E9B1BD80029634900D06349002841
:10F090000AD0604A121D4C69A40703D514780C608D
:10F0A000401E521C0028F6D102205E4A4C69A4077B
:10F0B00003D514780C60401E521C0028F6D16AA2B9
:10F0C00030462946FDF708FE04463018291B694AD8
:10F0D0003B46FDF701FE4F490968012911D8001987
:10F0E00000294D4900D04D4900280AD0494A121D37
:10F0F0004B699B0703D513780B60401E521C0028F8
:10F10000F6D15D4A30462946099F3B46FDF7E4FDAE
:10F110000446F800C00FB900C90F7A00D20F009260
:10F12000019102903019291BFB0F544AFDF7D4FDC1
:10F1300004193019291B3F233B40514AFDF7CCFDF0
:10F1400034490968012911D820180029324900D012
:10F15000324900280AD02F4A121D4B699B0703D55C
:10F1600013780B60401E521C0028F6D1454A3046E9
:10F1700029460B9BFDF7B0FD04463018291B424A77
:10F180000A9BFDF7A9FD23490968012911D8001937
:10F190000029214900D0214900280AD01D4A121D0A
:10F1A0004B699B0703D513780B60401E521C002847
:10F1B000F6D1364A304629460C9BFDF78DFD0446B4
:10F1C0003018291B324A0D9BFDF786FD114909684D
:10F1D0000129114A0DD80019002908D00F4A06E06C
:10F1E0005169890703D531781160401E761C0028CB
:10F1F000F6D128490E98091AA94200D32946890850
:10F2000000F03AFE24480068002800D0804700F053
:10F2100045F8C046F0E001020090014000A0014026
:10F22000A32F0100313D01008C2F01000D0A232383
:10F230002320415353455254204020307825303804
:10F2400058202323230D0A006630010046554E4303
:10F2500054494F4E3A2000004C494E452020202072
:10F260003A200000256400000D0A53503D25303837
:10F27000580D0A002B300100413001004D300100D3
:10F2800035300100EA2F0100F92F0100083001009C
:10F290001330010000F80202ECE00102F7480068B8
:10F2A000012811D8002801D00B4800E0FC480C21AF
:10F2B0000A4A01E0002907D043699B07FAD5137871
:10F2C0000360491E521CF5E71E20FFF7AFFA00BF8E
:10F2D00000BF00BF00BFFAE700A00140962F010069
:10F2E0008AB00646E448B06600F03AFAFFF77CFDC3
:10F2F0000346E248041D01200590C502E04A20466D
:10F300002946FDF7E9FC074608942018DB4C0995CF
:10F31000E91BF36C3F2206921340DAA2FDF7DCFCF6
:10F320002168012910D8C0190029DD4900D0DD4924
:10F33000002809D0221D4B699B0703D513780B6069
:10F34000401E521C0028F6D1F36BD7A2089C204621
:10F35000099D2946FDF7C0FC0746291A2018336C81
:10F36000069A134007D1D8A2FDF7B6FCC34C21681A
:10F37000012907D917E0CEA2FDF7AEFCBF4C2168EA
:10F38000012910D8C0190029C54900D0C549002855
:10F3900009D0221D4B699B0703D513780B60401ED3
:10F3A000521C0028F6D10027CBA5B8003058009099
:10F3B000089809992A463B46FDF78EFC21680129E9
:10F3C0000FD80029B64900D0B649002809D0221D1F
:10F3D0004B699B0703D513780B60401E521C002815
:10F3E000F6D17F1C0D2FE0D1736BBFA2089C204685
:10F3F000099D2946FDF770FC074620189F4CE91B24
:10F40000B36BBC4AFDF768FC2168012910D8C0190C
:10F410000029A34900D0A349002809D0221D4B6927
:10F420009B0703D513780B60401E521C0028F6D1B1
:10F43000336CB14A089C2046099D2946FDF74CFCD7
:10F440000746326CD000C00F9100C90F5300DB0F8C
:10F45000009301910290E019E91BD30FA74AFDF731
:10F460003BFC3246C619A019A91B1546136C069A17
:10F470001340A34AFDF730FC80490968012911D8DF
:10F4800080190029864900D0864900280AD07B4A85
:10F49000121D4B699B0703D513780B60401E521C4D
:10F4A0000028F6D12E466B6C964A089C2046099D92
:10F4B0002946FDF711FC07462018E91B0796B36C97
:10F4C000914AFDF709FC6D4A1168012910D8C0194D
:10F4D0000029734900D07349002809D0121D4B69D7
:10F4E0009B0703D513780B60401E521C0028F6D1F1
:10F4F0000798426E042360215C2004931A400B4657
:10F5000000D003460693002A00D00846079E3358D1
:10F510007E4A089C2046099D2946FDF7DDFB0746EB
:10F5200006983358E019E91B794AFDF7D5FBC6194F
:10F53000A019A91B079A536E76A2FDF7CDFB4F4980
:10F540000968022911D280190029554900D055496E
:10F5500000280AD0494A121D4B699B0703D513782E
:10F560000B60401E521C0028F6D10798C36C06465B
:10F570006DA2089C2046099D2946FDF7ADFB074674
:10F580002018E91B336D6B4AFDF7A6FBC619A019BD
:10F59000A91B079F7B6D68A2FDF79EFB8619A0192A
:10F5A000A91BBB6D67A2FDF797FB344909680129C8
:10F5B000059C11D880190029394900D03949002803
:10F5C0000AD02E4A121D4B699B0703D513780B6096
:10F5D000401E521C0028F6D10798476B5D4A97429F
:10F5E00037D2032087430026059CB00039580246D5
:10F5F000049B1A43BA5808230343FB580C250543C0
:10F600007D5900910192029303953B18089809993E
:10F61000514AFDF761FB1949096801290FD80029F2
:10F620001F4900D01F49002809D0089A4B699B0741
:10F6300003D513780B60401E521C0028F6D11B2EF8
:10F64000444A06D80798406B361DB10040189042D6
:10F65000CBD30798406B111A099A914201D88908B7
:10F6600000E0610200F008FC3C480068002800D07F
:10F670008047FFF713FEC04622224B4DF0E0010207
:10F680008C2F01000D0A0D0A2323232045584345E2
:10F690005054494F4E202564202323230D0A000097
:10F6A0000090014000A0014050433D2530385800F3
:10F6B0002C20457863657074696F6E4E756D626558
:10F6C000723D25640D0A00002C2054687265616447
:10F6D0004D6F64650D0A000052252D32643D2530C2
:10F6E00038580D0A0000000053503D253038580DA1
:10F6F0000A0000002B300100413001004D300100B4
:10F7000035300100EA2F0100F92F01000830010017
:10F71000133001004558435F52455455524E3D2524
:10F720003038580D0A000000494353523D25303807
:10F73000580D0A001E3001005343523D2530385801
:10F740000D0A00004343523D253038580D0A0D0A7A
:10F750000000000000F80202CE2F0100ECE00102E0
:10F76000F0B583B0344D2C68012C06D8601E84415E
:10F77000204601F077FB0028FAD10120EFF3108139
:10F780000140019102D1EFF3108072B62B48285A44
:10F790002B49695A814245D02A68002A01D02A4E55
:10F7A00000E0284E1F23DB020293284C022A27D2B6
:10F7B00005E01046214AA85282B2914232D087B267
:10F7C000B9420A4600D8621C131A21482B52180469
:10F7D0000DD0E819001D9FB201E0002F07D073691A
:10F7E0009B07FAD5037833607F1E401CF5E7A242E1
:10F7F000DFD902981018DDE7304683B299420CD069
:10F80000024680B281420E4600D8661CA642F3D959
:10F810000298301883B29942F2D108496852B01A5E
:10F820000B4968520B48002129540198002800D147
:10F8300062B603B0F0BDC046F0E001020A08000065
:10F84000080800000090014000A00140FF070000F0
:10F850000C0800000F080000F0B58DB007931746A4
:10F8600000240C9409AA13C215E006986849F0F721
:10F87000CBFDF1F793F8C117401848406549F0F700
:10F8800029FC009509A806223346F9F78BFABDE05A
:10F89000002C00D5BEE138787F1C25280DD000282B
:10F8A00000D1B7E10B9A511C0A9B9942F0D8099BF1
:10F8B0009854641C0C940B91EAE70894002539785D
:10F8C00023390D2914D801207944097949008F443E
:10F8D000090F0F0F0F0F0F0F0B0F060F0F0D054323
:10F8E0007F1CECE70820FAE70420F8E70220F6E79F
:10F8F0003878014630390024092902D9264639468C
:10F900000BE000260A2171430E18303E791C7878EE
:10F910000246303A0A2A0F46F4D32E2817D14A1C41
:10F92000487801463039092905D911464F1C253838
:10F93000532811D96AE000240A2161430C18303C95
:10F94000511C50780246303A0A2A0A46F4D34F1C1A
:10F950002538532800D959E04000C04678448088B3
:10F9600040008744A000530053005300530053004D
:10F9700053005300530053005300530053005300EF
:10F9800053005300530053005300530053005300DF
:10F9900053005300530053005300530053005300CF
:10F9A00053005300530060005300530053005300B2
:10F9B00053005300530053005300530053005300AF
:10F9C000530053005300530053009800530053005A
:10F9D000530053005300530053005300530053008F
:10F9E000AD00B600530060005300590053005300AF
:10F9F00053005900530053005300DE0053005300DE
:10FA0000BD005300D3005300530098000C9C3FE707
:10FA10000024744940420F00791C38780F4625387D
:10FA20005328F3D898E70799C91D07208143086830
:10FA300007914968F1F740F800210690F0F70EFFB2
:10FA400000280BD10B99481C0A9A904206D8099AB3
:10FA50002D2353540899491C0C910B90079808309A
:10FA600007900698F0F79AFF0095C2178118514049
:10FA700009A822463346F9F795F90B98411C0A9AD2
:10FA8000914200D9F1E6099A2E2313540B910C9858
:10FA9000401C0C90E9E6079802C807900096019573
:10FAA00009A8102239E00B98411C0A9A9142ADD85E
:10FAB000099A252313540B910C98401C0C90A5E730
:10FAC0000B9A511C079C201D0A9B994239D907901B
:10FAD0009CE7079802C80790009509A82246D3E63C
:10FAE000079901C9079109990A9A089E02E0401CEA
:10FAF000002E8BD40378002B88D00B9D6C1C944275
:10FB0000F5D84B55761C0C960B94F0E7079802C875
:10FB100007900096019509A80A222346F9F7E0F913
:10FB200074E7079B10CB102C079308D300202146C5
:10FB3000401C0A09FF291146FAD806280AD80820CD
:10FB400009E02368099CA354089A521C0C920B915B
:10FB500007905BE7401C069009230C980B9D0999C0
:10FB600005910A9E04940DE0202104463046059E2E
:10FB7000715506462046049C401C154601460891D6
:10FB800000290AD45B1E0699994206D26A1CB24229
:10FB9000EAD9089908910029F4D50C900B9508989A
:10FBA000002800D532E70126082501E06D1E360148
:10FBB000022DFBD220463146F0F78CFA0F28F6D8FA
:10FBC0000C980590099803900A9806900B9D204682
:10FBD0003146F0F77FFA691C069A914204D90899D8
:10FBE000089100290CD511E00C4A125C039B5A5570
:10FBF000089A521C0D46059211460891002905D419
:10FC00007043241A3009102E0646E0D205980C9055
:10FC10000B95FBE620460DB0F0BDC046E822010082
:10FC200070B588B00022032803D9D243104608B02B
:10FC300070BD7F4CC34D2A510F4B104EEE508123A7
:10FC40001E010123AB5528602C1962600128EDD8F4
:10FC500007930022069205920492032303930292D3
:10FC600001920091411E8841694600F02BFD024639
:10FC7000104608B070BDC04604080000FFC0FFC0B9
:10FC8000F0B583B00C460023D943012C56DB074660
:10FC900002910126EFF31085354002D1EFF3108079
:10FCA00072B65849584A505C002800D0A3E0565418
:10FCB0005E48115A5E48105A0196F202161A8142A5
:10FCC00040D832465218A24240DB00930295A64229
:10FCD000354600DB25464C490818001D39462A46A2
:10FCE000F0F748FAA642484E04DA7919621B301D33
:10FCF000F0F740FA4E48305A001981B24D4A91420D
:10FD000001D94D494018029D009B49497052304627
:10FD10004A4E805D002865D1EFF3108501980540BB
:10FD200002D1EFF3108072B6374A4048115A40486A
:10FD3000105A884232D1424813524FE00C462046B6
:10FD400003B0F0BD42425218A242BEDA3B4A2E4EE8
:10FD5000B25C002A0CD03A4AB25A51188AB2354CD9
:10FD6000A242284C029F01D9334A8918304A02E046
:10FD7000244C2F4A029F3355B152421A89B288420D
:10FD800002D22C488018421C93B22F4801212FA286
:10FD900000F0E8F83C46002DD1D128E0019F9755AE
:10FDA000884201D82348401C421A90B2800A01D0F0
:10FDB000019882022248144F3A52386801280DD81F
:10FDC000431E9841104B5918091D92B21D4B00F06B
:10FDD0008FFE009B002801D00B488355002D029D0B
:10FDE00000D162B6074808490B54002DA7D162B66E
:10FDF000204603B0F0BD21200201044804A108A35D
:10FE0000FFF754F80E080000F0E00102E2300100B4
:10FE100074726163655F6F757470757400000000C3
:10FE20005452414345204255535900000A080000EE
:10FE300008080000FF07000000F8FFFF0F0800009F
:10FE40000C0800009100010002FF00000D0A54722E
:10FE500061636520627566666572206973206675E8
:10FE60006C6C2C2064697363617264732025752047
:10FE700062797465730D0A00F0B587B005460026F7
:10FE800006960596049603960296800701D007B061
:10FE9000F0BD019102A8142126A2FCF71DFF2949FB
:10FEA0000968012911D80029274900D027490028CD
:10FEB0000BD002AA01E0002807D04B699B07FAD5B6
:10FEC00013780B60401E521CF5E701990029DED023
:10FED000204C3746B8002B58D80724D0581EA042D3
:10FEE00004D31B4818181C4A90421CD802A814219D
:10FEF0001AA2FCF7F1FE13490968012911D800295B
:10FF0000114900D0114900280BD002AA01E00028B5
:10FF100007D04B699B07FAD513780B60401E521C23
:10FF2000F5E7761C01997F1C8F42B0D2322ED1D3D7
:10FF3000ADE7C0460D0A4261636B74726163653A56
:10FF4000200D0A00F0E001020090014000A00140F5
:10FF5000FFFFFFFCFFFF0200FEFF010025303858C5
:10FF60000D0A000081B0F0B5C4B00E4607464993B3
:10FF7000812000012F49085C002845D00292012011
:10FF8000050204A82946F0F70EF9FCB20021C84387
:10FF90000C2C3AD8721E032A37D82748005DB0428D
:10FFA000084632D3F80535D50021B8050DD404A88C
:10FFB00001904018691AA20022A39B582E4AFCF710
:10FFC0008BFE0198F0F704F9014678050ED404AFD2
:10FFD0007818691AB20029A3D218121F1368264A8A
:10FFE000FCF77AFE3846F0F7F3F80146029A04AEC1
:10FFF00070180C46691A49AB0393FFF72DFC0119E1
:020000040001F9
:100000003046FFF73DFE00E0002044B0F0BC02BCEB
:1000100001B00847FEF7E8FE034604A8019007A2D6
:100020002946FCF759FE0198F0F7D2F80146B805C9
:10003000BDD5CAE7F0E00102144901002531307551
:10004000207C200086300100DC300100D630010029
:10005000B530010080300100A1300100CF30010037
:10006000C8300100C3300100793001008C3001003C
:100070009C3001007130010095390100BB30010056
:10008000A7300100AE3001009230010000000000F6
:10009000F0B581B00B460120EFF31084044002D18B
:1000A000EFF3108172B6990F07D0022001212DA223
:1000B000FFF758FF002C3DD141E02249224D002797
:1000C0006F54224AAB5A224AAE5AF3189EB2F60A2D
:1000D00001D0204E9B19AB52EFF31086064002D19F
:1000E000EFF3108372B6AA5A1C4BEB5A934202D11B
:1000F00016482F521AE06854934201D8164B5B1CE5
:100100009B1A99B2890A00D0830210482B522868A2
:1001100001280BD8411E8841A918091D9AB2104B1D
:1001200000F0E6FC002801D006482F54002E03D032
:10013000002C04D001B0F0BD62B6002CFAD162B63A
:1001400001B0F0BD0F080000F0E001020C08000053
:100150000A08000000F8FFFFFF0700000808000081
:100160009100010055415254204572726F72202552
:10017000780D0A0010B50446FEF7DAF8A08A0028C8
:1001800000D010BDFDF7D6FE034908620861486C37
:10019000401C486410BDC0466099010210B5044679
:1001A000FEF7C6F8A08A002800D010BD0A4CA06C4B
:1001B000401CA064FDF7BEFE6062606C002805D0A4
:1001C000FDF7B8FE60650020606410BDA069206581
:1001D0000120606410BDC046E0960102B0B50A205F
:1001E00000242146FBF7C6FC09202146FBF7C2FC90
:1001F0000124204600F03CF80E2004252946FBF798
:10020000B9FC0D202946FBF7B5FC0549204600F056
:1002100059FAA2021449154B204600F027FBB0BD45
:10022000D8940102B0B50E2000242146FBF7A2FCB1
:100230000D202146FBF79EFC0124204600F018F813
:100240000A2004252946FBF795FC09202946FBF7DF
:1002500091FC2046F9F738FAA2020349034B2046E5
:1002600000F004FBB0BDC04610CE0102A50A01009B
:1002700070B5012801D9012070BD48224243734B5B
:100280009C58A5691F218D43A5610625A5600F25F2
:1002900025629C18A27C002A05D1627C002A02D12A
:1002A000227C002A14D06368002B11D4251D0B403A
:1002B000012216469E400C4B1E60BFF34F8FBFF3CA
:1002C0006F8F2B68002B03D40B409A4007490A60BC
:1002D000002803D0012804D1092000E00820F9F704
:1002E000CDFB0020A06170BD80E100E080E200E075
:1002F000F0B585B00D460278E348C368934219D043
:10030000446D944216D08368934203D0016D9142AC
:1003100000D07FE09B1A591E8B410493482159431A
:10032000032D46D14418E16900294ED01C34002029
:1003300020606DE09B1A5A1E93410493032D1AD13D
:10034000039548225A438418A26B0121EFF31085CC
:100350000D4002D1EFF3108772B6A7691026B7439C
:10036000A761A669002E01D118342160002D00D1AB
:1003700062B6039D0CE04821594342189169183236
:10038000302902D0116810294CD18021116000223F
:100390004821594340180021816301628162243061
:1003A00000210160002A33D004A82946904705B0F7
:1003B000F0BD421891691832302902D01168202905
:1003C00039D180211160002216E00395E26B0126ED
:1003D000EFF31085354002D1EFF3108172B6A169B9
:1003E0002027B943A161A169002901D118342660F1
:1003F000002D00D162B6039D4821594340180021C9
:10040000C163C1624163303000210160002ACBD159
:1004100005B0F0BD00920E4A2E329C480D490E4B9D
:10042000FEF744FD10680093019098480949084A76
:100430000A4BFEF73BFD106800930190044A2432FA
:1004400092480449054BFEF731FDC046F89401027D
:10045000B10200005E3101003331010017310100AB
:10046000F0B585B0049048210A464243864B9C581B
:10047000E6690F2535409A18167C002E31D04F20A2
:1004800040026169014200D185E0A06904218843EE
:10049000A06102202062012081076918D161D36B1D
:1004A000EFF31084044002D1EFF3108572B6956922
:1004B0002026B54395619569002D00D173E0104663
:1004C0003C30002C00D162B600240460D462546336
:1004D000303200201060002B63D004A8984705B08C
:1004E000F0BD0C2D5DD8C0467D442D796D00AF4424
:1004F00067586B580658A1635858585806009569B4
:10050000202D04D0154618352D68302D49D1156B96
:10051000566B3432AE4217D26669360714D564681A
:1005200015686E1C166048431818C06A4455049834
:100530000C4644431A19156B566B3432AE4203D243
:100540001C5966693607EAD41268AA4229D1414388
:10055000585882690524A24382615A18D36B01213D
:10056000EFF31080084002D1EFF3108472B6946963
:100570002025AC4394619469002C02D114461834B0
:10058000216014463C34002800D162B6002121606D
:10059000D16251639CE70C2D00D176E7012D00D18B
:1005A00073E705B0F0BD15461835286010463C309D
:1005B000002C00D187E787E70420206205B0F0BD5A
:1005C0000120206205B0F0BD0825256216461836C8
:1005D0009569102D02D03568302D4BD10396566A9F
:1005E00015462835976AB74228D1A0690221884369
:1005F000A061936B0121EFF31080084002D1EFF36B
:10060000108472B6039E34681027BC43346034688B
:10061000002C00D1316014463834002800D162B675
:100620000021216029601162243200201060002B1B
:10063000B7D052E70220206205B0F0BD2A68B2426E
:10064000AFD262699207ACD52A68561C2E60484327
:100650001818006A805C206004980A4642439D187E
:10066000AC6A6E6AB4429CD228359C586269920783
:10067000EAD496E7316800900191044804A1094A40
:1006800009A3FEF713FCC046F8940102FD300100F7
:10069000756172745F6972715F68616E646C6572B6
:1006A000000000003D0300005561727420256420A5
:1006B000737461746520676F65732077726F6E67FE
:1006C00020256400F0B585B00E460546022804D307
:1006D000002E02D1012005B0F0BD002D03D0012D68
:1006E00008D1092400E008242046F9F7CFF9204674
:1006F000FEF79CF848216943E74A505883691F2454
:100700000294A3438361062383600F230193036252
:1007100057180023BB62BB63FB633B627B62FB62D7
:100720003B63317F3974727F7A74B27FBA740493F9
:100730007B637368B268F468920022435B1E032BEC
:100740000ED8C0467B441B795B009F44010503071C
:10075000082304E0282302E0182300E038231A438A
:10076000C260C907090F72699201D2B28918B269D1
:100770009207920E8918491C8160796131690129BB
:1007800001D122210161012D5CD831680E2959D295
:100790003846123003900324002D01D0204600E09B
:1007A00004204C432D490E19B178F9F7FFF9396847
:1007B000CA68802510462843C8602848005D7378C1
:1007C0001B021818C862AA43CA60F9F737FA0398DF
:1007D0000078002809D1384611300078002804D16B
:1007E000384610300078002827D07868002815D4C3
:1007F000032102468A431B4953588407E40EFF260F
:10080000A640B343A5401D43555002990140012025
:100810008840A2490860144908600EE08107C90EAB
:10082000FF228A40019C0440083C032084430C487A
:10083000235893438D401D4325500120B8610498EF
:1008400005B0F0BD02480349DA22034BFEF72EFB48
:10085000FD300100703101004D3101007C200100AC
:100860001CED00E000E400E000E100E0F0B58FB036
:100870000E900125002900D14BE0039304910592CD
:10088000002A00D145E00121EFF3108201910A40D6
:1008900002D1EFF3108172B64827029747437E4991
:1008A000CE19B5690023302D23D831461831C04602
:1008B0007D442D796D00AF44202426262626262649
:1008C00026262626262626265E2626262626262690
:1008D00026262626262626261826262626262626C6
:1008E000262626262626262618000223002A0CD095
:1008F0000CE0402D01D0802D05D10123002A04D029
:1009000004E020240C60002A00D162B61D46002BB2
:1009100002D028460FB0F0BD002575630399F1633E
:100920000499F162059931635B4CE35959691322CB
:10093000D202114205D0062199600F211962716916
:100940009960317C00290CD0F561099508950795CF
:1009500006950D950B9502210A91012810D01720BC
:100960000FE0717C9A6900292CD0952002439A618E
:1009700028460FB0F0BD30240C60002AC5D0C5E772
:100980001920049F0C907068002805D41F2108408E
:10099000019981404148016014209861B06806A91E
:1009A000F9F7BCF90E9802994143601880686158C4
:1009B0003B4A0092091D3A46059BF9F71FFA284663
:1009C0000FB0F0BD3436110602D580218A439A61FA
:1009D00031680025059A91422DD205955D694F2118
:1009E0004A0215421BD1E90502D4029CF24F0AE0EB
:1009F000596833685C1C3460029C6043EE4F3818C1
:100A0000C06AC1540E98214641437E18736B346B03
:100A1000A34238D234367B585D691542E3D00221B7
:100A20001962019EB10729433546E34CEFF310826A
:100A3000324006D008E02946019EEFF31082324092
:100A400002D1EFF3108372B6029B4343E01883692F
:100A50002024A34383618369002B05D0002A08D09A
:100A6000C26B002A0AD154E7034618331E60002ADD
:100A7000F6D162B6C26B002A00D14AE70EA89047B1
:100A800028460FB0F0BD2946059D019E3C46EFF378
:100A900010823240D5D0D7E7F894010280E200E01E
:100AA000F102010080B5012082020249024BFFF7EA
:100AB000DDFE80BD10CE0102A50A0100B0B582B0F6
:100AC00079208400E54D285D01A90870652080002B
:100AD0002818F2F781FF2F20C00028582919012279
:100AE000024BFFF7C3FE02B0B0BDC046BD0A010015
:100AF000F0B591B010900126002900D19BE003933E
:100B00000591002A00D196E007900121EFF31080B3
:100B10000291084002D1EFF3108172B6049248238B
:100B2000069307994B43D649C9188D690026302D85
:100B30006ED80C461834AD00374602A675593E46AD
:100B4000AF46C046190C0100210C0100250C010024
:100B5000250C0100250C0100250C0100250C0100CD
:100B6000250C0100250C0100250C0100250C0100BD
:100B7000250C0100250C0100250C0100250C0100AD
:100B8000250C0100090C0100250C0100250C0100B9
:100B9000250C0100250C0100250C0100250C01008D
:100BA000250C0100250C0100250C0100250C01007D
:100BB000250C0100250C0100250C0100250C01006D
:100BC000250C0100B70C0100250C0100250C0100CB
:100BD000250C0100250C0100250C0100250C01004D
:100BE000250C0100250C0100250C0100250C01003D
:100BF000250C0100250C0100250C0100250C01002D
:100C0000250C0100090C0100022600280CD00CE084
:100C1000402D01D0802D05D10126002804D004E00C
:100C200010252560002800D162B6002E069D944F45
:100C3000049C079802D0304611B0F0BD00268E62A9
:100C4000039A8A63059A0A624C620A7C002A0BD0D6
:100C50000C960B960A96099608960E9602220D920D
:100C600001282DD018202CE08A7C2831002A3BD086
:100C70000A68A24216D22B464343FA585469A40785
:100C800010D50868441C0C60F918096A085C1060EB
:100C90001098294641437A1811462831936A526ABE
:100CA0009342E8D345437859816982220A4382619D
:100CB000304611B0F0BD302525600028B4D0B4E72F
:100CC0001A200F90C86808A9F9F728F8109845432A
:100CD0007A597819C0683949009105992346F9F77E
:100CE0008DF8304611B0F0BDFB589A69140602D554
:100CF0008024A2439A610A680026049882422ED278
:100D00005D694F225202154207980AD002211962EA
:100D1000029EB10729431FE028315D6915423E4616
:100D2000F4D137465C69A40702D40699544E0AE010
:100D30000C68661C0E6006994843514E3018006AD4
:100D4000005D186010984143735871188C6A4E6AA0
:100D5000B442E1D329463E46069D494F01E0314663
:100D600007985A6A002AFCD1EFF31082029B1A40BE
:100D700002D1EFF3108372B64543781983691024CA
:100D8000A34383618369002B05D0002A09D0826BBD
:100D9000002A0BD14FE703461833029C1C60002A3F
:100DA000F5D162B6826B002A00D144E710A89047C3
:100DB000304611B0F0BDC046F8940102F1020100C6
:100DC000B0B5264900684A68824202D10D1D002054
:100DD00016E080228A58824203D10D4680350120D8
:100DE0000EE0FC228A58824203D10D46FC350220D7
:100DF00006E02F22D2008B5883422ED18D1803207B
:100E00007C2242438C18A068012814D0002824D1E9
:100E100040342046F3F7CFF901462046F3F7A1F915
:100E20002046F3F7C8F9002817D006C828680C4BED
:100E3000FFF75EFEB0BD40342046F3F7BCF9014633
:100E40002046F3F78EF92046F3F7B5F9002804D0D1
:100E500006C82868024BFFF74BFEB0BD88BE0102F2
:100E6000C10D010048214143054842189269D2064C
:100E700001D4002070474058416901200840704764
:100E8000F894010280B511480078C0011049097832
:100E9000890101430F480078400108430E49097851
:100EA000090101430D480078C00008430C49097846
:100EB000890001430B480078400008430A4909783B
:100EC0000143C8B2F3F728FC80BDC046109F010261
:100ED000DE9601022994010294EA0102C9AD0102E1
:100EE000119F010254A3010255A30102F0B587B07E
:100EF00001460127022505283A4600D02A4600204F
:100F00000929014600D01146C900374A54180E215C
:100F10000591615EFDF796FA1026A15F3846FDF750
:100F200091FA1227E15F2846FDF78CFA0695142501
:100F3000615F03200490FDF785FA0598235EA05FAA
:100F4000E15F625F00AD07C528A2069F3846049D99
:100F50002946FFF707F82046263004263146FBF7DE
:100F600031FF2620235E2820205E2A21615E2C226C
:100F7000A25E00900191029224A238462946FEF713
:100F8000F1FF27463E3738463146FBF739FF3E2012
:100F9000235E06983C5EB95F0622BA5E009401911A
:100FA000029221A207462E462946FEF7DBFF562471
:100FB0000D4D285FFBF718FF2B5F2C4621A238460A
:100FC00031463546FEF7CEFF264658363046FBF70B
:100FD000F7FE5820235EF05F00901FA23846294696
:100FE000FEF7C0FF07B0F0BDF4A00102546F462029
:100FF000616E742064656C617973202564202564BA
:101000002025642025640D0A0000000050446F4133
:101010002064656C61797320256420256420256433
:101020002025640D0A00000050446F41206761696B
:101030006E732025642025642025642025640D0A14
:101040000000000050446F4120616E742073706195
:1010500063652025640D0A0050446F4120616E676E
:101060006C65206F66667365747320256420256443
:101070000D0A0000F0B587B015467A4B1A680F24A8
:10108000A2432F783A431A60774C23462C3B774A89
:101090001A60049003462246283A12681207FAD5CD
:1010A000734E092F029306D9754A326072600C2F75
:1010B00009D175480FE0042F07D9704A3260704A91
:1010C0007260092F06D3714805E06A48306070608D
:1010D000694800E06B486E4A1060EB7AFF2B039181
:1010E00002D10020B0620AE003210B406948C05CD5
:1010F00040220243B2620220674AFEF733FF029F9A
:101100000021384605952A460B46FBF7E5FE0646C4
:101110000225032161A2284601913346FEF722FFF2
:1011200006963046FCF7ACFB01210498009108407C
:101130002CD13D4033D1604900283AD1002D1ED03A
:101140006548A062E062206360636448606264484E
:101150000860152085046E1C8E608D606424204616
:101160000F46F8F76BFD3E603D602046F8F766FDE0
:10117000281D386003215BA24E48FEF7F3FE059858
:10118000007BFAF7BDFF069807B0F0BD2E46054676
:101190000698FCF701FF284635463D40CBD02E4649
:1011A00005460698FCF774FB284635464249002858
:1011B000C4D04248086142484861424888611520CD
:1011C000C8614148016840220A43026007210803C0
:1011D000274B5A6982430098400310185861052232
:1011E000039842432A4803689818334E766B477831
:1011F0000F40995C0907490EC919CA03334B3340A4
:101200009A18C9015118324A89182B4A51632A4940
:10121000896B3822914382785207920E89180422F2
:101220000A4325498A63124B19690279019E3240AB
:10123000C0784007C00E80181F229143081818611B
:1012400055204003411C216020606420F8F7F6FC23
:10125000204A18483146039BFEF784FE1649002DAC
:101260008DD06DE7040400402C6000400004008035
:10127000000600400F040F04052B010003040304C3
:1012800000040004362C0100D4290100672D010060
:1012900044940102982E01009C31010050485920CD
:1012A000706172616D7320736574732025303878B6
:1012B0000D0A0000020800009060004012A83E00E5
:1012C0009DD79B5AD579BD49340200403F0080FF2D
:1012D000404000007E3101002008820002D50F004E
:1012E000020255007577625F72785F696E69740DEE
:1012F0000A00000080B522480021017022480078D1
:10130000C001204909788901014320480078400143
:1013100008431F490978C90001431E48007880002E
:1013200008431D490978490001431C4800780843D7
:10133000C0B2F3F7F1F980BD80B511480121017009
:1013400010480078800110490978C90101430F480D
:101350000078400108430E490978C90001430D484F
:101360000078800008430C490978490001430B4884
:101370000078084310210143C8B2F3F7CDF980BDCE
:1013800094EA0102DE960102109F010229940102F3
:10139000C9AD0102119F010254A3010255A301022C
:1013A000F0B581B01820FDF741FA1920FDF73EFA9B
:1013B000002420462146F7F7E5FF20462146FAF7AC
:1013C00023FE012603257F23304629462A46FAF7C5
:1013D0002DFF3046FBF7D2F802273846FBF75CFDBD
:1013E00030463146FCF7AAFD03A238462946FEF7EF
:1013F000B9FD204601B0F0BD7577625F6F70656E14
:101400000D0A0000F0B581B0164600910446002098
:1014100001273946FCF7BAFFEFF310853D4002D1B2
:10142000EFF3108072B62720400170430A21EEF7D7
:1014300051FE0246002C02D00020009901E002205B
:101440000021FBF7A1F80446FBF768F9002D00D155
:1014500062B6204601B0F0BDF0B581B01D460E4623
:101460000446022A09D1012738463946FCF78EFF87
:1014700000960022384629460FE017460120002139
:10148000FCF784FF012F04D1009600202946024674
:1014900003E00096022000210A462346FBF756F996
:1014A0000446FBF73BF9204601B0F0BD70B50028BB
:1014B00001D0012070BD0325A9020F4802680F4B1F
:1014C000535000249460012253030D4E3360BFF348
:1014D0004F8FBFF36F8F0B4E336003685A50847287
:1014E00004811020F8F7CAFA022007A22946FEF765
:1014F00039FD204670BDC0468895010251E5CC1AE1
:1015000080E100E080E200E057445420636C6F7398
:10151000650D0A000FB47CB50C0009AD01D0611E49
:1015200000E0002101910090074B6A462946089887
:1015300000F012F9002C02D0009A002111707CBC3E
:1015400008BC04B018470000911E01007CB51D4680
:1015500016460C0001D0611E00E0002101910090B0
:10156000054B6A462946304600F0F6F8002C02D0BA
:10157000009A002111707CBD911E01002021020CF7
:1015800001D010211046020A01D010460839020984
:1015900001D01046091F820801D01046891E42085A
:1015A00001D0881E7047081A704700000048704735
:1015B0000890010202E008C8121F08C1002AFAD1EF
:1015C00070477047002001E001C1121F002AFBD1C3
:1015D00070470000F0B51FB486B00998089A030D53
:1015E0000021024314D05148514A181850430514A1
:1015F0001198012810981AD0281A401C00264D4F27
:101600004D49009601910490002812DA444211E0FD
:101610001198012449A3012801D11098C1430698CB
:10162000119A84600360C26041600BB0F0BD40421B
:10163000E4E70446210500203F4A001C5141039184
:10164000029012E0E00707D032463B46019900982D
:10165000EFF708F80191009032463B4610461946D4
:10166000EFF700F806460F466410002CEAD1049804
:10167000039B0028029A0999089806DAEEF7F2FF10
:10168000019B009AEEF7EEFF05E0EFF753F8019BA0
:10169000009AEFF74FF804460E460022284BEFF76A
:1016A00015FC03D80020C043014607E00022254B6B
:1016B00020463146EEF724FFEFF7E8FB102409E05F
:1016C000002C0ADB0A220023EFF712FA079B3032C4
:1016D0001A55641E02460A43F2D11122641C079B6C
:1016E000121B1C19119B012B03D0012308430ED19F
:1016F0000AE0084304D0112010900020119077E7F1
:101700001098151A6D1E0BE01098824202DD00231E
:101710006D1C03E0824201DA00236D1E002BEED027
:10172000069811998260C16030C07EE701FCFFFF1E
:10173000104D0000000014400000F03F3000000099
:101740000000F0430000E03F30380A2801D20120B9
:101750007047002070470000FFB597B0064600258F
:1017600018E2252877D100242746FD49049400E09B
:101770000443761C32780120203A90400842F7D189
:1017800030782A280ED002223078014630390929D3
:1017900016D804990A235943303940181443761C4B
:1017A0000490F1E7189802C804911890002904DA0F
:1017B0000120400304434842049002200443761C65
:1017C00030782E2814D1042004437078761C2A28FF
:1017D00009D11898761C80C8189009E00A214F4357
:1017E000303FC719761C3078014630390929F5D9C0
:1017F00030786C2810D006DC4C281AD068280ED01F
:101800006A2817D104E0742813D07A2812D110E086
:101810000120400504430CE00121090501E00321FA
:1018200009050C437178814203D101200005241879
:10183000761C761C3078119066280BD013DC582863
:101840007DD009DC00287BD04528F6D04628F4D08E
:1018500047281AD1A5E118E0632835D0642870D054
:10186000652812D19DE170286CD008DC6728F1D082
:1018700069287BD06E280DD06F2806D1BAE0732876
:101880002ED0752871D0782859D01A9A1999904776
:101890006D1C7EE16002400F022809D003280DD0A4
:1018A0000428189801680DD00D60001D189070E193
:1018B0001898EA1701680D604A60F6E71898016801
:1018C0000D80F2E70D70F0E718986A460178117202
:1018D000001D18900020507202A80090012005E021
:1018E000189802C8189000200091C04361070DD5D8
:1018F000002101E00199491C0191B94212DA8142AB
:10190000F8DB009A515C0029F4D10BE0002101E0E2
:101910000199491C01918142FADB019A0099895C85
:101920000029F5D1019904981A9B471A2146384697
:10193000199A00F097FA0199401945180BE04FE009
:101940002CE113E04EE0009800990078491C0091CA
:101950001A9A199990470198401E0190401CF2D1A3
:10196000214638461A9B199A10E137E00A200021D7
:10197000009001916002410F022907D0189A01CA14
:101980001892C2179446032908D00AE01898C01D7F
:10199000C108C90005C91891944607E000B2C217F2
:1019A0009446042902D140B2C1178C4600226146F8
:1019B000944506DA0A460021404291418C462D2189
:1019C00002E0210504D52B216A461173012103E0B1
:1019D000E10701D02021F7E7029155E00A200AE053
:1019E000102008E010200090002104200443019101
:1019F000082703E008200021019100906002410FB8
:101A0000022907D0189A01CA189200229446032985
:101A100008D008E01898C01DC108C90005C9189170
:101A2000944603E080B2042900D1C0B200210291A3
:101A3000210729D51199702906D0009A1021019B00
:101A40004A401A4305D00EE040216A461173012135
:101A500008E06146014306D030216A4611731199AE
:101A6000517302210291009A0821019B4A401A43B6
:101A70000AD16146014301D1610705D530216A468B
:101A8000117301217F1E02911199582904D035A1AB
:101A90000E910DA90D910DE037A1F9E76146019B6B
:101AA000009AEFF725F80E9B8C469B5C0D9A521E10
:101AB0000D92137061460143F0D10D9805A9081AE3
:101AC00020300190600703D501200004844300E02A
:101AD00001270198874201DD381A00E000200199B2
:101AE00000904118029809180498401A0490E003E5
:101AF00006D421461A9B199A049800F0B3F94519A7
:101B0000002706E003A81A9AC05D199990476D1C3A
:101B10007F1C02988742F5DBE0030CD521461A9B17
:101B2000199A049800F09EF9451904E01A9A302099
:101B3000199990476D1C0099481E00900029F5DC0A
:101B400008E00D980D990078491C0D911A9A199981
:101B500090476D1C0199481E01900029F1DC63E15A
:101B60000928010030313233343536373839616273
:101B70006364656600000000303132333435363737
:101B800038394142434445460000000000F05AF90C
:101B90004519761C3078002800D0E2E528461BB0B5
:101BA000F0BD600700D406271898C01DC108C90001
:101BB00048680A680831C30FDB071891190001D083
:101BC0009CA108E0210501D59BA104E0E10701D01B
:101BD0009AA100E09AA1430011985B081091652832
:101BE0000CD006DC452809D046281DD0472841D115
:101BF00041E0662818D067283CD13CE00021112F35
